:10200000008000104B210000092100000B2100007E
:102010000D2100000F2100001121000074B9FEEF16
:102020000000000000000000000000002126000069
:102030001521000000000000C12600000527000057
:102040001B2100001B2100001B2100001B210000A0
:102050001B210000A5B100001B2100001B21000076
:10206000B5B100001B210000418E00001B210000C3
:102070001B2100001B2100001B2100001B21000070
:102080001B2100001B2100001B2100001B21000060
:102090001B2100001B2100001B2100001B21000050
:1020A0001B2100001B2100001B2100001B21000040
:1020B0003D2E00004D9200001B2100001B2100005E
:1020C0001B2100001B2100001B210000582A0100D9
:1020D00040000010B8000000582A010000C007208E
:1020E00000000000582A010000000010000000005D
:1020F000F8000010A462000000C0072000000000EB
:102100000000001000000000FEE7FEE7FEE7FEE72B
:10211000FEE7FEE7FEE7FEE7FEE7FEE70023934269
:1021200009D210B404680C600433043004319342C3
:10213000F8D310BC70477047002303E00022026010
:10214000043304308B42F9D3704710B50E4B07E0CF
:1021500003F10C049A6859681868FFF7DFFF2346FB
:102160000A4A9342F4D306E01C46596854F8080B17
:10217000FFF7E2FF2346064A9342F5D308F098FFA3
:1021800006F046FCFEE700BFCC200000F020000077
:1021900008210000FFFFFFFFFFFFFFFFFFFFFFFF22
:1021A000FFFFFFFFFFFFFFFFFFFFFFFFFFFFFFFF3F
:1021B000FFFFFFFFFFFFFFFFFFFFFFFFFFFFFFFF2F
:1021C000FFFFFFFFFFFFFFFFFFFFFFFFFFFFFFFF1F
:1021D000FFFFFFFFFFFFFFFFFFFFFFFFFFFFFFFF0F
:1021E000FFFFFFFFFFFFFFFFFFFFFFFFFFFFFFFFFF
:1021F000FFFFFFFFFFFFFFFFFFFFFFFFFFFFFFFFEF
:10220000FFFFFFFFFFFFFFFFFFFFFFFFFFFFFFFFDE
:10221000FFFFFFFFFFFFFFFFFFFFFFFFFFFFFFFFCE
:10222000FFFFFFFFFFFFFFFFFFFFFFFFFFFFFFFFBE
:10223000FFFFFFFFFFFFFFFFFFFFFFFFFFFFFFFFAE
:10224000FFFFFFFFFFFFFFFFFFFFFFFFFFFFFFFF9E
:10225000FFFFFFFFFFFFFFFFFFFFFFFFFFFFFFFF8E
:10226000FFFFFFFFFFFFFFFFFFFFFFFFFFFFFFFF7E
:10227000FFFFFFFFFFFFFFFFFFFFFFFFFFFFFFFF6E
:10228000FFFFFFFFFFFFFFFFFFFFFFFFFFFFFFFF5E
:10229000FFFFFFFFFFFFFFFFFFFFFFFFFFFFFFFF4E
:1022A000FFFFFFFFFFFFFFFFFFFFFFFFFFFFFFFF3E
:1022B000FFFFFFFFFFFFFFFFFFFFFFFFFFFFFFFF2E
:1022C000FFFFFFFFFFFFFFFFFFFFFFFFFFFFFFFF1E
:1022D000FFFFFFFFFFFFFFFFFFFFFFFFFFFFFFFF0E
:1022E000FFFFFFFFFFFFFFFFFFFFFFFFFFFFFFFFFE
:1022F000FFFFFFFFFFFFFFFFFFFFFFFFFFFFFFFFEE
:1023000010B4124B1A6882421AD359685C1884427E
:1023100003D1406801445960184641684418A242FC
:1023200012D10B4C2468A2420CD052681144416077
:102330001A6812680260984200D0186010BC70479A
:102340001346DFE70460F6E70260F4E708010010D7
:10235000F8000010324B1B6843B94FF0280383F399
:102360001188BFF36F8FBFF34F8FFEE770B5044640
:1023700005F0F8F82B4B1B681C420FD134B1083420
:1023800014F0070F02D024F0070408346CB1264B78
:102390001B68A3420DD3254B1D6810E005F07CF9A6
:1023A000002606F0A3F9304670BD05F075F9002649
:1023B000F7E705F071F90026F3E72B4615466A6842
:1023C000A24202D22A68002AF7D1154A1268AA420C
:1023D00003D105F061F90026E3E71E6808362A6894
:1023E0001A606B681B1B102B04D9281943606C60A2
:1023F000FFF786FF6A680C490B689B1A0B600C4953
:1024000009688B4201D20A490B60064B1B681343D3
:102410006B6000232B6005F03FF9002EC3D1C0E7AD
:10242000F8000010FC00001000010010080100106E
:102430000401001080B338B50446A0F1080550F837
:10244000042C164909680A4208D14FF0280383F387
:102450001188BFF36F8FBFF34F8FFEE750F8080C62
:1024600040B14FF0280383F31188BFF36F8FBFF3A0
:102470004F8FFEE722EA010244F8042C05F072F8BF
:1024800054F8041C064A13680B4413602846FFF7EF
:1024900037FF05F001F938BD704700BFFC000010A0
:1024A00000010010014B1868704700BF00010010C8
:1024B000324B1B68002B47D04FF0280383F3118861
:1024C000BFF36F8FBFF34F8FFEE72C4D2D684DB3D9
:1024D000954230D2294E35681344083B23F0070358
:1024E000336000265E601E6016469F1A57601360B8
:1024F00005B12A6073681944013400EBC4025368C3
:102500003BB3126812F0070F05D0D51D25F0070563
:10251000521B13442A46002CD7D1194D2A6000269D
:102520006E60D7E74FF0280383F31188BFF36F8FF6
:10253000BFF34F8FFEE74FF0280383F31188BFF3FB
:102540006F8FBFF34F8FFEE7F0B4024600242146A1
:10255000D5E70C4B19600C4B196041B94FF02803BB
:1025600083F31188BFF36F8FBFF34F8FFEE7074BE5
:102570004FF000421A60F0BC704700BFF800001036
:10258000080100100401001000010010FC00001000
:1025900082B0002301930D4B1B68B3F1FF3F08D0BD
:1025A0004FF0280383F31188BFF36F8FBFF34F8F72
:1025B000FEE74FF0280383F31188BFF36F8FBFF35B
:1025C0004F8F019B002BFCD002B0704740000010E1
:1025D00006480068006880F3088862B661B6BFF3F9
:1025E0004F8FBFF36F8F00DF00BF000008ED00E0EA
:1025F0004FF0807340F8043C21F0010140F8081CC2
:10260000034B40F80C3C40F8202C4038704700BF8A
:1026100091250000FFFFFFFFFFFFFFFFFFFFFFFF10
:10262000074B19680868B0E8F00F80F30988BFF31A
:102630006F8F4FF0000080F311884EF00D0E704741
:10264000740400104FF0280383F31188BFF36F8FD9
:10265000BFF34F8F0A4A136801331360012B00D078
:102660007047084B1B6813F0FF0FF9D04FF0280399
:1026700083F31188BFF36F8FBFF34F8FFEE700BF67
:102680004000001004ED00E0094B1B6843B94FF017
:10269000280383F31188BFF36F8FBFF34F8FFEE7DB
:1026A000013B034A13600BB983F31188704700BFE5
:1026B00040000010FFFFFFFFFFFFFFFFFFFFFFFFD6
:1026C000EFF30980BFF36F8F0D4B1A6820E9F00F0D
:1026D00010602DE908404FF0280080F3118805F0C4
:1026E0007BF84FF0000080F31188BDE808401968BE
:1026F0000868B0E8F00F80F30988BFF36F8F704768
:102700007404001008B54FF0280383F31188BFF359
:102710006F8FBFF34F8F04F033FF18B1034B4FF0AF
:1027200080521A60002383F3118808BD04ED00E095
:10273000084A0023136008490B60084B1B680849CE
:10274000A1FB03135B09013B06490B6007231360E0
:10275000704700BF10E000E018E000E09863001050
:102760001F85EB5114E000E010B582B0274B1A78BA
:10277000D2B20192FF221A701B78DBB28DF80330BF
:102780009DF8033003F02803214A1370214B0722E0
:102790001A6009E01F4A1368013B13609DF803307B
:1027A0005B00DBB28DF803309DF8033013F0800F2F
:1027B000F0D1184B1B68022B08D04FF0280383F38D
:1027C0001188BFF36F8FBFF34F8FFEE71B0203F437
:1027D000E063104A1360019BDBB20C4A13700E4B8E
:1027E0001A6842F478021A601A6842F078421A6055
:1027F000FFF79EFF0024094B1C60FFF7E9FE04F081
:10280000EBFFFFF7C5FE204602B010BD00E400E07C
:10281000100100101401001020ED00E04000001035
:10282000EFF305830F2B0FD9104A9B5CDBB2104AE4
:1028300012789A4208D94FF0280383F31188BFF326
:102840006F8FBFF34F8FFEE70A4B1B6803F4E06303
:10285000094A1268934208D94FF0280383F311887C
:10286000BFF36F8FBFF34F8FFEE77047F0E300E0D9
:10287000100100100CED00E01401001082B00E4BAE
:102880001A6892090D4BA3FB0232920A4FF47A7335
:1028900003FB00F0009006E000BF019B01330193B1
:1028A000019B9A42F8D8009B013B009313B100238F
:1028B0000193F5E702B07047986300101791650225
:1028C00010B504464FF0A040D0F82C21032392B25B
:1028D0000749098809F017FE022807D0044B1A8817
:1028E000044B1B6843F83240012010BD0020FCE778
:1028F0004A01001028010010484B1B7803B17047B3
:1029000010B51820FFF726FD454C20600C20FFF77E
:1029100021FD444B18602020FFF71CFD424B18603E
:102920002020FFF717FD414B186023681BB33D4A79
:10293000126802B33C4A1268EAB1E0B118220021E1
:1029400018460BF06EFA0C220021364B18680BF07B
:1029500068FA20220021344B18680BF062FA20221A
:102960000021324B18680BF05CFA0024304B1C80BD
:10297000304B1C801FE04FF0280383F31188BFF316
:102980006F8FBFF34F8FFEE719214FF4107000F0E7
:1029900033FBA0B18069E300234A1268D11842F8E2
:1029A0003400254A4A60214A11680B44002241F84C
:1029B00034205A600134032CE6DD002316E04FF08A
:1029C000280383F31188BFF36F8FBFF34F8FFEE7A8
:1029D000134A126802EBC301184842F83300002280
:1029E0004A601049096841F823200133022BEFDDCA
:1029F00003230C4A12680A4909684FF0A04009F005
:102A000048FD0423094A1268074909684FF0A040AD
:102A100009F05CFD014B01221A7010BD400100104D
:102A2000280100102C0100102001001024010010CA
:102A3000480100104A0100103F020080EFBEADDEE9
:102A400008B509F091F910F0080F14D00F4B1B686E
:102A5000834210D00D4B186010F0100F0CD04FF0C7
:102A6000A0434FF480729A6110F0200F09D14FF00B
:102A7000A04009F0F4FC08BD4FF0A04300229A6189
:102A8000F2E74FF0A04009F0D0FCF4E74401001059
:102A9000F0B583B04FF0A043D3F8E42F4FF0FF32EE
:102AA000C3F8E42F624B282283F81C234FF0805296
:102AB0001A60AAE05F4A137803F0FE0313705D4BBF
:102AC0001B7813F0020F78D15A4B1B78002B00F0C3
:102AD0009680584B1B7813F0010FF0D001238DF82E
:102AE00000300023019321E019214FF4107000F011
:102AF00083FA0746002843D0304600F03CFD0646E6
:102B0000C461B9694C4B1A884C4B1B6843F83210AE
:102B100001900021684600F0F7FF002837D04FF001
:102B2000A04009F038FD444B18802B465A1CD5B202
:102B3000022BC4D84FF0A040D0F8141104233E4A11
:102B4000128889B209F0DFFC0028B3D03A4B1B8809
:102B50003A4A126852F83360394A126852F8332000
:102B6000C2F30A03DC1E04D0002ABDDA12F0806F23
:102B7000BAD14FF0A04009F00EFD2F4B1880D4E7DA
:102B80004FF0A04009F007FD2B4B1880CDE73046F1
:102B900000F010FAC3E700231A46194629480068D6
:102BA00003F0EAFF284A136801331360274A1378B9
:102BB0000133DBB21370022B17D8244B1A7891B271
:102BC0004FF0A043D3F82C319BB2994211D0204B47
:102BD00053F822000028DED000F0ECF91B4B1A78E5
:102BE0001B4B002143F82210D5E7134600221A7030
:102BF000E3E7104A137803F0FD03137064E704F071
:102C0000B9FC144B1B6883420CD3FFF74BFC124BEF
:102C100018604FF0A043D3F82C313221012005F089
:102C2000DDF851E732300B4B1860FFF709FFECE796
:102C300000E100E0410100104801001020010010F7
:102C4000240100105401001018010010420100106E
:102C5000580100104C0100101C01001010B582B08A
:102C600001214FF0A04009F00AFB38494FF0A04085
:102C700009F06EFB012201464FF0A04009F046FB2F
:102C8000334B59791A7942EA01224FF0A044226469
:102C9000D9789A7842EA012262645A781B7843EA2A
:102CA0000223A36400231A462A49012008F0ECFFFE
:102CB000FFF722FED4F8003143F00203C4F80031DC
:102CC000D4F8003143F00103C4F80031236843F025
:102CD00001032360D4F8003123F08003C4F80031ED
:102CE000D4F8003243F02203C4F800321A4B0193A7
:102CF0000623009300234FF496721849184804F0F5
:102D0000BBFB40B94FF0280383F31188BFF36F8FEB
:102D1000BFF34F8FFEE70446124B1B6823B1FFF74A
:102D20008FFE204602B010BD0221084603F003FFCB
:102D30000C4B18600028F2D14FF0280383F3118860
:102D4000BFF36F8FBFF34F8FFEE700BFA0252600B4
:102D50008C0000107D280000500100105815010063
:102D6000912A00005401001070B584B004460E464C
:102D70000A230393C369002B48D02B4B1868002803
:102D80004BD00A2104F0C8F8012802D000231D46C8
:102D90003EE001A804F070FEA069FFF791FD38B98C
:102DA00003A901A804F090FE0028F5D0012300E05B
:102DB00000230BBB3EB14FF0A043D3F828319BB2A8
:102DC0001A4A42F82340E369013BC3F30A03184D52
:102DD0002988184A126802EBC10243F0404353604D
:102DE0004FF0A04009F0B9FB2880134A1368013363
:102DF000136001231D460BE000231A4619460A48BA
:102E0000006803F0B9FE00231D4601E000231D46C3
:102E100003B92EB9284604B070BD00231D46F7E75C
:102E2000204600F0C7F8F5E75401001058010010E3
:102E30004A010010280100103401001010B582B0C2
:102E40000023019320E02B4A1368013313602A4AC0
:102E5000137843F00103137001A9284B186804F09C
:102E6000F9FF1DE0264A136801331360224A1378E4
:102E700043F00203137001A9204B186804F0EAFF25
:102E800011E014F0100F1BD14FF0A043D3F8E04F26
:102E900024B34FF0A043C3F8E84F14F0080FD2D189
:102EA00014F0800FDED114F0010FEAD04FF0A042F1
:102EB000136843F480631360124B00221A80E0E72A
:102EC000114A1368013313604FF0A042136843F4B2
:102ED000807313600D4B00221A80D5E7019B3BB134
:102EE0000B4B4FF080521A60BFF34F8FBFF36F8FC1
:102EF00002B010BD3001001041010010500100105F
:102F000038010010480100103C0100104A01001077
:102F100004ED00E038B51E4B1B682BB11C4B1B6841
:102F2000002B33D0012038BD0C21084603F003FEEE
:102F3000174B186040B94FF0280383F31188BFF393
:102F40006F8FBFF34F8FFEE7124904F0C7F8104BA5
:102F50001B68002BE2D0104803F084FC00250FE032
:102F6000EB002B449A000D4C14440023A36120462F
:102F700003F083FCE4602146074803F08DFC013533
:102F80000B2DEDDD064B0C221A60C7E70020CAE7C7
:102F90002C03001064150100680100107C01001072
:102FA0006401001020B108B50A38FFF743FA08BDE4
:102FB0007047FFFF38B504468069FFF7F3FF002331
:102FC000A361FFF73FFB2569094B9D4203D02146D2
:102FD000184603F055FCFFF757FB054B9D4206D002
:102FE00000231A4619460348006803F0C5FD38BDA2
:102FF000680100102C03001070B5431E402B00D850
:103000004220841C14F0030F02D044F00304013466
:103010001B4B186803F080FF01282DD1FFF712FB2E
:10302000184EF368DD68284603F050FCFFF72CFBD0
:103030003368154A12689A4201D9134A1360AB6982
:1030400043B14FF0280383F31188BFF36F8FBFF3B1
:103050004F8FFEE78CB104F10A00FFF77BF9A861FE
:1030600020B92846FFF7A6FF002506E00560AB69FA
:103070000A33AB61EC6100E00025284670BD00BF5B
:103080002C03001068010010640100100023052BC0
:1030900021DC10B503EB4304A200104CA25882427D
:1030A00004D00133052BF5DD002010BD03EB4302F6
:1030B000900022460244D27A5AB1084603EB4303F9
:1030C0009A0021461144062204310AF0A6FE01208E
:1030D000EBE70220E9E70020704700BF3003001053
:1030E0002DE9F04705460E46474B5B69474A526853
:1030F0005940114246D0002B40F084804FF0FF0928
:103100004FF0000A4FF0FF37B84654460EE0002D4E
:1031100041D004EB440293003D481844062229465E
:1031200004300BF0FFFB08B3A0460134052C33DC60
:1031300004EB44029300364AD358B342E7D055B16A
:1031400004EB440293003248184406222946043016
:103150000BF0E8FBA0B104EB44039A002C4B1344A2
:103160009B7A4B45E1D29946A246DEE7284A6300A6
:10317000181981001144962088720123CB7241E016
:103180002746D2E74FF0FF094FF0000A4FF0FF3714
:10319000B8465446CAE7A046002F1FDBB8F1000F1F
:1031A00012DA07EB47029300194AD650EDB9B8F18D
:1031B000000F27DA164A7B00D81981001144052038
:1031C00088720023CB721DE008EB480293000C22AA
:1031D00000210F4818440AF024FEE2E7B8F1000F7E
:1031E00001DB4746DDE75746DBE77C00E3199E003D
:1031F000164406222946301D0AF00FFE9623B372AC
:103200000123F372BDE8F08744000010B4030010FE
:103210003003001070B582B0044600F11C05042292
:1032200029460DEB02000AF0F8FDD4F826602A4B7F
:103230005B69002B4DD0A28AB2F5807F04D0B2F535
:10324000007F3FD0002045E0B34201D0002041E0A4
:10325000019904F11600FFF743FF002323750223B1
:103260006375019BB34218D0062204F1160104F1E4
:1032700020000AF0D2FD019BC4F82630164E06222B
:10328000314604F116000AF0C8FD042206F11401CB
:1032900028460AF0C2FD02201CE006220F49A018B1
:1032A0000AF0BBFD0622002104F120000AF0B9FD5E
:1032B000002384F8263084F8273084F8283084F8F6
:1032C0002930DBE7019904F11600FFF709FF002020
:1032D00000E0002002B070BD44000010A8150100FD
:1032E00038B5054608462C68B4F1FF3F18D0124B9C
:1032F0001B699C4214D0114B5B69C3B10E4A5268E2
:103300006340134203D00C4B9B6803B11C4684B14D
:1033100001462046FFF7BAFE034630B92C6004E0B0
:10332000062207490AF079FD0123184638BD022319
:10333000FBE70223F9E700BFB403001044000010CC
:10334000A815010070B50546846926220E4920465D
:103350000AF063FD0D4E06223146A0180AF05DFD0D
:103360000622314604F116000AF057FD042206F148
:10337000140104F11C000AF050FD6B69C4F82630FA
:103380002A23EB6170BD00BF7015010044000010DE
:1033900038B5054600212A20FFF72EFE38B1044635
:1033A0004561FFF7CFFF01212046FFF7DDFC38BD67
:1033B00010B5002411E0204A1058FFF7E9FF04EB94
:1033C00044039A001C4B13449B7A2BB904EB440230
:1033D0009300194A0021D1500134052C1ADC04EB6A
:1033E00044039A00144B13449B7A002BF4D0013B06
:1033F000DBB21046104A02449372D27A002ADAD025
:10340000032BDCD804EB440293000B4AD058FFF79F
:10341000BFFFD4E704F0AEF80446084B1B681BB1AD
:10342000C31AB3F5FA6F05D9054B5869FFF7B0FF1A
:10343000024B1C6010BD00BF300300107803001069
:10344000440000100C4B1B7813F0010F07D00A4BFF
:10345000DB68B3F57A7F09D2074B1B6901E04FF4B3
:103460007A73064AD068984203D270474FF47A7351
:10347000F7E71846F9E700BF80030010DC030010EF
:10348000002380F82230D0F81A30C0F81E30084BE4
:103490005B69C0F81A30838C4FF6F672934204D9F8
:1034A00003F5847383840220704708338384FAE72A
:1034B0004400001008B590F82230082B02D1FFF725
:1034C000DFFF08BD0020FCE738B504460D46043098
:1034D00004F0D2FAE56045B123786FF3410323701D
:1034E000237843F00103237038BD237843F00203AF
:1034F0002370F5E708B50161FFF7E6FF08BD037823
:1035000013F0010F10D010B5044613F0020F05D1CF
:1035100000F10C01043004F0D7FA38B121692046DB
:10352000FFF7D2FF012010BD002070470020FAE70E
:1035300008B504F00FFB044B1B68834201D0002048
:1035400008BD0120FCE700BFAC03001038B50546FC
:1035500008460021FFF750FD044650B16B694361F6
:103560002B8C03846B8C4384EA69A96980690AF017
:1035700054FC204638BD38B1A0F10A0212F0030F06
:1035800004D150F80A0C70470020704700207047A3
:1035900010B50446062201460C480BF0C3F948B9A1
:1035A000A289130A43EA02239BB2B3F5C06F0AD87B
:1035B000002010BD0622214605480BF0B3F9002873
:1035C000EED00020F5E70120F3E700BF4400001033
:1035D000A815010008B5064B01221A60002005F06D
:1035E00087F84FF47A710348FFF784FF08BD00BFE6
:1035F000D003001080030010F0B40502ADB245EA1C
:103600001025ADB22B4600260C4601F0030011F048
:10361000010705D022B114F8011B61F30F26013A0E
:10362000411E012906D922F0030CACF10C0CA44474
:10363000002508E0012AF6D934F8020B2B18023ACB
:10364000F1E701F110042146A44510D920681818AB
:1036500000D301354B68C01800D301358C680019C0
:1036600000D30135CB68C318EBD30135E9E798B235
:1036700000EB1340431902F00E00014402E034F85D
:10368000020B0344A142FAD812F0010F02D02278B3
:1036900062F30706981983B203EB10439AB202EB68
:1036A00013432FB11A0292B2C3F3072042EA000378
:1036B000180220F07F4222F0FF02C3F307201043DC
:1036C00080B2F0BC7047F8B5837B03F00F039B001A
:1036D000A3F114060644C47D112C08D0062C2CD06E
:1036E000621ED2B2012A48D806F1240501E006F193
:1036F000280529B300222A80B0F810C04FEA1C2206
:1037000042EA0C2292B2D21A072A39D9C3F51073B1
:10371000934238D30F46022C1AD806F1220100201A
:10372000FFF76AFFC04383B2EFB91BB3180A40EA40
:10373000032080B237B3288024E006F13205D8E7B1
:103740002A88002AD8D1112CD6D14FF6FF7019E063
:1037500093B22344083200F11A0198B2FFF74CFFEC
:10376000C04383B2E0E7002BE0D1112CDED14FF64D
:10377000FF73DBE74FF6FF73D8E744F2213001E037
:1037800041F23420F8BD41F23420FBE738B5D0F8DF
:103790001E40838A23F0F0039BB23BBB837B453BF7
:1037A000DBB20A2B24D8164B5B69A34207D0B4F1D5
:1037B000FF3F04D0134D2D69A54200D0D3B90C466C
:1037C000C37D012B08D000F10E010020FFF714FF8C
:1037D0004FF6FF7398420FD10021A069FFF773FFE6
:1037E0004FF6FF73984209D1012038BD0020FCE755
:1037F0000020FAE70020F8E70020F6E70020F4E7D1
:1038000044000010B40300102DE9F04706460C46B2
:1038100000F10E0A857BAD0005F03C0590F817809D
:103820002A46FFF7B3FF074601282CD1142D0FD9E4
:10383000A5F11409E269A2EB0902223A0AEB05019B
:1038400006F122000AF0EBFAE369A3EB0903E36156
:10385000B8F1110F04D0D6F81A10B01DFFF740FCD4
:10386000B8F1060F27D0B8F1110F0FD0B8F1010F42
:1038700009D1A069D6F81E20144B5B699A4202D187
:10388000FFF718FE07463846BDE8F087A269D18CDD
:103890000B0A43EA01239BB2083BE361538C238468
:1038A000D2F81A306361918C204602F081FE012823
:1038B000E9D10327E7E7204602F074FC012800D194
:1038C0000327034A136801331360DCE74400001048
:1038D000D403001070B504460D4681B174B1A069DF
:1038E000861D062231460AF098FA0622074930461C
:1038F0000AF093FA29462046FFF736FA70BDC169EF
:10390000FFF724FE04460125E8E700BF440000104D
:1039100040B94FF0280383F31188BFF36F8FBFF3D3
:103920004F8FFEE710B582B004468069FFF730FE86
:103930008DF80700A0699DF80730DBB2012B0AD093
:103940009DF80730DBB2022B1AD0032B1CD0204687
:10395000FFF730FB18E08389082B07D0B3F5C16F60
:103960000AD1FFF757FC8DF80700E9E72146FFF77A
:103970004BFF8DF80700E3E700238DF80730DFE702
:1039800001212046FFF7A6FF02B010BD08B5FFF7E2
:10399000BFFF08BD014B1868704700BFB00300109F
:1039A000F0B583B004460F4616461D46FFF7F2FFFA
:1039B00040B14FF0280383F31188BFF36F8FBFF33B
:1039C0004F8FFEE7484B1B6843B14FF0280383F34A
:1039D0001188BFF36F8FBFF34F8FFEE7434B1B6818
:1039E00043B14FF0280383F31188BFF36F8FBFF308
:1039F0004F8FFEE700220821112003F078F83A4BA0
:103A0000186040B94FF0280383F31188BFF36F8F1C
:103A1000BFF34F8FFEE7364903F060FBFFF77AFAFA
:103A200001285AD1E278A3781B0443EA0263627842
:103A300043EA0223227813432E4C2360F978BA78A4
:103A4000120442EA0162797842EA012239780A4393
:103A50006260F078B178090441EA0061707841EA67
:103A6000002130780143A160E878A978090441EA8F
:103A70000061687841EA002128780143E16063EA47
:103A800002032361142221461B480AF0C6F9236869
:103A90001A4A5361A26862B1616853400B4208D070
:103AA0004FF0280383F31188BFF36F8FBFF34F8F5D
:103AB000FEE70622089911480AF0AFF900F0BAFAB9
:103AC0000A4B01930523009300234FF461720C49C4
:103AD0000C4803F0D1FC03B0F0BD034C206803F0A8
:103AE00027FB00202060F6E7CC030010AC03001099
:103AF00098150100B4030010980300104400001052
:103B0000A0150100713C000038B504460D46FFF7D2
:103B100041FF10B994F9003003BB94F90030052B34
:103B20000BD0FFF705FD012814D000232A462146BB
:103B30000B48006803F020F838BD0A4A137843F0B8
:103B400002031370064B186803F0B4FA0028E8D09B
:103B50000120F1E7002DE8D00025E6E70020EBE7A3
:103B6000CC030010DC03001008B500210648FFF765
:103B7000CBFF012803D0054B01221A6008BD034B7F
:103B800000221A60FAE700BFB0150100C803001058
:103B900008B50F4B1A786FF300021A700D4B1B68B3
:103BA000012B0DD00B4B01221A60FFF757F80128AB
:103BB0000AD04FF4967003F0E9FDFFF7D5FF08BD7A
:103BC000012004F095FDEDE7FFF704FDF7E700BFE6
:103BD000800300109403001000B583B08DF800003E
:103BE000002101916846FFF78FFF03B05DF804FBE9
:103BF00010B51948FFF783FC38BB184B186803F061
:103C000059FA30BB012403F0B5FC154B1B683BB1DE
:103C1000C31A03EB83035902124A13680B4413605F
:103C20000F4B18601048FFF76AFC104B1B6803B17C
:103C300004B948B1204600F083FE01460A48FFF768
:103C400043FC0A4B00221A6010BD0220FFF7C4FF9C
:103C5000D3E70024D7E700BF80030010CC03001097
:103C6000D803001020040010DC030010D40300105F
:103C700010B584B0FFF778FF64213E48FFF73AFCA7
:103C80003D4B01221A6008E03C4B00221A60FFF70E
:103C90007FFF3B4B1B68002B68D1FFF7A9FFFFF7A5
:103CA000D1FB04A9FF2301F8083D0246354B1868F3
:103CB00003F086F89DF908300A2BEAD801A252F8E1
:103CC00023F000BF893C0000F13C0000F93C0000FB
:103CD000353D0000933C0000453D0000513D000093
:103CE000933C0000FF3C00002D3D00003D3D0000E6
:103CF0000398FFF74BFECCE7FFF75AFBC9E7039C9D
:103D000000230193A18C0A0A42EA0122ADF80220A5
:103D1000A38408226946204600F0CEFA236843F0C7
:103D200010032360204600F0C8FBB2E7039800F0C0
:103D300033FBAEE7039802F0CFFBAAE7039801F04C
:103D400043F8A6E70B4A137843F002031370A0E789
:103D5000039C204602F0C0FA00289AD0236843F062
:103D600004032360204600F0A8FB92E7FFF7FCFE67
:103D700093E700BFDC030010B0030010D003001075
:103D8000C8030010CC030010431E13F1030F0BD81F
:103D90000AB1836953B190F82730C9B28B4201D080
:103DA00000207047012070470020704700207047B6
:103DB000808C0C4BDB6800E05B680B4A93420FD0B1
:103DC000DA6892F853100129F6D1918C8142F3D12F
:103DD000B2F84E100029EFD00139A2F84E1070470A
:103DE000704700BFF4030010FC030010F8B507464D
:103DF0000D4616461C46FFF7CDFD00283BD0022F8E
:103E000008D04FF0280383F31188BFF36F8FBFF3FF
:103E10004F8FFEE71A4B9B68B3F1FF3F08D04FF07E
:103E2000280383F31188BFF36F8FBFF34F8FFEE733
:103E3000144B9B68B3F1FF3F08D04FF0280383F386
:103E40001188BFF36F8FBFF34F8FFEE7112E07D19D
:103E5000022D03D101204C2323600DE00020FAE75E
:103E6000062E0AD1012D04D101204FF49C7323604A
:103E700002E00020F9E70020F8BD0020FCE700BFC9
:103E800008040010F403001038B505460C46FFF78F
:103E900081FD60B16DB105F10802E868904204D07F
:103EA0000368A34202D04068F8E7002038BD002034
:103EB000FCE70020FAE7FFFF70B506281FD1114E7E
:103EC0000125114A32F8153001339BB222F8153022
:103ED000B3F57F4F04D313464FF4414223F8152026
:103EE000094B33F815301C0A44EA0324A4B22146D6
:103EF0003046FFF7C9FF0028E3D1204670BD034ECE
:103F00000025DEE7F4030010F003001008040010A1
:103F100010B584B004460A238DF8083003901021B0
:103F2000006802F017FC4FF0FF3102A8FFF7ECFD2C
:103F300058B14FF0FF330093002301221021206875
:103F400002F082FBA06804B010BD0020FBE7FFFF79
:103F5000F8B505460F46C9B1446EC36D6BB9A3F100
:103F60003333A3FB04239B08C365B0F84A20934274
:103F700003D2B4EB420F00D3C2652B6E3BB9A30052
:103F8000124AA2FB03239B082B6600E0846E0434D4
:103F900024F0030404F11400FEF7DCF9064640B1F6
:103FA0001422002109F03DFF34616FB92E673046BD
:103FB000F8BD95F8423043F0080385F842300821F7
:103FC000284601F02BFCF2E7EE66F0E7CDCCCCCC36
:103FD00038B504460D4601220621FFF7D5FEC8B1CB
:103FE00094F8423013F0080F17D194F85330BBB156
:103FF00094F8413013F0400F15D1B5B1236F0BB1D8
:10400000012011E000212046FFF7A2FF236F73B1CA
:10401000012009E06FF0150006E06FF00B0003E0EF
:104020006FF07F0000E0002038BD0020FCE76FF05B
:104030000B00F9E708B5074802F014FC064B4CF2F8
:1040400001021A800549012008605A80044802F0E4
:1040500009FC08BD08040010F00300102004001043
:10406000F403001070B582B0154601ABFFF7BEFE39
:1040700020B94FF0FF34204602B070BD0198FEF722
:1040800069F90446B0B302F0D2FA064638B3019A91
:104090000021204609F0C5FE6660112D25D004F1EF
:1040A000080002F0EAFB64614FF0FF33E361236232
:1040B000022384F8263084F82750062DDBD140F205
:1040C0000A23A4F84A30A4F84C3040F21443636643
:1040D000A3660123C4F8CC30C4F8D030CBE7204627
:1040E000FEF7A8F94FF0FF34C5E704F1380002F0FD
:1040F000B9FBD4E74FF0FF34BDE710B50C20FEF755
:1041000029F9044638B10C22002109F08AFE02F098
:104110008EFA206008B1204610BD2046FEF78AF9CD
:104120000024F8E758B110B5044689B94FF02803C8
:1041300083F31188BFF36F8FBFF34F8FFEE74FF00C
:10414000280383F31188BFF36F8FBFF34F8FFEE710
:1041500002F00F03C26A1343C36213F00F0F05D0BE
:104160000846A16200234B60FFF7D2FE10BD034654
:1041700048B189B94FF0280383F31188BFF36F8FDB
:10418000BFF34F8FFEE74FF0280383F31188BFF38F
:104190006F8FBFF34F8FFEE702F00F00DA6A22EA5B
:1041A0000002DA6212F00F0F01D09962704700220C
:1041B0009A62704748B189B94FF0280383F3118898
:1041C000BFF36F8FBFF34F8FFEE74FF0280383F3EA
:1041D0001188BFF36F8FBFF34F8FFEE7826A8A4269
:1041E00003D1006B00F00F0070470020704740B90A
:1041F0004FF0280383F31188BFF36F8FBFF34F8F06
:10420000FEE730B587B00446039104A803F034FC00
:104210002068039B009300231A460F2102F014FA32
:10422000012363602046FFF773FE0021206802F03F
:1042300091FA054628B903A904A803F045FC002813
:10424000E6D0284607B030BD431E13F1030F26D831
:1042500083693BBB10B584B008238DF80830039008
:10426000D1B14A8822FA03F343EA02238384044645
:104270004FF0FF3102A8FFF747FCB0B14FF0FF331A
:104280000093002301221021606802F0DDF9A36988
:1042900073B1002004B010BD00238384E7E76FF002
:1042A000150070476FF0150070476FF08B00F1E755
:1042B0006FF01500EEE7FFFFF0B583B005460C4642
:1042C0001F4690F8270006280DD0254E6DB1B5F198
:1042D000FF3F13D14FF0280383F31188BFF36F8F93
:1042E000BFF34F8FFEE71F4EF0E74FF0280383F335
:1042F0001188BFF36F8FBFF34F8FFEE71CB9002308
:10430000ADF802306C4644B94FF0280383F31188AE
:10431000BFF36F8FBFF34F8FFEE76388C3B11FB149
:1043200095F82730062B04D061883046FFF7ACFDA6
:1043300090B96388AB606288130A43EA0223AB84B6
:1043400005F10801304602F09BFA002003B0F0BDF1
:10435000FFF7B2FD6080E2E76FF06F00F6E700BFA5
:1043600008040010F403001000B583B009238DF891
:1043700000300190013810F1030F03D9002003B081
:104380005DF804FB00216846FFF7BEFB08B1012081
:10439000F5E74FF0FF30F2E738B5044690F82730E4
:1043A000062B12D0A3691BB104F1080002F08EFAAB
:1043B00094F82730112B1CD0606808B102F033FA52
:1043C0002046FEF737F8002038BDC06E08B1FEF772
:1043D00031F8206F08B1FEF72DF82046FFF7E8FC12
:1043E000E0E7636CDD68284602F070FA2846FEF7C5
:1043F000E1FDA36B002BF4D1DEE7FFFF08B501461A
:104400000848FFF741FD58B1C06800B108BD4FF042
:10441000280383F31188BFF36F8FBFF34F8FFEE73D
:104420000020F3E70804001070B483B001260025D3
:104430001AE003EB830359005318303B0134227810
:10444000A2F13001C9B20929F3D9844211D0FF2B5E
:1044500013D802A9294401F8043C022D0BD82E2AB6
:1044600016D1601C5EB10135032D08D80446002327
:10447000E5E70026EBE72046F4E720460026037830
:1044800003B10026042D06D0002003B070BC704795
:1044900020460026F3E70EB90020F6E79DF8073026
:1044A0009DF80600000440EA03609DF8053040EAEC
:1044B00003209DF804301843E7E710B50446836AEB
:1044C0001BB10168C1F3032149B9216801F07F01E3
:1044D0002160606800B149B90023236010BD026B00
:1044E0000A430263186802F058F9EEE702F055F942
:1044F000F2E72DE9F04389B005460F4691460122C7
:104500000621FFF741FC002878D095F8403013F0E1
:10451000080F0AD195F85330012B02D04FF0FF3429
:104520006EE04FF0000846462DE04FF0000846468A
:1045300029E02C462FE003F0AFF80024B8F1000F7B
:1045400008D006238DF80C3004954FF0FF3103A8F6
:10455000FFF7DAFA002C53D13EB9EB690793002B31
:104560004ED005A803F088FA012607A905A803F094
:10457000ABFA002844D1079B0093002301220421B9
:10458000686802F061F802F0EDFF95F8403013F032
:10459000080FCED16C6D64B100236B6594F8403088
:1045A00013F0020FC7D094F840306FF3410384F842
:1045B000403003F071F8002CC0D08FB1A26B130211
:1045C00003F47F0343EA0263110A01F47F410B43C2
:1045D00043EA12637B60A28F130A43EA02237B80C3
:1045E000B9F1000F02D00823C9F8003095F8403027
:1045F00013F0080FA2D14FF00108A2E74FF0FF34EB
:10460000204609B0BDE8F0832DE9F04786B00446A6
:10461000894690461E4601220621FFF7B5FB002879
:1046200000F09680E36E002B5FD09D681A681B69CE
:104630001D44AD1AAB4200D8ED1A0027002D36D02C
:1046400006E094F8423013F0080F50D06FF00B05DD
:10465000002D16DD16F0010F4CD0E26E1068956843
:10466000136811690D44EB1A994200D85B1A02F1E4
:1046700014010144C9F8001015692D1A9D4228BF84
:104680001D46284606B0BDE8F08705A903A803F03B
:104690001BFA82460028DBD1059B009300230122F0
:1046A0006121606801F0D0FFE36E5546A3B994F82C
:1046B0005330002BC5D0083B012BC2D9002FE4D1C9
:1046C000E3690593002BC3D016F0100FC0D103A8E7
:1046D00003F0D2F90127D8E79D681A681B691D44C9
:1046E000AD1AAB42AAD8ED1AA8E70025A5E76FF0EE
:1046F0007F05ADE7C6F38006009643464A46002193
:10470000E06E00F06CFC054694F94030002BB8DAFE
:10471000E26ED1681368126913445B1A013B9A4236
:1047200000D89B1A226E9A42ABD894F840306FF3AF
:10473000C71384F8403094F8413043F0010384F803
:1047400041300123A4F848300520FFF745FA98E7E7
:104750006FF0150595E72DE9F04F87B006460F4637
:10476000924699461146FFF733FC002876DD336FF9
:104770009A681C681B691C44A41A013CA34200D817
:10478000E41A55464FF0000841E002F0EBFE96F8BF
:10479000403043F0400386F840304FF0010B01E019
:1047A0004FF0000B23463A460021306F00F0C2FB69
:1047B0000446BBF1000F3BD10123A6F84830FEF7B9
:1047C000B7FE002837D02D1B3FD02744B8F1000F8B
:1047D00035D1336A0593002B37D019F0100F34D13F
:1047E00003A803F049F94FF00108059B009300234B
:1047F00001222221706801F027FF336F9A681C683C
:104800001B691C44A41A013CA34200D8E41A002DE1
:104810001BDD002CDADDAC4200DD2C4696F8403082
:1048200013F0100FBCD0AC42AFD04FF0000BB9E783
:1048300002F032FFC0E70520FFF7CEF9C3E705A974
:1048400003A803F041F90028CFD0BAEB050005D149
:1048500096F85330052B04D96FF07F0007B0BDE800
:10486000F08F6FF01B00F9E738B504460D460122C2
:104870000621FFF789FA00283CD094F853300BB199
:10488000082B3AD14FF6FF739D42A8BF1D46A4F8EE
:10489000505094F8403013F0080F25D0E36E23B148
:1048A00000229A601A60DA605A60236F23B10022F6
:1048B0009A601A60DA605A604222002104F17A009C
:1048C00009F0AFFA6022002104F1D40009F0A9FA3E
:1048D0000422002104F1400009F0A3FA94F84030CA
:1048E00043F0080384F840300121204600F096FF91
:1048F000002038BD6FF05E00FBE76FF05E00F8E768
:1049000010B5044601220621FFF73EFA88B194F85B
:104910005330052B10D194F8403043F0200384F835
:1049200040300123A4F848300520FFF755F9002056
:1049300010BD6FF05E00FBE76FF05E00F8E7FFFF71
:104940002DE9F041804602F015FE1B4B1E681B4A04
:10495000D4681860861B29D06427194B9C4227D045
:10496000E5686468B5F84830002BF6D0B34210D93A
:104970009B1BA5F848302B681BB1B8F1000F11D173
:104980000027B5F84830002BE7D0BB42E5D21F46E0
:10499000E3E70023A5F84830284601F01DF9002878
:1049A000E9DADAE72846FFF788FDEAE70126D3E7E8
:1049B0003846BDE8F08100BF1C040010F40300106D
:1049C000FC030010F0B40F48C468002001E0284642
:1049D00064680D4DAC4210D0E568AF8C8EB2B74222
:1049E000F6D195F85360012EF1D0AF8F9EB2B74249
:1049F000EED1AE6B9642EBD100E0002505B1284622
:104A0000F0BC7047F4030010FC0300102DE9F041E6
:104A100004460E4617469846C56E35B343463A4699
:104A20003146284600F086FA0546DEB994F9403052
:104A3000002B0CDBE26ED1681368126913445B1A19
:104A4000013B9A4200D89B1AE26D9A4216D2236823
:104A500043F001032360E26A12F0010F02D043F435
:104A6000807323602846BDE8F0810121FFF770FACA
:104A700005460028D2D14FF0FF35F3E794F84030D7
:104A800043F0800384F8403094F8413043F0010350
:104A900084F841300123A4F848300520FFF79CF842
:104AA000D5E790F82730062B15D110B4826B13028E
:104AB00003F47F0343EA0263140A04F47F442343AC
:104AC00043EA12634B60828F130A43EA02234B804E
:104AD000082010BC70476FF01500704790F8273021
:104AE000062B0DD1036F4BB19A6818681B691844E7
:104AF000801A0138834205D8C01A7047806E70470B
:104B00006FF01500704790F82730062B0AD1036F1D
:104B10005BB198681A681B691844801A834205D8EB
:104B2000C01A70476FF01500704700207047C0B181
:104B300070B582B004461D460F2A00F20681DFE8F8
:104B400012F019001F002D0004013E003E00040178
:104B500004010401040104018D00A3006000B800F9
:104B6000E3004FF0280383F31188BFF36F8FBFF387
:104B70004F8FFEE72B68C3610023184602B070BD5B
:104B80002B68036290F82720112A40F0E180022B65
:104B900040F2E080022303620023EEE73DB990F883
:104BA000263023F0020380F826300023E5E790F852
:104BB000263043F0020380F826300023DDE790F82A
:104BC0002730062B40F0C880042A03D1036F002B46
:104BD00040F0C580052A03D1E36E002B40F0C2806F
:104BE0002B68042A0AD1B4F84C201344013BB3FBD0
:104BF000F2F303FB02F3A3660023BEE76366002320
:104C0000BBE790F82730062B40F0AF80036F002BF6
:104C100040F0AE80C36E002B40F0AD8004260096BD
:104C20002B4632460021FFF782FF009605F108036C
:104C3000052200212046FFF77AFF0123C4F8CC307B
:104C4000C4F8D03094F8D43013F0010F00F09680FF
:104C5000B4F84C30C4F8D83000238EE790F82730F1
:104C6000062B40F08D802B683BB190F8403043F02C
:104C7000080380F8403000237FE790F840206FF36E
:104C8000C30280F8402078E790F82730062B7AD1CD
:104C90002B683BB190F8403043F0100380F840306F
:104CA00000236AE790F840206FF3041280F8402058
:104CB00063E790F82730062B68D12B68EBB190F8AA
:104CC000D43043F0020380F8D43094F8D43013F099
:104CD000020F5ED194F85330042B5CD92046FFF7C5
:104CE00012FF034600283FF448AF0123A4F84830E0
:104CF0000520FEF771FF00233FE790F8D4306FF3F3
:104D0000410380F8D430E0E790F82730062B44D1F7
:104D10002B689BB190F8423043F0040380F8423096
:104D200094F8413043F0010384F841300123A4F8A2
:104D300048300520FEF750FF00231EE790F8423070
:104D40006FF3820380F84230EAE76FF06C0314E7F8
:104D5000002312E7002310E76FF015030DE76FF053
:104D600015030AE76FF0150307E76FF0150304E773
:104D70006FF0150301E76FF01503FEE60023FCE674
:104D80006FF01503F9E66FF01503F6E66FF0150303
:104D9000F3E60023F1E60023EFE66FF01503ECE6FF
:104DA00090F82730062B0AD1C36E5BB198681A6859
:104DB0001B691844801A834205D8C01A70476FF0E7
:104DC00015007047002070472DE9F84F80460023FA
:104DD00083609A46994688E0544F8EE095F84030BB
:104DE00013F0040F05D113F0020F15D04FF0000B94
:104DF00001E04FF0000BEA6A12F0010F21D095F8A4
:104E00005320012A0BD003F00A030A2B40D0BBF138
:104E1000000F0DD1002615E04FF0010BEBE76B6D95
:104E200093B393F8403013F0020F2FD1002609E01E
:104E30002846FFF7B5FF002801DD012602E0002625
:104E400000E00026EB6A13F0040F06D095F853201B
:104E5000082A00D00AB946F0040613F0020F2AD03F
:104E6000BBF1000F16D195F8413013F0080F18D0A0
:104E700095F85320042A19D913F0100F18D143F0D4
:104E8000100385F841300EE00026DBE70126D9E764
:104E90000126D7E72846FFF721FE0028E3DD01239E
:104EA00000E000233BB146F0020604E00023F9E7EE
:104EB0000023F7E700262E634AEA060A6468BC422C
:104EC00011D0E568AB6A4345F8D195F82730062B39
:104ED00084D0EB6A13F0010FECD0AB6B0BB900265A
:104EE000E9E70126E7E709F10109B9F1010F06DC5D
:104EF000B9F1000F3FF470AF0D4F7C68DFE7002180
:104F0000D8F8000001F026FC20EA0A0010F00F019A
:104F100007D14AF01001D8F8000001F03EFCBDE8CE
:104F2000F88FD8F8000001F015FCF2E7100400102B
:104F3000FC0300102DE9F0478468056806693544D4
:104F40002D1B6C1EA64200D8A41BA1423CD2641AA1
:104F50009C4228BF1C46A4B3856819B10D44B542D4
:104F600000D3AD1B1746884681466AB1761BA64220
:104F700028BF264600F1140A324639460AEB0500DE
:104F800008F04BFFB44221D8B8F1000F07D12544F7
:104F9000D9F81030AB4200D8ED1AC9F80850D9F84A
:104FA0000C20D9F800309A422CBF002001209D42ED
:104FB0002CBF0021012188420ED09D4201D2C9F8A8
:104FC0000C502046BDE8F0870024C1E7A21BB919A8
:104FD000504608F022FFD7E7AA42F0D9F1E72DE9C1
:104FE000F04785680468066935442C1BA64200D842
:104FF000A41BA1422ED2641A9C4228BF1C4634B383
:10500000D0F8008021B18844B04501D3A8EB060850
:1050100017460D46814672B1A6EB0806A64228BF88
:10502000264600F1140A32460AEB0801384608F019
:10503000F4FEB44210D8089B4BB945B908EB040301
:10504000D9F810209A4200D89B1AC9F8003020469F
:10505000BDE8F0870024CFE7A21B5146B81908F03D
:10506000DCFEE8E70B2809D8DFE800F006080808AE
:105070000808080606060806002070470120704749
:105080008A6902F1360392F82E100909053903EBFB
:10509000810104E0013302E05A7852B313448B4299
:1050A00027D21A782AB3012AF4D0022AF4D15A78E6
:1050B000042AF1D19A78DB7843EA0223B0F84C2035
:1050C0009A4216D990F8402042F0010280F8402020
:1050D000D0F8D820B2FBF3F203FB02F2C0F8D820DC
:1050E000A0F83231A0F83031A0F84C30A0F84A30A6
:1050F00070477047B0F84C30022281F83620042007
:1051000081F837001A0A81F8382081F83930704761
:1051100070B4846994F82E309B0803F03C0303F1CB
:10512000220222440A60C5690E3D268A300A40EAFE
:10513000062080B2854200DC28461433834212DA0E
:10514000C01A94F82F3013F0200F0AD0A48E230A2F
:1051500043EA04239BB21A440A609842D4BF001A5F
:10516000C01A70BC70470020EBE70346896990F8CD
:10517000100193F85320042A04D993F8402012F028
:10518000010F00D1704793F840206FF3000283F8BD
:105190004020022281F83620042081F83700B3F83D
:1051A0004A20120A81F8382093F84A3081F83930C1
:1051B000602381F82E30E5E740F20A23A0F84A3058
:1051C000A0F84C30704710B5026F916854681369AD
:1051D0001944091B8B4200D8C91A00291BDD04465B
:1051E0005268D43001F0F2F8002814DD226F936881
:1051F000546811690B441B1B994200D85B1A9842F2
:1052000000D803465068034453605368994202D85B
:105210005368591A516010BD70B5184C246834B1E8
:1052200079B11A443632CA610D46284670BDD51888
:105230003635422DB8BF422529B1CC69AC42F0D2F7
:1052400001E040F256250C46064600212846FDF7AF
:10525000D3FE05460028E8D044B1E269A16980691F
:1052600008F0DBFD2046FDF7A5FEDEE7422206F151
:105270007A01806908F0D1FDD7E700BF6015010011
:1052800010B582B0D0F8CC4040F20A21D0F8D0203E
:10529000B0F84C300193D0F800310093D0F8E430EE
:1052A00001FB02F201FB04F1D43001F074F802B00A
:1052B00010BDFFFF30B585B00446826B130203F4C6
:1052C0007F0343EA0263110A01F47F410B4343EA7F
:1052D0001263039301A903A8FEF702F801280AD07C
:1052E00094F85230013384F852300398FEF750F8A6
:1052F000002005B030BD002584F8525094F84130AC
:1053000043F0080384F841304222294604F17A0030
:1053100008F087FD062201A904F1800008F07DFD58
:10532000082384F8863084F88750452384F8883031
:1053300084F88A50342384F88B30802384F89030AA
:10534000062384F891301C4B5B69C4F89830A26B3B
:10535000130203F47F0343EA0263110A01F47F415D
:105360000B4343EA1263C4F89430A28F130A43EA52
:105370000223A4F89C30A28C130A43EA0223A4F867
:105380009E30C4F8E4500D4A1368C4F8003103F5A8
:1053900081731360502384F8A830022384F8A93065
:1053A0002046FFF709FFB4F84C30C4F8C830204657
:1053B000FFF766FF01209CE7440000102004001066
:1053C0002DE9F0418AB005461746002900F0CC804F
:1053D00098460E4633B9F1693046FEF7B7F80646EF
:1053E0004FF00108002E00F0BC80B469002D00F0E1
:1053F000CB80EB6E002B00F0C280D9681A681B6965
:105400001A44521A013A934200D8D21AD5F8C81059
:10541000D5F8D8308B4228BF0B46286C664901402E
:1054200001B10023B5F84A10994202D9914200D83F
:105430000B464FF6FC72934200F2A3801A4611020B
:1054400021F07F4121F0FF01C2F307220A432286A7
:1054500095F841206FF3000285F84120D5F8E4204B
:1054600013446B64D5F80021130203F47F0343EA6D
:105470000263110A01F47F410B4343EA1263C4F84B
:10548000263094F82F3013F0010F0CD0A7F128012B
:10549000D5F800210A44D5F8F8108A4203D023F049
:1054A000010384F82F30D5F8E420130203F47F03BE
:1054B00043EA0263110A01F47F410B4343EA12639A
:1054C000C4F82A308023A3753B029BB243EA17231A
:1054D000238215B1394B5B690BB9D4F81E30D4F86F
:1054E0001A20C4F81E20C4F81A30638CA28C62847F
:1054F000A38433490B881A0A42EA032262820133E9
:105500000B8000202075607520766076142204F1EF
:105510000E01FEF771F8030A43EA002080B2C0438F
:10552000208301212046FEF7CEF8638E2BB94FF081
:10553000FF3384F8323084F833300E37F761A51D1D
:1055400006222946204608F068FC06221B49284608
:1055500008F063FC41463046FDF706FCB8F1000F49
:105560001BD00AB0BDE8F081242201A808F059FC44
:1055700005F17A0307934223089301AE2BE76A6E85
:1055800044E74FF6FC725AE7D4F82630D4F82A20C4
:10559000C4F82620C4F82A3094E7638CA28C628475
:1055A000A384D4F81E30C4F81A30062221462846B7
:1055B00008F033FCD5E700BF800004004400001071
:1055C0007C03001008B501468369142283F82F205C
:1055D000502283F82E20002328221846FFF7F0FEE1
:1055E000002008BD70B50D461C46D0F8D810D0F884
:1055F000E430D0F8EC209B1A1944C0F8C810C66EED
:1056000086B1F368326836693244D21A531E9E421C
:1056100000D89B1B8B4228BF0B46C0F8C8301CB972
:10562000204670BD436EF5E7012322462968FFF747
:10563000C7FE00232B60F3E710B582B0044644F6A2
:105640002063019390F85330022B06D0B0F8483015
:105650005BB3B4F8480002B010BD90F8413013F0CD
:10566000080F0ED090F85230022B06D8013B40F6BE
:10567000B83202FA03F3019306E042F6F8230193ED
:1056800002E04FF4FA730193019A642303FB02F3DF
:10569000B3F57A7F07D3154AA2FB0323C3F38F1315
:1056A000A4F84830D5E70123FAE701AAD0F8C410DE
:1056B000D43000F0D8FE019B13B980B101230193CF
:1056C000019A642303FB02F3B3F57A7F0BD3074AF5
:1056D000A2FB0323C3F38F13A4F84830B9E744F6C1
:1056E00020630193ECE70123F6E700BFD34D62107E
:1056F00010B5044601F03EFFA06510BD10B582B0A4
:105700000446CB69C3610B6A036291F8263080F8C6
:1057100026304B6E43668B6E8366CB6DC3650B6E16
:105720000366D1F8CC30C0F8CC30D1F8D030C0F816
:10573000D0308B6A23B18362CB6A43F00503C36226
:10574000114B5B6901938A8C130A43EA0223ADF87B
:10575000023094F8403043F0040384F8403061652F
:10576000B1F84E300133A1F84E30012308226946CA
:105770002046FEF7A1FD10B9012002B010BD204661
:10578000FEF70AFE0020F8E7440000102DE9F84378
:105790009469D4F826502C0204F47F0444EA05648A
:1057A0002E0A06F47F46344344EA156473B300F1CD
:1057B000D4071D4690F85330032B27D9C66EEEB19F
:1057C000D6F808C0336836693344A3EB0C03013BB9
:1057D0009E4200D89B1B9046894606462A46214693
:1057E000384600F0E2FD011E16DB2B464A463046E5
:1057F000FFF70CF9854203D100200BE0436EEAE786
:105800004046FFF7DFFE4FF0FF3003E0002380F853
:1058100010311846BDE8F8830020FBE770B5044658
:105820000E4690F85330042B05D9082B01D00122E5
:1058300002E0002200E00022042E05D9082E01D04B
:10584000012302E0002300E000239A425FD0002BF6
:105850003BD094F8403013F0040F29D013F0080F18
:105860000AD1656D4DB94FF0280383F31188BFF35A
:105870006F8FBFF34F8FFEE7254665B16B6DABB100
:105880002B6843F004032B60EA6A12F0010F02D088
:1058900043F480732B600023636594F8403003F079
:1058A000FB0343F0020384F840301AE06C65E7E73D
:1058B000236843F008032360E26A12F0020F22D04B
:1058C00043F40073236000250BE0236843F02003BA
:1058D0002360E26A12F0040F17D043F48063236060
:1058E000002594F85300FFF7BDFB10B90023A4F87E
:1058F000483084F853602046FFF7FAFE15B1284679
:10590000FEF7DBFD70BD0025EBE70025E9E776B982
:1059100094F8403013F0060F0BD013F0080F01D0AD
:105920000025E6E72046FEF71FFD0025E1E70025FC
:10593000DFE70025DDE72DE9F04784B0044688461F
:1059400017460B68A3B39D6904F1D40900230393A0
:1059500095F82F3043F0100385F82F30236F002B7C
:1059600079D0B4F84A30012B25D80026002E03DB6D
:1059700094F85330052B70D0002E40F3968095F8A4
:105980002F3003F0F70307F11402D2B2920085F82A
:105990002E2043F0100385F82F301EB143F008038A
:1059A00085F82F303E442836304604B0BDE8F087F5
:1059B00000F17A05C8E703AAD4F8C410484600F0FD
:1059C0001FFD824606460028D0DD3B460246D8F839
:1059D00000102046FFF720FC002863D0C8F8000024
:1059E000856907F136022A44206FD0F800E0036988
:1059F00003991944A1EB0E018B4200D8C91A012367
:105A000000935346FFF7EBFAB4F8403023F47E538B
:105A100023F03F035B045B0C402BA7D1226F9368FC
:105A20001269134403995B1A9A4200D89B1A984250
:105A30009CD195F82F3043F0010385F82F30D4F82E
:105A400000315344C4F8F83094F8413043F0400337
:105A500084F841308AE700268AE794F8403013F052
:105A6000200F89D0484600F0F8FC002884D094F834
:105A700040306FF3451384F8403095F82F3043F0F1
:105A8000010385F82F3094F8413043F0410384F846
:105A90004130D4F8F430C4F8F83006212046FFF73E
:105AA000BDFE69E74FF0FF3666E794F8413013F02A
:105AB000030F7FF464AF77E72DE9F04180460D4690
:105AC00000273C46072C11D8002229464046FFF704
:105AD00032FF061E0ADD0123324629684046FFF7E1
:105AE0006FFC00232B6037440134EBE73846BDE8F8
:105AF000F08130B583B0044690F85330022B0ED1BC
:105B000090F85230022B18D890F8413013F0080F5B
:105B100018D1FFF7CFFB012814D000250AE002A915
:105B2000002341F8043DFFF7C7FF0546019808B17F
:105B3000FDF740FA284603B030BD0821FFF76EFE9E
:105B40000025F7E704F17A012046FFF7D3FA00F1C8
:105B500028051430C0B2800084F8A80094F85230B0
:105B6000013384F8523000232A4619462046FFF7B5
:105B700027FCDFE790F85330082B06D8DFE803F066
:105B80002525050505250505250010B5044601F068
:105B9000F1FCA36DC01A0F4B984201D8012010BD33
:105BA00008212046FFF73AFE94F8403013F0040F26
:105BB0000DD013F0080F02D04FF0FF30EFE7204672
:105BC000FEF7EAFB4FF0FF30E9E7002070470120C5
:105BD000E5E700BFA086010010B5044690F85330F9
:105BE000042B03D9036F0BB1FFF7EDFA94F8533090
:105BF000042B01D8022B02D12046FFF77AFF204662
:105C0000FFF71AFD2046FFF7B5FF10BDF8B50546B2
:105C10000E468F6990F8403013F0080F43D043F0E0
:105C2000040380F8403068650446002C39D07A8C33
:105C3000130A43EA0223A387D7F81A20130203F4B6
:105C40007F0343EA0263110A01F47F410B4343EAF5
:105C50001263A363244D2B68C4F80031D7F82620C3
:105C6000130203F47F0343EA0263110A01F47F4144
:105C70000B4343EA1263C4F8E4302046FFF79CFA72
:105C80002046FFF7FDFA2B6803F581732B60032193
:105C90002046FFF7C3FD4222B16904F17A0008F003
:105CA000BCF82046F8BDB0F84E20B0F850309A420B
:105CB00010D2062201210220FEF7D4F90446431E29
:105CC00013F1030F0BD82946FFF718FD0028ACD1BC
:105CD0000024E6E70846FFF775FC0024E1E73046BC
:105CE000FFF770FC0024DCE7200400102DE9F041F0
:105CF000044617461D460B689E69D43096F82F203F
:105D0000D6F826804FEA082303F47F0343EA0863AA
:105D10004FEA182101F47F410B4343EA186894F8D5
:105D2000531002292CD04FF0100C02F017036345DA
:105D300029D1A38FA4F82E31A38CA4F82C310229E9
:105D400033D00FB9C4F8E480D4F8F0300133C4F88C
:105D5000003194F85330022B01D0002F40D0102393
:105D600086F82F3005F128071435EDB2AD0086F81E
:105D70002E5005212046FFF751FD3846BDE8F08141
:105D80004FF0120CD1E708212046FFF747FD96F8A7
:105D90002F3043F0040386F82F3005F1280714351F
:105DA000EDB2AD0086F82E50E7E7102384F8A93055
:105DB000B4F84A30D4F80021414600F0C3FA08F1A3
:105DC0000103C4F8EC30C4F8E430D4F8F430013303
:105DD000C4F8F430D4F808310133C4F80831B3E71B
:105DE0000027C6E738B504468D6995F82F00D5F829
:105DF0002A20130203F47F0343EA0263110A01F429
:105E00007F410B4343EA126310F0010F04D0D4F832
:105E1000E8200132C4F8E42094F8412012F0400F49
:105E20002AD1D4F8F430C4F8F83042F0400384F8B2
:105E3000413094F8422012F0010F29D0D4F8F83004
:105E40000133C4F8F43094F94130002B2CDB0023EB
:105E500085F82F30D4F8F430C4F8003195F82F309D
:105E60008BB394F81001283094F810311433DBB25E
:105E70009B0085F82E3038BDD4F8F82001329A42C4
:105E8000D7D194F8423043F0010384F84230D0E790
:105E9000D4F8F830C4F8F430112385F82F300A21F3
:105EA0002046FFF7BBFCD5E712F0020F07D1102305
:105EB00085F82F3008212046FFF7B0FCCAE7002301
:105EC00085F82F30F6E70020CEE72DE9F04F83B0BC
:105ED00004460E4692461F460B689D6900F1D409A0
:105EE00095F82F80D5F826B04FEA0B2303F47F03F3
:105EF00043EA0B634FEA1B2202F47F42134343EA57
:105F00001B6B2A8E130A43EA02239BB2C0F8C430EB
:105F100018F0100F29D1236F13B12046FFF753F962
:105F2000D4F8F430C4F8003194F8413013F0200F65
:105F300002D118F0010F6FD013F0400F3ED1484648
:105F400000F0C4FA8046484600F087FAB8F1000F26
:105F50005DD000285DD00BEB0A03D4F8E4209B1A37
:105F6000012B2BDD0023984634E0D5F82A100B02D4
:105F700003F47F0343EA01630A0A02F47F421343F6
:105F800043EA1161484600F094FA0346206F002866
:105F9000C1D0002BBFD0002100910A46FFF71FF8A7
:105FA0000028B8D0236843F002032360E26A12F0AD
:105FB000020FB0D043F400732360ACE794F8413093
:105FC00043F0200384F8413031682046FFF70AFF90
:105FD00080460123BBB9102385F82F30BAF1000F9A
:105FE00010D007F1280807F11403DBB29B0085F8F5
:105FF0002E3094F8413013F0400F03D0D4F8F8302D
:10600000C4F8F4305FB1404603B0BDE8F08F002320
:10601000E0E780460023DDE74FF00008DBE73A4683
:1060200031462046FFF787FC0028ECDD8046EAE792
:106030002DE9F04F83B004460E4608688769D7F80B
:1060400026301D0205F47F0545EA03651A0A02F4AD
:106050007F42154345EA136597F82FA001A9FFF782
:1060600057F8804694F85330042B04D9D4F8E42030
:106070006B1C9A423ED005EB080BD4F8EC30ABEB2E
:106080000303002B01DDC4F8ECB0434632680199EC
:106090002046FFF77BFB00287EDB31682046FFF7B8
:1060A00064F8814694F85330042B2AD01AF0010F7B
:1060B00014D094F94130002B10DBC4F8E8B094F808
:1060C000413043F0800384F8413013F0400F05D194
:1060D00094F8423043F0020384F8423094F853308D
:1060E000023B082B5BD8DFE803F0411541495151D1
:1060F0005A5A510094F8413043F0010384F841307A
:10610000B9E70AF01F03022BD0D103212046FFF785
:1061100085FBCBE739462046FEF7ECFF122387F8D4
:106120002F3000F128091430C0B2800087F82E000B
:1061300004212046FFF772FB0135C4F8EC50C4F887
:10614000E450D4F8F0300133C4F80831C4F8F43026
:10615000B9F1000F06DD4B46424631462046FFF7B7
:1061600041FA8146484603B0BDE8F08F4B464246AF
:1061700031462046FFF7BAFD8146E9E74B464246E5
:1061800031462046FFF7A1FE8146E1E7316820460F
:10619000FFF728FE8146DBE74FF0FF39E2E74FF0DB
:1061A0000009DFE7F0B583B00190846994F82F50BF
:1061B000D4F81E60330203F47F0343EA0663300A17
:1061C00000F47F401843A18C0B0A43EA0121D4F864
:1061D0001A703B0203F47F0343EA07633A0A02F4AE
:1061E0007F421A43B4F822C04FEA1C2343EA0C232F
:1061F0009BB242EA176289B240EA1660FEF7E2FB00
:1062000030B1064690F853703846FEF72BFF70B950
:1062100005F01F03102B5AD015F0040F02D00020F8
:1062200003B0F0BD0198FFF7CDF90020F8E7002397
:1062300086F85230012F28D015F0040F3CD105F01C
:106240001F05022D01D1042F43D8019B9969142207
:10625000223106F19C0007F0E0FD3046FFF748FAD6
:1062600094F82E3003F0F003502B2BD801A93046C0
:10627000FFF7DEFE019818B1FCF79CFE00230193A6
:106280003046FFF7D9F90120CAE705F01F03022BBA
:1062900009D015F0040F01D00020C1E70198FFF7E5
:1062A00091F90020BCE701993046FFF7AFFC0646A4
:1062B0000028D2D10020B3E700213046FFF7AEFA24
:1062C0000020ADE701993046FEF7DAFECEE7002068
:1062D000A6E70020A4E7FFFF838C190A41EA032107
:1062E00089B2124BDB680BE092F8404014F0020FC9
:1062F00012D04265012000E0002010BC70475B68AE
:106300000B4A934210D01A688A42F8D110B4DA6866
:1063100092F82740062CE7D05B68054A9342EBD001
:106320001A688A42F8D1F2E700207047F40300109F
:10633000FC030010B0F85E308B4201D9002070479A
:106340000120704710B4002404600124047093B14C
:106350001C46B0F85E300BB1A0F85E40B0F85C307F
:10636000A34200D83BB94368B3FBF4F304FB03F347
:106370004360A0F85C40B0F85C3043644FF4FA73BB
:106380008363C16001618161C261026242638262B2
:10639000C26210BC704738B51D4641608260059BE3
:1063A000049A2946FFF7CEFF38BD10B404698C4229
:1063B00006D1934207D314440461002010BC7047F7
:1063C0004FF0FF30FAE74FF0FF30F7E770B5836C1E
:1063D000002B02DD0026304670BD456C8D4200D397
:1063E0000D460446436B03642E468564C264002355
:1063F000436501F0BFF82065636B1D446563EAE700
:10640000F8B5856C2DB31646044690F8563013F057
:10641000010F0CD0876B90F854309F4001F0AAF820
:10642000236DC01A00EB800043009F4213D894F8FC
:10643000563043F0010384F8563094F85430013359
:1064400084F8543001F096F82065236CE362E36C25
:1064500033602846F8BD0025FBE7836C0BB10020B4
:1064600070470120704738B500231360836CE3B197
:106470001546044690F8563013F0010F04D1FFF78B
:1064800059FF98B1012011E001F074F8236DC01A92
:1064900000EB80004200A36B94F854108B409342B1
:1064A00005D99B1A2B60012000E0002038BD012097
:1064B000FCE7836C33B1026A1A448A4204D8026250
:1064C00000228264184670470023FBE70369806955
:1064D000181AC043C00F70472DE9F04182B004463E
:1064E000436902A840F8043DA5692946FCF7F8FE77
:1064F000064602280BD0012811D050B9019900207E
:10650000FCF7EEFD019B63612046FCF71BFF022EAA
:1065100047D12046FCF74EFD02B0BDE8F081238C48
:10652000AB84638C6B84E36908339BB21A0A42EA3A
:106530000323EB84002785F8287085F82970A36968
:1065400093F8068018221949A81D07F066FCE36934
:106550001C339BB22B820E33E3612A8A130A43EA6F
:1065600002232B826369C5F81E302F766F761422C2
:1065700005F10E013846FDF73FF8030A43EA002310
:106580009BB2DB432B8318F0020F05D1002385F863
:10659000283085F82930BAE701212846FDF793F81D
:1065A000B5E701212046FCF7DFFBB5E7440000100A
:1065B00070B5054686690846FDF720FF28B30446F6
:1065C000D6F81A10B01DFCF78BFD00F0CBFFFCF7DE
:1065D00039F8294604F1380000F052F9FCF754F874
:1065E00001F05AF8606810B1012100F0D6F8A36AF2
:1065F0006BB1E26A12F0010F01D1012006E0012126
:10660000186800F0CAF8012000E0002070BD0120E9
:10661000FCE71AB9084206D10020704731EA0003AE
:1066200003D000207047012070470120704710B54B
:106630001C20FBF78FFE044620B1002340F8043BEA
:1066400000F010F9204610BD2DE9F047DDF820904C
:1066500060B1064611F07F4A11D04FF0280383F352
:106660001188BFF36F8FBFF34F8FFEE74FF0280302
:1066700083F31188BFF36F8FBFF34F8FFEE741B9EC
:106680004FF0280383F31188BFF36F8FBFF34F8F51
:10669000FEE7984617460C4601F062FA58B9B9F180
:1066A000000F08D04FF0280383F31188BFF36F8FDA
:1066B000BFF34F8FFEE700F055FF35684246214695
:1066C0002846FFF7A6FF58B317B125EA0403336045
:1066D00000F0E2FFBAF1000F1FD038B91C4B4FF0A9
:1066E00080521A60BFF34F8FBFF36F8F01F05CFBD6
:1066F000054610F0007F0ED1FBF7A4FF3568424637
:1067000021462846FFF785FF18B117B125EA040492
:106710003460FBF7B9FF25F07F452846BDE8F087D8
:10672000B9F1000F11D06FB90021B8F1000F01D0FD
:1067300041F080614A462143301D01F0C9F8CA4644
:106740000025C5E74FF08071EFE7CA46C0E700BFFC
:1067500004ED00E040B94FF0280383F31188BFF344
:106760006F8FBFF34F8FFEE770B5054611F07F4F77
:1067700008D04FF0280383F31188BFF36F8FBFF366
:106780004F8FFEE70C46FBF75DFF2E6826EA0404F8
:106790002C60FBF779FF304670BDF8B540B94FF07B
:1067A000280383F31188BFF36F8FBFF34F8FFEE78A
:1067B000044611F07F4F08D04FF0280383F311886F
:1067C000BFF36F8FBFF34F8FFEE70D4600F10C064E
:1067D00000F0C8FE206923682B432360002504E0F5
:1067E000216833EA01010CD03846B04213D0476823
:1067F000026822F07F4312F0806FF1D121681942C4
:10680000F2D012F0807F00D01D43216841F000716A
:1068100001F0EEF8E8E7236823EA0503236000F0BF
:106820003BFF2068F8BD10B5044600F09BFE63688E
:1068300093B1206904F10C03984204D04FF0007129
:1068400001F0D6F8F3E74FF0280383F31188BFF384
:106850006F8FBFF34F8FFEE72046FBF7EBFD00F095
:106860001BFF10BD00F1080343604FF0FF32826050
:10687000C360036100230360704700230361704716
:1068800043684B609A688A609A68516099600861B1
:10689000036801330360704730B40D68B5F1FF3F02
:1068A00002D000F1080202E0026904E01A465368CF
:1068B0001C68AC42FAD953684B6099608A60516099
:1068C000086103680133036030BC704703694268A4
:1068D000816891608268416851605A68824206D03E
:1068E000002202611A68013A1A60186870478268CB
:1068F0005A60F5E7436A23B1036B1868C0F10700DB
:1069000070470020704710B50446FBF79BFEA26B52
:10691000E36B9A4204D00024FBF7B6FE204610BD7C
:106920000124F9E710B50446FBF78CFEA36B23B1F5
:106930000024FBF7A9FE204610BD0124F9E770B53D
:1069400004461646856B026C5AB903681BB10020D9
:106950000135A56370BD406801F06EF900236360E6
:10696000F6E76EB9806807F058FA226CA368134402
:10697000A3606268934219D32368A3600020E7E70D
:10698000C06807F04AFA226C5242E3681344E3609D
:1069900021688B4202D263681A44E260022E01D061
:1069A0000020D5E725B1013D0020D1E70020CFE749
:1069B0000020CDE7026C72B110B5C3681344C36008
:1069C0004468A34201D30368C3600C46C1682046F3
:1069D00007F023FA10BD704738B50546FBF732FEC5
:1069E00095F8454064B203E001F0AEF8013C64B2B2
:1069F000002C08DD6B6A33B105F1240000F0B2FF12
:106A00000028F3D0F0E7FF2385F84530FBF73CFE84
:106A1000FBF718FE95F8444064B203E001F094F8E7
:106A2000013C64B2002C08DD2B6933B105F1100084
:106A300000F098FF0028F3D0F0E7FF2385F84430FA
:106A4000FBF722FE38BDFFFF38B540B94FF02803F1
:106A500083F31188BFF36F8FBFF34F8FFEE70446B8
:106A60000D46FBF7EFFD2168E26B236C03FB021080
:106A700060600020A063A160013A02FB0313E360A1
:106A8000FF2384F8443084F84530A5B923691BB945
:106A9000FBF7FAFD012038BD04F1100000F062FFA1
:106AA0000028F5D0084B4FF080521A60BFF34F8F8B
:106AB000BFF36F8FECE704F11000FFF7D3FE04F192
:106AC0002400FFF7CFFEE3E704ED00E038B51D46F4
:106AD000049C0B4649B12260E063236401212046F7
:106AE000FFF7B2FF84F84C5038BD2460F4E740B99A
:106AF0004FF0280383F31188BFF36F8FBFF34F8FDD
:106B0000FEE7F0B583B0054611B101FB00F000E0EF
:106B1000002017460C465030FBF71CFC064638B1E7
:106B200000903B4600F1500221462846FFF7CEFF79
:106B3000304603B0F0BD40B94FF0280383F311880D
:106B4000BFF36F8FBFF34F8FFEE7884208D24FF03D
:106B5000280383F31188BFF36F8FBFF34F8FFEE7D6
:106B600010B50C4602220021FFF7C1FF034600B119
:106B70008463184610BDFFFFF0B585B0019260B187
:106B8000044699B9026C8AB14FF0280383F3118847
:106B9000BFF36F8FBFF34F8FFEE74FF0280383F3F0
:106BA0001188BFF36F8FBFF34F8FFEE7022B0BD11E
:106BB000E26B012A08D04FF0280383F31188BFF35A
:106BC0006F8FBFF34F8FFEE71E460F4600F0C8FFE2
:106BD00050B9019B53B14FF0280383F31188BFF3E1
:106BE0006F8FBFF34F8FFEE700253AE0002538E0B6
:106BF000324639462046FFF7A2FE636A4BB9A8B178
:106C00003B4B4FF080521A60BFF34F8FBFF36F8F33
:106C10000CE004F1240000F0A5FE38B1344B4FF035
:106C200080521A60BFF34F8FBFF36F8FFBF72CFDBD
:106C3000012005B0F0BDFBF727FD0020F9E702A811
:106C400000F036FF012519E0002384F8443021E0EC
:106C5000002384F8453023E02046FFF7BDFE00F016
:106C60001BFDFBF7EFFCA26BE36B9A42C0D3022E35
:106C7000BED0019B002BDED0002DE0D0FBF704FD41
:106C800000F070FCFBF7DEFC94F844305BB2B3F12B
:106C9000FF3FD9D094F845305BB2B3F1FF3FD7D076
:106CA000FBF7F2FC01A902A800F00EFFC8B92046CC
:106CB000FFF729FE0028CFD0019904F1100000F061
:106CC000EFFD2046FFF788FE00F0E6FC0028C8D163
:106CD000074B4FF080521A60BFF34F8FBFF36F8F97
:106CE000BFE72046FFF778FE00F0D6FC0020A0E7C3
:106CF00004ED00E02DE9F84360B1044699B9006C59
:106D000088B14FF0280383F31188BFF36F8FBFF36F
:106D10004F8FFEE74FF0280383F31188BFF36F8F87
:106D2000BFF34F8FFEE7022B0BD1E06B012808D099
:106D30004FF0280383F31188BFF36F8FBFF34F8F9A
:106D4000FEE71F4690468946FBF76AFDEFF3118682
:106D50004FF0280383F31188BFF36F8FBFF34F8F7A
:106D6000A26BE36B9A4203D3022F01D000200FE005
:106D700094F845506DB23A4649462046FFF7DFFD8C
:106D8000B5F1FF3F08D06B1C5BB284F845300120A1
:106D900086F31188BDE8F883636A5BB104F12400CF
:106DA00000F0E0FD40B1B8F1000F07D00120C8F8B5
:106DB0000000EDE70120EBE70120E9E70120E7E72C
:106DC000F0B585B0019260B1044699B9036C8BB1FE
:106DD0004FF0280383F31188BFF36F8FBFF34F8FFA
:106DE000FEE74FF0280383F31188BFF36F8FBFF3E3
:106DF0004F8FFEE70F4600F0B3FE50B9019B53B131
:106E00004FF0280383F31188BFF36F8FBFF34F8FC9
:106E1000FEE700263EE000263CE039462046FFF72C
:106E2000C9FD013DA563236923B9FBF72DFC0120B2
:106E300005B0F0BD04F1100000F094FD0028F4D07E
:106E4000344B4FF080521A60BFF34F8FBFF36F8FF8
:106E5000EBE7FBF719FC0020EAE702A800F028FEA8
:106E6000012621E0002384F8443029E0002384F83F
:106E700045302BE02046FFF7AFFD00F00DFC09E0A8
:106E80002046FFF7A9FD00F007FC2046FFF74AFD6A
:106E900000283DD1FBF7D6FBA56B002DBDD1019B92
:106EA000002BD6D0002ED8D0FBF7EEFB00F05AFB1B
:106EB000FBF7C8FB94F844305BB2B3F1FF3FD1D08D
:106EC00094F845305BB2B3F1FF3FCFD0FBF7DCFB6A
:106ED00001A902A800F0F8FD0028D1D12046FFF753
:106EE00021FD0028C6D0019904F1240000F0D8FC4F
:106EF0002046FFF771FD00F0CFFB0028CAD1054BFB
:106F00004FF080521A60BFF34F8FBFF36F8FC1E70E
:106F100000208DE704ED00E070B584B0019140B928
:106F20004FF0280383F31188BFF36F8FBFF34F8FA8
:106F3000FEE70446036C43B14FF0280383F3118846
:106F4000BFF36F8FBFF34F8FFEE700F009FE50B91C
:106F5000019B5BB14FF0280383F31188BFF36F8F60
:106F6000BFF34F8FFEE700252E4651E000252E4649
:106F70004EE0013BA363236813B900F021FF60607A
:106F8000236963B104F1100000F0ECFC38B1484B08
:106F90004FF080521A60BFF34F8FBFF36F8FFBF734
:106FA00073FB0125284604B070BD45B14FF028039E
:106FB00083F31188BFF36F8FBFF34F8FFEE7FBF7AB
:106FC00063FBEFE702A800F073FD01262AE000232F
:106FD00084F8443032E0002384F8453034E0FBF795
:106FE00031FB606800F0CCFD0546FBF74DFB3BE054
:106FF0002046FFF7F1FC00F04FFB09E02046FFF7C9
:10700000EBFC00F049FB2046FFF78CFC002840D148
:10701000FBF718FBA36B002BABD1019B002BC4D05B
:10702000002ECFD0FBF730FB00F09CFAFBF70AFBF9
:1070300094F844305BB2B3F1FF3FC8D094F84530C8
:107040005BB2B3F1FF3FC6D0FBF71EFB01A902A85C
:1070500000F03AFD0028D1D12046FFF763FC00285C
:10706000C6D02368002BBAD0019904F1240000F0A7
:1070700017FC2046FFF7B0FC00F00EFB0028C7D13C
:107080000B4B4FF080521A60BFF34F8FBFF36F8FDF
:10709000BEE7002D86D0FBF7D5FA2046FFF72AFC85
:1070A0000146606800F020FEFBF7EEFA002579E764
:1070B00004ED00E040B94FF0280383F31188BFF3DB
:1070C0006F8FBFF34F8FFEE710B50446FBF7BAFA98
:1070D000A46BFBF7D9FA204610BDFFFF0023092B54
:1070E0000CD8074A52F833200AB10133F7E7044AB3
:1070F00042F8331002EBC30358607047704700BF7B
:10710000240400100023092B0FD8084A02EBC30205
:107110005268824201D00133F5E7044A002142F867
:10712000331002EBC303596070477047240400100A
:1071300040B94FF0280383F31188BFF36F8FBFF37B
:107140004F8FFEE710B50446FFF7DCFF2046FBF744
:1071500071F910BD70B504460D461646FBF772FA7C
:1071600094F844305BB2B3F1FF3F0DD094F8453052
:107170005BB2B3F1FF3F0BD0FBF786FAA36B5BB1B9
:107180002046FFF729FC70BD002384F84430EDE76A
:10719000002384F84530EFE73246294604F1240005
:1071A00000F0C4FBECE7FFFF084B1B681B683BB11A
:1071B000064B1B68DB68DB685A68054B1A60704732
:1071C000034B4FF0FF321A60704700BF7804001085
:1071D0005005001010B50446006BFBF72BF9204654
:1071E000FBF728F910BD2DE9F04781460D461746FB
:1071F0009A46089EDDF824800A9C9200A521206B07
:1072000006F00FFE236B07F18042013A03EB820781
:1072100027F007070023082B07D8E95CE21882F85B
:107220003410EA5C0AB10133F5E7002384F83C30FE
:10723000062E00D90626E662A6640025E564201D18
:10724000FFF71BFB04F11800FFF717FB2461C6F1E1
:107250000706A6616462256584F854505246494683
:107260003846FBF7C5F92060B8F1000F01D0C8F827
:107270000040BDE8F087FFFF38B5002407E004EBCD
:10728000840293000E481844FFF7ECFA0134062CF0
:10729000F5D90C4D2846FFF7E5FA0B4C2046FFF7D1
:1072A000E1FA0A48FFF7DEFA0948FFF7DBFA094876
:1072B000FFF7D8FA084B1D60084B1C6038BD00BFB3
:1072C0008004001024050010380500105805001037
:1072D0008405001070050010780400107C04001074
:1072E00010B50446FBF7AEF9214A13680133136069
:1072F000204B1B685BB1204B1B686BB91D4B1B6897
:10730000DA6AE36A9A4207D81A4B1C6004E0194B08
:107310001C601368012B27D0184A136801331360CF
:107320002364E36A01229A401549086802430A600F
:1073300003EB83039A00211D12481044FFF7A0FAC3
:10734000FBF7A2F90C4B1B686BB10A4B1B68DA6A9E
:10735000E36A9A4207D20C4B4FF080521A60BFF397
:107360004F8FBFF36F8F10BDFFF786FFD4E700BFCD
:107370000C050010740400106C0500101C050010B2
:10738000200500108004001004ED00E00F4B1B6886
:10739000D3B110B5FBF756F90D4BDB68DC68201D47
:1073A000FFF794FA0B4A1368013B1360074A13680E
:1073B000013B1360FBF768F92046FFF70BFF034B17
:1073C0001B68002BE6D110BD704700BF10050010F0
:1073D000840500100C05001008B5FFF7D7FFFCE787
:1073E00070B504460E461D4B1D681D4B18680430D1
:1073F000FFF76CFA50B91A4B1B68DA6A012303FADB
:1074000002F218490B6823EA02030B60B4F1FF3F54
:1074100013D02C44124B1B685C60A54216D8124B4B
:1074200018680F4B19680431FFF736FA0F4B1B68C9
:10743000A34212D90D4B1C600FE0002EE9D0084B7F
:10744000196804310A48FFF71BFA06E0094B18686F
:10745000034B19680431FFF71FFA70BD980500103F
:10746000740400102005001078040010500500106E
:10747000700500107C0400102DE9F04385B007462C
:107480008846154699469000FAF764FFF8B106461B
:107490005820FAF75FFF0446A8B10663D4B1002371
:1074A000039302940D9B01930C9B00934B462A4639
:1074B00041463846FFF797FE2046FFF711FF0120AF
:1074C00005B0BDE8F0833046FAF7B4FFE6E74FF0C9
:1074D000FF30F5E74FF0FF30F2E7FFFF00B583B074
:1074E0001A4B0193002300934FF4967218491948E0
:1074F000FFF7C2FF012807D0012808D0B0F1FF3FF5
:107500001AD003B05DF804FB00F06EFDF4E74FF015
:10751000280383F31188BFF36F8FBFF34F8F0E4B98
:107520004FF0FF321A600D4B01221A600C4B002203
:107530001A60FBF719F9E4E74FF0280383F3118889
:10754000BFF36F8FBFF34F8FFEE700BF4C050010F6
:10755000B8150100D9730000500500106C0500102B
:1075600098050010024A136801331360704700BF8A
:1075700018050010014B1868704700BF98050010EF
:10758000F8B53A4B1B68002B64D1394B1D680135A7
:107590001D60C5B9374B1B681B6843B14FF028030A
:1075A00083F31188BFF36F8FBFF34F8FFEE7314A2C
:1075B0001168314B186810601960304A1368013344
:1075C0001360FFF7F1FD2E4B1B68AB4238D9002446
:1075D0002C4B1B68DB6A03EB83039A002A4B9B58F6
:1075E000012B3CD901243AE00124224B1B681B6883
:1075F00043B3204B1B68DB68DE6873689D4226D36B
:10760000371D3846FFF762F9B36A1BB106F118005F
:10761000FFF75CF9F36A01229A401C4908680243AB
:107620000A6003EB83039A00394617481044FFF7BA
:1076300027F9F26A134B1B68DB6A9A42D4D2D4E76B
:107640000024D2E70E4B4FF0FF321A60C0E70C4A1D
:107650001360BDE70E4A13680133136000240D4B1D
:107660001B6803B101242046F8BD00BF18050010B7
:1076700098050010780400107C04001054050010D8
:107680005005001074040010800400102005001044
:10769000140500109C05001038B5334B1B6843B926
:1076A0004FF0280383F31188BFF36F8FBFF34F8F21
:1076B000FEE7FAF7C7FF2C4B1A68013A1A601B68FD
:1076C000002B4DD1294B1B6823B90024FAF7DCFFAE
:1076D000204638BD0024264B1B681BB3244BDB68B7
:1076E000DC6804F11800FFF7F1F8251D2846FFF7C4
:1076F000EDF8E36A01229A401E49086802430A60D5
:1077000003EB83039A0029461B481044FFF7B8F89F
:10771000E26A1A4B1B68DB6A9A42DCD3184B0122DF
:107720001A60D8E70CB1FFF73FFD164B1C6854B147
:10773000FFF726FF10B1124B01221A60013CF7D16E
:10774000104B00221A600E4B1B685BB10E4B4FF0C2
:1077500080521A60BFF34F8FBFF36F8F0124B5E7DC
:107760000024B3E70024B1E7180500100C05001051
:10777000580500102005001080040010740400104B
:107780009C0500101405001004ED00E010B5A8B130
:1077900004460F4B1B6843B14FF0280383F3118855
:1077A000BFF36F8FBFF34F8FFEE7FFF7DBFE0021C4
:1077B0002046FFF715FEFFF76FFF38B9054B4FF076
:1077C00080521A60BFF34F8FBFF36F8F10BD00BFA1
:1077D0001805001004ED00E02C4B1B681BB12C4B6E
:1077E00001221A60704710B5294B00221A60294BFC
:1077F0001B681B6B1A68B2F1A53F03D15A68B2F13E
:10780000A53F1BD0234B18681968343100F06FFF77
:10781000214B1B68B3FA83F3DBB2C3F11F0303EB05
:1078200083018A001D498A588AB94FF0280383F3DF
:107830001188BFF36F8FBFF34F8FFEE79A68B2F1E5
:10784000A53FDFD1DB68B3F1A53FDBD1E0E713480B
:107850009A00D418A10001444C6864684C601A4432
:10786000910008310844844209D003EB83039A0055
:107870000A4B13445B68DA68064B1A6010BD6168F6
:107880000648142202FB03025160EEE718050010BF
:107890009C050010740400102005001080040010E6
:1078A00040B94FF0280383F31188BFF36F8FBFF304
:1078B0004F8FFEE710B50C46044B19681831FEF7E0
:1078C000EBFF01212046FFF78BFD10BD7404001073
:1078D00040B94FF0280383F31188BFF36F8FBFF3D4
:1078E0004F8FFEE703460F48006840B94FF028036A
:1078F00083F31188BFF36F8FBFF34F8FFEE710B58F
:10790000184614460B46084A116843F000438B6141
:1079100011681831FEF7B4FF01212046FFF760FD22
:1079200010BD00BF180500107404001038B540B930
:107930004FF0280383F31188BFF36F8FBFF34F8F8E
:10794000FEE70C461546064A11681831FEF798FF07
:107950000DB14FF0FF3429462046FFF741FD38BDF9
:107960007404001038B5C368DC6844B94FF02803CC
:1079700083F31188BFF36F8FBFF34F8FFEE704F1DE
:1079800018052846FEF7A2FF134B1B68E3B9251D17
:107990002846FEF79BFFE36A01229A400F490868D8
:1079A00002430A6003EB83039A0029460C48104403
:1079B000FEF766FFE26A0B4B1B68DB6A9A4208D946
:1079C0000120094B186038BD29460848FEF758FFCA
:1079D000F0E70020F7E700BF1805001020050010B1
:1079E00080040010740400109C050010580500105D
:1079F00038B51C4B1B6843B94FF0280383F311883B
:107A0000BFF36F8FBFF34F8FFEE741F0004101607E
:107A1000C468F4B1FEF75AFF251D2846FEF756FF4D
:107A2000E36A01229A401049086802430A6003EBA6
:107A300083039A0029460D481044FEF721FFE26AAD
:107A40000B4B1B68DB6A9A4202D90A4B01221A606F
:107A500038BD4FF0280383F31188BFF36F8FBFF356
:107A60004F8FFEE71805001020050010800400105D
:107A7000740400109C05001040B94FF0280383F3F4
:107A80001188BFF36F8FBFF34F8FFEE710B5044629
:107A9000FAF7D8FD044B1B682360044B1B68636036
:107AA000FAF7F2FD10BD00BF540500109805001054
:107AB000034B1B680360034B1B684360704700BFA8
:107AC0005405001098050010F8B550B1054689B965
:107AD0004FF0280383F31188BFF36F8FBFF34F8FED
:107AE000FEE74FF0280383F31188BFF36F8FBFF3D6
:107AF0004F8FFEE70C46FAF7A5FD114B1968686831
:107B00000A1A2368B3F1FF3F16D02F680D4E36686E
:107B1000B74201D0884211D9934203D80023236091
:107B2000012405E09B1A23602846FFF7C1FF0024CB
:107B3000FAF7AAFD2046F8BD0024F9E70124F7E78B
:107B40009805001054050010014B01221A6070477F
:107B50009C050010014B1868704700BF74040010AA
:107B6000054B1B6833B1054B1B680BB100207047F8
:107B700002207047012070476C05001018050010A6
:107B8000002850D038B50446C26A28490968C96A35
:107B90008A423ED28169002905DB24490968C96A05
:107BA000C1F107018161606902EB82029100204A04
:107BB0000A44904205D01D4A1268D26AE26201204E
:107BC00038BD251D2846FEF781FE68B9E36A03EB40
:107BD00083018A0016498A5832B901229A40154910
:107BE0000B6823EA02030B60104B1B68DB6AE3623D
:107BF000012404FA03F20F49086802430A6003EB08
:107C000083039A0029460A481044FEF739FE2046AD
:107C1000D6E7826C054B1B68DB6A9A4201D20120D1
:107C2000CEE70020CCE70020704700BF74040010AE
:107C30008004001020050010002849D038B5044603
:107C4000264A1268824208D04FF0280383F3118835
:107C5000BFF36F8FBFF34F8FFEE7C26C42B94FF097
:107C6000280383F31188BFF36F8FBFF34F8FFEE7B5
:107C7000013AC264C06AA16C88422BD062BB251D48
:107C80002846FEF723FE70B9E26A142303FB02F3D1
:107C90001349CB583BB9012303FA02F211490B688F
:107CA00023EA02030B60A36CE362C3F10702A26143
:107CB000012404FA03F20B49086802430A602946CA
:107CC000074A142000FB0320FEF7DAFD204638BDEA
:107CD000002070470020FAE70020F8E77404001045
:107CE0008004001020050010002855D038B5034648
:107CF000C06C40B94FF0280383F31188BFF36F8F36
:107D0000BFF34F8FFEE79A6C8A4200D20A46D96AC7
:107D1000914201D0012800D038BD20480068984227
:107D200008D14FF0280383F31188BFF36F8FBFF39F
:107D30004F8FFEE7DA629869002802DBC2F1070282
:107D40009A615A691648142404FB01018A42E3D15E
:107D50001C461D1D2846FEF7B9FD70B9E26A1423C2
:107D600003FB02F30E49CB583BB9012303FA02F29D
:107D70000C490B6823EA02030B60E26A012393407B
:107D80000849086803430B602946054B142000FB93
:107D90000230FEF775FDBFE7704700BF74040010A6
:107DA0008004001020050010044A136898691368C5
:107DB000DB6A1268C3F10703936170477404001013
:107DC000054B1B6823B1044B1A68D36C0133D36491
:107DD000014B1868704700BF7404001038B50546A1
:107DE0000C46FAF72FFC194B1B681B6D2BB9174B70
:107DF0001B68012283F85420ACB9FAF745FCFAF766
:107E000021FC124B1B681C6D24B1CDB90F4B1B68B4
:107E1000621E1A650D4B1B68002283F85420FAF786
:107E200033FC204638BD11462046FFF7D9FA084BEF
:107E30004FF080521A60BFF34F8FBFF36F8FDCE7B4
:107E4000024B1B6800221A65E4E700BF74040010AF
:107E500004ED00E0F8B540B94FF0280383F3118832
:107E6000BFF36F8FBFF34F8FFEE704460D46FAF75F
:107E7000D7FCEFF311864FF0280383F31188BFF38B
:107E80006F8FBFF34F8F94F85430DBB2022284F827
:107E90005420226D01322265012B02D086F3118815
:107EA000F8BDA36A43B14FF0280383F31188BFF3F1
:107EB0006F8FBFF34F8FFEE7144B1B68DBB9271D95
:107EC0003846FEF703FDE26A012393401049086833
:107ED00003430B6039460F4B142000FB0230FEF7C2
:107EE000CFFCE26A0C4B1B68DB6A9A42D6D945B1DB
:107EF00001232B60D2E704F118010848FEF7C0FC0B
:107F0000EFE7074B01221A60C8E700BF1805001011
:107F100020050010800400107404001058050010A3
:107F20009C050010064B1A681368B3FA83F35B09CB
:107F3000036013B9D368186870470020704700BF0A
:107F4000A005001008B54160006191420CD8D21A1A
:107F500083699A4201D3012010E0011D094B186882
:107F6000FEF79AFC002009E09A4201D2994206D21B
:107F7000011D054B1868FEF78FFC002008BD01208D
:107F8000FCE700BFA4050010A005001038B5FAF703
:107F900059FB0F4B1B6813B1FAF776FB38BD0D4D3B
:107FA0002846FEF75FFC0C4C2046FEF75BFC0B4BB3
:107FB0001D600B4B1C6000220C210520FEF797FD75
:107FC000034B18600028E7D00649FFF787F8E3E77E
:107FD000D4050010A8050010BC050010A005001075
:107FE000A4050010C015010000B583B0FFF7CEFF57
:107FF0000D4B1B685BB10D4B0193062300930023CF
:108000004FF496720A490B48FFF736FA40B94FF021
:10801000280383F31188BFF36F8FBFF34F8FFEE701
:1080200003B05DF804FB00BFD4050010D8050010B4
:10803000C8150100FD820000C8B130B585B01546F5
:108040000446174A106840B31A46019102950394FA
:1080500005291DDCFFF784FD022811D000231A46F4
:1080600001A90F480068FEF787FD05B030BD4FF04D
:10807000280383F31188BFF36F8FBFF34F8FFEE7A1
:108080000023089A01A906480068FEF775FDECE791
:10809000002301A9FEF72EFEE7E70020E5E700BF79
:1080A000D405001070B582B01A4B1B681A6852B321
:1080B000DB681E68DC68251D2846FEF707FC636A3E
:1080C00020469847E369012BEED1A36933449E42D1
:1080D00007D26360246129460E4B1868FEF7DCFB6B
:1080E000E2E7002100910B4632462046FFF7A4FF4D
:1080F0000028D9D14FF0280383F31188BFF36F8F85
:10810000BFF34F8FFEE7044A10680249086013600E
:1081100002B070BDA0050010A405001038B50546DA
:10812000FFF728FA0446074B1B68834205D8002353
:108130002B60044B1C60204638BDFFF7B3FF0123C2
:108140002B60F6E7D005001070B582B005460E46EC
:10815000144B1B68DB68DC68201DFEF7B7FBE36986
:10816000012B04D0636A2046984702B070BDA16914
:108170002B46324629442046FFF7E4FE0028F1D082
:10818000002100910B462A462046FFF755FF0028A4
:10819000E8D14FF0280383F31188BFF36F8FBFF34B
:1081A0004F8FFEE7A005001070B582B006460C4662
:1081B000FFF7D8F901A8FFF7B1FF019B1BBB0546EC
:1081C0000CB9B04218D22CB1114B1B681C68B4FA20
:1081D00084F464092246711B0E4B1868FEF7BAFF3F
:1081E000FFF75AFA88B90C4B4FF080521A60BFF370
:1081F0004F8FBFF36F8F08E0FFF74EFA29463046E6
:10820000FFF7A2FF01E0FFF747FA02B070BD00BF21
:10821000A4050010D405001004ED00E030B587B0CF
:10822000002203A9344B1868FEF7CAFD002860D06D
:10823000039B002BF4DB059C636913B1201DFEF743
:1082400045FB02A8FFF76AFF039B092BE8D801A2B0
:1082500052F823F07D8200007D8200007D820000C4
:1082600021820000C5820000EB8200007D820000B8
:108270007D82000021820000C58200000499A5696A
:108280000B46024629442046FFF75CFE0028C7D073
:10829000636A20469847E369012BC1D1A269002196
:1082A00000910B46049802442046FFF7C5FE0028C3
:1082B000B6D14FF0280383F31188BFF36F8FBFF35C
:1082C0004F8FFEE70499A16131B103460246014494
:1082D0002046FFF737FEA3E74FF0280383F311880A
:1082E000BFF36F8FBFF34F8FFEE72046FAF7A2F878
:1082F00096E707B030BD00BFD405001000B583B0CD
:1083000001A8FFF70FFE0199FFF74EFFFFF786FF69
:10831000F6E7F8B51746446B866A002005460BE081
:10832000192003F0DBF8002006E0324604F13C019E
:10833000206805F0DDFC0544BD420CDA0644226CE1
:10834000A36CE16C5B1AD21A1F2AE9DD7B1B9342F6
:10835000EBDB1346E9E7D4E90623501943EBE5715B
:10836000C4E906010020F8BD08B501F0DDF9124BA3
:108370005B6913F0200F1CD0002000F0F9FE3221C1
:108380000E4B1868FEF7C8FD0028F0D000F0F8FF8B
:1083900000231A46194609480068FEF7EDFB00F075
:1083A000C1FE022000F0E4FE4FF4FA70FFF7EEF990
:1083B000DDE70120E1E700BF00C00920DC05001077
:1083C00008B503F035FD03F0C5FA01F0DFF908BD8B
:1083D00070B506464FF0804005F0F0FC4FF0804449
:1083E00001252561002003F00BFF800806FB00F645
:1083F0006660236843F0030323600C21204605F0E8
:10840000ECFC23682B432360AA23A3605523A360BD
:10841000034BC3F880511D60024B1D7070BD00BF3F
:1084200000E100E07442001010B586B00A23039307
:1084300002248DF81140030A43EA0023ADF81230FC
:10844000062201212046FBF70DFEB0F1FF3F15D0BB
:108450000446082204A9FBF7F7FE88B90421204648
:10846000FCF702FA70B90423009303AB0022114613
:108470002046FCF75CFB204606B010BD0024FAE75E
:108480000024F8E70024F6E770B506460D461446CA
:10849000B4B10023224629463046FCF75CF9002897
:1084A00010DB844201DC002070BD0544241A074B18
:1084B0004FF080521A60BFF34F8FBFF36F8FE7E723
:1084C0002046F1E74FF0FF30EEE700BF04ED00E09B
:1084D0002DE9F04F83B000AF8146C2B0C7F804D099
:1084E000456BFFF747F83860E8464FF0000B5E46F3
:1084F00035E04FF0000A04E04FF0010A01E04FF0D0
:10850000000ABAF1000F03D000247B689C550AE0F2
:10851000FFF730F83B68C01AFF2EF5DC0128F3D8CE
:10852000A0441CE00134022C09DCA31D59F82300EF
:108530000028F7D032467968FFF7A6FFF2E7BAF1D4
:10854000000F01D1FF2E29DD0BF1010BBBF1040F50
:1085500024DCFFF70FF83860D7F80480002629469E
:1085600051F8280BC6F58073424605F0F1FB04462E
:10857000D5E90423101843EBE471C5E90401361969
:108580000CD00023A342BADA95F85820012AB0D1C2
:1085900018F803200A2AAFD00133F3E70C37BD46A1
:1085A000BDE8F08F38B505460C46084607F01BFEBF
:1085B000024621462846FFF767FF38BD2DE9F04106
:1085C00088B006460C46456B8B1D50F8238001F0A1
:1085D0003FFF074690B904F1080305EB83035B688E
:1085E00083B1083405EB84046268023208496846A6
:1085F00005F052FC69464046FFF7D4FF384608B004
:10860000BDE8F08104F1080305EB83035E60E8E751
:108610009816010030B589B08B1D50F8235001F039
:10862000BFF9044610B1204609B030BD0449684680
:1086300005F032FC69462846FFF7B4FFF3E700BFB8
:108640008C16010008B54FF480721249124805F0EB
:10865000E4FB0123002204E00F49895C0B44DBB2F8
:1086600001329B2AF8D90C4A92F898209B1A594259
:10867000DBB2C9B258BF4B42DBB292B29A4207D0CA
:108680004FF480720021044805F0CBFB012008BDA7
:108690000020FCE700FC07008006001010B5002356
:1086A000104A82F89830012204E00E49C95C0A445D
:1086B000D2B201339B2BF8D90A4C84F898201D21A3
:1086C000084600F007FB1D21084600F0E7FA1D21CF
:1086D000084600F0FFFA4FF480720349204600F08C
:1086E00009FB10BD8006001000FC0700FEE7FEE756
:1086F000C8B930B583B00C4C0C4B019302250095E2
:108700000B4B4FF496720B492046FEF7B5FE0A4B11
:1087100001930095094B4FF4967209492046FEF7E4
:10872000ABFE03B030BD7047C98A00006C12001068
:108730001C070010C016010070120010780800100D
:10874000C8160100FEE7FFFF2DE9F04707460D467A
:108750004FF48070F9F7FEFD002870D080464FF48A
:108760008070F9F7F7FD814600286AD04FF48072D7
:108770000021404605F055FB4FF480720021484629
:1087800005F04FFB2C220021384605F04AFB2C2235
:108790000021284605F045FB38220021894805F0D4
:1087A00040FB38220021884805F03BFB382200219D
:1087B000864805F036FB38220021854805F031FB5C
:1087C00060220021834805F02CFB602200218248B2
:1087D00005F027FB30220021804805F022FBFFF73F
:1087E00031FF80BB7E4C062221467E4805F015FBFA
:1087F000A11D7D4807F0D6FC04F116017B4807F067
:10880000D1FC04F126017A4807F0CCFC01246D4E1E
:108810004FF0000A304600F802AB764907F0C2FC80
:1088200086F801A0744BF362C6F8288037636B4B5F
:108830007363F4B16A4B5B8FDBB1B38420E0FFF765
:1088400081FFFFF77FFF664C06226649204605F050
:10885000E4FA6549A01D07F0A5FC644904F116007F
:1088600007F0A0FC624904F1260007F09BFC0024FD
:10887000CDE742F21073534A9384594A5387002438
:10888000504A537803F00F03554981F83830534B61
:108890004D4E1E604D4959609A604D4ADA6004227F
:1088A0001A624FF0010A304600F802AB534907F054
:1088B00079FC86F801A0524BF362C6F82890356324
:1088C000444B73632CB1464BB3F846300BB1B384C1
:1088D00007E042F211733C4A9384414AA2F84630C1
:1088E0000024394B5A7802F00F023D4B83F84420A4
:1088F00003F14C02996C374802F0A4FD334E304628
:10890000022300F8023B3F4907F04CFC012373703F
:108910003B4BF362C6F8289035632F4B736334B337
:108920002F4BB3F85220B284284B5A7802F00F0232
:108930002B4B83F8502003F15802596D264802F062
:10894000A7FD234E3046032300F8023B2E4907F0D3
:1089500029FC022373702D4BF362C6F8288037631D
:108960006CB11F4BB3F85E304BB1B3840FE042F2F1
:108970001273164A93841A4AA2F85230D4E742F28C
:108980001373134A9384164AA2F85E300024104BE6
:108990005B7803F00F03124A82F85C307CB102234B
:1089A0003B62084A3A600A4A7A60012285F824202C
:1089B0002B62054B2B60054B6B60BDE8F087FFF722
:1089C0006DFEECE71806001048070010E0070010E5
:1089D000E005001080070010180800105006001075
:1089E000800600108C0000106C0000105C0000106D
:1089F0007C000010A0160100BD850000A816010033
:108A000013830000B0160100B8160100158600009F
:108A100000B58DB006AC214D0FCD0FC495E8030015
:108A200084E8030006A8F9F743FDFFF7C9FC1C49D9
:108A30001C48FFF789FE032200210120FEF757F8AA
:108A4000194B186020B100231A461946FEF794F816
:108A50001648FBF7E9FC05901548FBF7E5FC049088
:108A60001448FBF7E1FC039000240CAB43F8284DBD
:108A7000114A009203AA04A905A8FAF791FF0F4B27
:108A800001930223009323464FF496720C490D483C
:108A9000FEF7F2FCFEF722FDFEE700BFD015010055
:108AA000780800101C070010DC0500106C00001096
:108AB0007C0000105C0000108C0000106812001098
:108AC000B8160100698300002DE9F04397B006460F
:108AD0000A23029390F8243033B94FF00A08FBF7C9
:108AE0000CFBB06200240DE04FF00008F7E756F8E9
:108AF0002450A88CFFF798FC68610522B16AFBF747
:108B000011FB0134336AA342F1DCA9E056F82400DA
:108B1000FFF7DEFC0134336AA342F7DCA5E0002452
:108B2000F9E75948FFF70EFE04F1060955F8290048
:108B300002F004FD0522B16A55F82900FBF717FB86
:108B4000002345F829300134022C26DCA31D55F8FA
:108B500023000028F7D0B16AFBF72CFB0028F2D0E5
:108B6000A01D00234FF48072A96A55F82000FBF77E
:108B70004BFD021ED8DDEB6A2146284698470028A7
:108B8000D2DB6B78012BDED0404B4FF080521A6065
:108B9000BFF34F8FBFF36F8FD5E7686918B1B16A24
:108BA000FBF708FB38B90137336ABB4255DD56F88D
:108BB00027500024C8E716AA082342F80C3D14A940
:108BC0006869FBF796FC81460423009302AB002200
:108BD0001146FBF7ACFF0024022C0DDCA31D55F859
:108BE00023300BB10134F7E70522B16A4846FBF7A1
:108BF00099FAA31D45F82390022C13DCF9F752FCD7
:108C0000B0F5005F16D36B78012B1BD16B78012B6D
:108C1000C9D01E4B4FF080521A60BFF34F8FBFF385
:108C20006F8FC0E71A494846FFF7BCFC484602F080
:108C300085FCB8E717494846FFF7B4FC484602F000
:108C40007DFCB0E7AA1C1346134903A805F024F9DC
:108C500003A94846FFF7A6FCD8E796F824307BB175
:108C600096F82430002B7FF45AAF4146B06AFBF7E8
:108C7000BEFA0028FFF655AF0028F1D0002793E791
:108C8000322002F02BFCEBE7E815010004ED00E0D8
:108C9000F01501001C1601006816010000B58BB02C
:108CA0003423059306900791074B1B68074AA2FBE4
:108CB00003239B09089301A905A8054B9847019830
:108CC0000BB05DF804FB00BF98630010D34D621039
:108CD000F11FFF1F00B58BB032230593069007915B
:108CE00001A905A8024B984701980BB05DF804FB59
:108CF000F11FFF1F00B58BB033230593069107903A
:108D00000892074B1B68074AA2FB03239B090993A0
:108D100001A905A8044B984701980BB05DF804FB26
:108D200098630010D34D6210F11FFF1F10B5044669
:108D300004F096F918B9204604F0DAF910BD20467F
:108D400004F0A6F9FAE7FFFF30B583B004460D46FC
:108D500000238DF80730B1F1FF3F2CD001238B4069
:108D6000DBB28DF80630154B1968A1420CD04900D2
:108D7000E03101230DF10702C1F34701002004F0A7
:108D8000E9F8012002F0B4FB0C4B1C600C4B1C609A
:108D90000C4B1D606100E03101230DF10602C1F3AF
:108DA0004701002004F0D6F80446022002F0A0FBA0
:108DB000204603B030BD0023D3E700BF940000106D
:108DC000E84C0010E44C001010B50446A9B901238A
:108DD00003FA00F215490B6823EA02030B601449F9
:108DE00004F046F83CB10B22510901239340114A8B
:108DF00042F8213010BD0A22F6E701460E4805F080
:108E000067FD012303FA04F208490B6813430B6062
:108E100054B90A2201239340064AC2F88030074918
:108E2000204604F025F8E5E70B22F3E7F84C0010A4
:108E300029CD000000E100E0D816010075CD00004A
:108E400008B50020FFF772FF08BDFFFF38B5084CDA
:108E50004FF48075E561322002F040FBA5613220BD
:108E600002F03CFBE561322002F038FB38BD00BF68
:108E700000C0092008B52E2800DD0230282800DDBA
:108E80000730024600280ADB434200F0070103F0E6
:108E9000070358BF5942D010FFF756FF08BDC21D47
:108EA000F2E7FFFF2DE9F04383B08146884616467E
:108EB0001D469DF82870012400E00134052C14DCC7
:108EC0000095334642464946002004F06FF885423B
:108ED00019D0002FF1D1114A13680133136004EB4C
:108EE0008403580002F004FBE7E700206FB998B94B
:108EF0000B4A1368013313600023AB420ADA0022E5
:108F0000F2540133F9E70120F0E780F0010003B0EB
:108F1000BDE8F0830120FAE70020F8E7004D0010DB
:108F2000084D0010564B03EB40131B7F032B04D05E
:108F3000534B03EB40135B7F03B9704770B588B0A8
:108F40000E460446FFF796FF18B94E4A13680133E0
:108F500013604B4B03EB44135B7F022B77D1484BE1
:108F600003EB44131B7F032B04D02B238DF81C3001
:108F700001250DE0142002F0BBFAF6E7414A136820
:108F80000133136005EB8503580002F0B1FA013597
:108F9000052D53DC97238DF81D3011238DF81E30DD
:108FA000032307AA0B21002003F0D4FF0328E5D1F7
:108FB000012002F09DFA2EB307238DF81D3000200A
:108FC0008DF81E00032307AA0B2103F0C3FF03281B
:108FD0001AD10023009302230DF10A022B210B204A
:108FE000FFF760FFD0B9BDF80A304FF6FF72934229
:108FF0001ED01EB103F00302032A19D12EBBBBB948
:1090000001231CE03346D8E71E4A1368013313607E
:1090100005EB8503580002F06BFAB8E7194A1368AC
:109020000133136005EB8503580002F061FAAEE7E7
:109030002246154903A804F02FFFA8E70023CBB967
:10904000124A13680133136014E00123F7E73F234A
:109050008DF81C3000208DF81D008DF81E60032354
:1090600007AA0B2103F076FF032803D0054A1368F3
:1090700001331360024800EB4410067708B070BD5E
:1090800080420010004D0010F8160100084D00103D
:1090900038B50546002404E029462046FFF742FF84
:1090A0000134362CF8DD38BD014B1868704700BF1D
:1090B000004D0010014B1868704700BF084D0010AC
:1090C000014B1888704700BF60490010014B1868B9
:1090D000704700BFF04C0010014B1888704700BF6C
:1090E000EC4C0010004870470C4D0010034B1B78EF
:1090F00013B1034B18787047002070477C42001072
:1091000078420010014B1870704700BFD44C00101B
:10911000024B1A68024B1A60704700BFFC4C0010EB
:10912000D84C001008B50D4B1B781BB10C4B1B78AD
:10913000022B00D008BD0B4B1B680B4A12689B1A10
:10914000782BF7D9094B2022DA614022DA6100201E
:10915000FFF79EFF024B01221A70EBE7D44C001080
:109160007D420010FC4C0010D84C001000C00920BB
:10917000014B1870704700BFF44C001008B52E4822
:10918000026801322D4B83FB02139918D317C3EBEE
:109190002113C3EB03135900531A0360284B1B78A8
:1091A000012B03D083B1022B2BD008BD012100205D
:1091B00002F046FB0121084602F042FB0123214A4E
:1091C0001370214A1370F0E70121002002F038FBF0
:1091D0001C4B1B7813B1184B00221A60164B1B68EE
:1091E0000E2B09DC0121084602F02AFB0023154A58
:1091F0001370154A1370D8E70021012002F020FBFC
:10920000F4E7104B1B78022B02D00B4B00221A60A4
:10921000094B1B68042B07D9074B00221A600A4B25
:109220001A78074B1A70C0E70021084602F008FBC5
:10923000044B02221A70B8E7E04C00108988888835
:10924000F44C0010920000109300001008B50D4A75
:10925000936843F0010393600B48026801320B49A5
:1092600081FB0231D317C3EBE10303EB83039900C6
:10927000531A03601BB9064A136801331360FFF7E2
:109280007DFF08BD00000B40DC4C00106766666681
:10929000FC4C001010B582B0002405E01B4B03EB22
:1092A000441302221A770134FFF720FFA0422BDD7E
:1092B000164B03EB44135B7F022BF4D12046FFF7E0
:1092C000D9FD00208DF8040010238DF805308DF8AD
:1092D0000600032301AA0B2103F03CFE032803D060
:1092E0000B4A136801331360192002F0F7F80323C7
:1092F00001AA0B21002003F02DFE0328CED0044A42
:10930000136801331360C9E702B010BD804200103A
:10931000004D0010F0B583B0B0F1FF3F03D006461A
:109320000127354617E0FFF7E1FE07460026F8E77C
:10933000114A02EB0512C4F13F01002300930223FE
:1093400002EB4402C9B20B20FFF7ACFD0134E4B2DA
:10935000072CEDD90135F319AB420ADD074B03EBBE
:1093600045131B7F032BF5D02846FFF783FD002410
:10937000EEE7014803B0F0BD6449001080420010E0
:109380002DE9F04F89B04FF6FF7B4FF0000947F60B
:10939000FF7AA94B0293CDF80C904C46D7E0A74B2F
:1093A00003EB44135A884FF6FF739A421ED16B1C8D
:1093B000DBB2042D1AD81D46A04A02EB4412012349
:1093C000009302231A4416210B20FFF76BFD00289F
:1093D000E5D09A4B03EB441300225A8003211977FE
:1093E0009A82DA825A831A830126D8E7002E40F047
:1093F000AD80934B1B782BB1904B03EB44139B8AAE
:10940000002B3BD10025009502230DF1160203210C
:109410000B20FFF747FDBDF8162042F4C042ADF81F
:10942000162003238DF81C308DF81D20120A8DF8AC
:109430001E2007AA0B21284603F08CFD009502236D
:109440007E4A02EB44121C210B20FFF72BFD0095F6
:10945000022305AA18210B20FFF724FD50B9BDF8FF
:10946000142040F648539A427ED0744B03EB4413C9
:1094700001225A7700212046FFF754FD6F4D4FEA35
:10948000441808F110062E44002700970223321DCD
:1094900009210B20FFF706FD00970223B21D0F21C3
:1094A0000B20FFF7FFFC08F118062E44009702235B
:1094B000F21817210B20FFF7F5FC00970223324624
:1094C0000A210B20FFF7EEFC4544B5F91820029B5A
:1094D0009A4200DD0292594B03EB44139B8A4B45A1
:1094E00000D99946524500DA92465B4500D29B4628
:1094F000524B03EB44131B7F33B9504B03EB441324
:109500009B7F13F0010F35D14E4B1B7813B94E4A98
:109510001268DAB933B9494B03EB44135B8813F48F
:10952000006F06D1454B03EB44139B7F13F0020FF2
:109530002ED000212046FFF7F5FC404B03EB4413EF
:1095400000221A779A7F22F003029A770134362C90
:1095500023DC2046FFF78EFC18B93C4A1368013320
:1095600013600026354627E7344B03EB44130222F1
:109570005A777FE701212046FFF7D4FC2F4B03EBFE
:10958000441301221A779A7F22F001029A77BBE7EF
:10959000039B0133DBB20393D8E7039B192B0BD852
:1095A000284B1B7843B9284B1B6843B9284B1B68D1
:1095B0003C33254A136002E0234B00221A60224B01
:1095C0001B681BB1224A12689A4214D80121052057
:1095D000FFF7BAFBF8B91D4A13680133136007217E
:1095E0000520FFF7B1FB00283AD1184A1368013370
:1095F000136000256CE00399164805F069F9164BD5
:109600002022DA614022DA610020FFF741FD0D4B94
:1096100001221A70DAE7114D0021009102232A4637
:109620004820FFF73FFC2A88130A43EA0223C3F3CA
:109630000B132B80D3E700BF0080FFFF8042001098
:109640007C4200107D420010044D0010004D0010BF
:10965000FC4C00100817010000C0092060490010F0
:109660002B4D01232A462721002003F073FC3220D2
:1096700001F034FF04232A462721002003F0C5FC13
:10968000042803D0234A13680133136020490A6871
:1096900090B2030A43EA00231F480380130C1B0205
:1096A0009BB243EA12639B080B60A2E7022306AA5F
:1096B0004821002003F0A9FC022816D19DF81820AB
:1096C0009DF8193043EA0223144A22F81530013577
:1096D000042D14DCA91C0520FFF736FB0028E5D17A
:1096E0000C4A136801331360F1E70A4A1368013327
:1096F00013600A4B42F20F7223F81520E7E7084B7C
:1097000001221A70074B1C6009B0BDE8F08F00BF42
:10971000F04C0010004D0010EC4C00100C4D0010EF
:109720007C4200107842001010B5FFF78FFB4FF419
:10973000DC620021114804F074FB002406E04FF0C5
:10974000FF312046FFF700FB0134E4B2072CF6D9C5
:109750000B4C204603F0DCFF3221204603F0F0FFE3
:10976000084B4FF000521A600120FFF7CBFCFFF7C7
:10977000CFFC054B00221A6010BD00BF80420010D4
:1097800000000B4000E100E0FC4C001008B51B4B52
:109790001A6842F010021A601A6842F020021A6039
:1097A0001A6842F040021A601A6842F080021A6099
:1097B0001A6842F480721A601A6842F400721A60E1
:1097C0001022DA612022DA614022DA618022DA6135
:1097D0004FF40072DA610A4B01221A70002002F085
:1097E000CBF8002003F0F6FA0649002003F00CFB4A
:1097F00000210846FFF7E8FA08BD00BF00C00920B5
:109800007D4200108038010010B404460346002059
:1098100001E060B101331A1B8A4206DA1A78202A65
:10982000F7D80028F6D000221A7010BC70471846EE
:10983000F0E730B403460024254602E09DB1012440
:1098400001331A1A8A4209DA1A78202A01D9002C1F
:10985000F6D0202AF2D825B100221A70284630BC52
:1098600070470124ECE71D460124E9E770B5054681
:109870000E46144606F0B7FCA04201D2002070BD8F
:10988000284606F0B0FC0446304606F0ACFC8442A4
:1098900001D90020F3E7284606F0A5FC0246294638
:1098A000304606F0C5FCB0FA80F04009E7E7FFFF5C
:1098B0002DE9F04F83B0074689460023019306F057
:1098C00092FC06285ED90023C9F800303C469B462E
:1098D0001E469A4698461EE0C9F800404FF001081F
:1098E00029E003222D4901A806F0A2FC002839D066
:1098F0004FF0FF3040E00BF1010B0322002101A8E3
:1099000004F08FFA4FF0FF3603E002AA324402F867
:10991000043C01340136E51B384606F064FC854200
:1099200026D22378202B02D8B8F1000FF1D0D9F835
:109930000030002BD0D02378202B03D800232370B5
:109940004FF0010A032E20DC23782E2B02D0BAF12F
:10995000000FDAD0002E1BDD01A806F0F5FB05464E
:109960000028BED0B5F5807F15D8BAF1000FC2D05F
:10997000BBF1030F03D1002003B0BDE8F08F4FF01F
:10998000FF30F9E74FF0FF30F6E74FF0FF30F3E735
:109990004FF0FF30F0E74FF0FF30EDE7AC1601007D
:1099A0002DE9F04F9FB0063150F82150866A002310
:1099B000B354012A02DD3378FF2B0CD0002A03DDDB
:1099C0003378FF2B00F02685072A0AD00024204692
:1099D0001FB0BDE8F08F7378EC2BEFD14FF0FF3460
:1099E000F5E70522B849304606F022FC0446C8B126
:1099F000B64B1B78002B67D00522B549304606F0E0
:109A000017FC0446002840F081804FF47A71B14B76
:109A10001868FDF781FA00285CD1AF492846FEF7A7
:109A2000C1FDD4E7AD4FAE49384604F035FA3E18D3
:109A3000AC49304604F030FA0644AB49304604F0F5
:109A40002BFA0644A949304604F026FA0644A849F0
:109A5000304604F021FA0644A649304604F01CFAC8
:109A60000644A549304604F017FA0644A349304697
:109A700004F012FA0644A249304604F00DFA0644F6
:109A8000A049304604F008FA06449F49304604F0E5
:109A900003FA06449D49304604F0FEF906449C4909
:109AA000304604F0F9F906449A49304604F0F4F9D6
:109AB00006449949304604F0EFF93218D21B394672
:109AC0002846FEF7E1FC82E794492846FEF76AFD46
:109AD00000247CE792492846FEF764FD914B202242
:109AE000DA614022DA614FF40072DA618022DA61D1
:109AF000FFF7D0FB00231A46194676480068FDF7A9
:109B00003BF889492846FEF74DFD60E70522874965
:109B1000304606F08DFB044650B30522844930469A
:109B200006F086FB044650B305228249304606F013
:109B30007FFB044650B305227F49304606F078FB90
:109B40000446002846D17D492846FEF72BFD754B7B
:109B50002022DA614022DA614FF47A715D4B186895
:109B6000FDF7DAF9E0B95C492846FEF71BFD2EE760
:109B7000FFF7CEFA72492846FEF714FD27E7FFF7F4
:109B8000C1FA70492846FEF70DFD20E70120FFF7D6
:109B9000B9FAFFF7BDFA6C492846FEF703FD16E750
:109BA0000120FFF775FA00231A4619464948006854
:109BB000FCF7E2FFFA2001F091FC5A4B20229A6157
:109BC000624B02221A70FFF7A3FA57492846FEF7A4
:109BD000E9FCFCE605225E49304606F029FB044616
:109BE00060BB5C492846FEF7DDFC4E4B2022DA6163
:109BF0004022DA614FF47A71364B1868FDF78CF920
:109C000020B935492846FEF7CDFCE0E60120FFF7F4
:109C10003FFA00231A4619462E480068FCF7ACFFAD
:109C2000FA2001F05BFC3F4B40229A61474B002237
:109C30001A703D492846FEF7B5FCC8E6052246499C
:109C4000304606F0F5FA044628B30522434930466B
:109C500006F0EEFA044650B305224149304606F0BC
:109C6000E7FA0446002840F095803E492846FEF772
:109C700099FC2C4B2022DA614022DA614FF47A7190
:109C8000144B1868FDF748F9002871D1124928468D
:109C9000FEF788FC9BE634492846FEF783FC214BFF
:109CA00080229A6120492846FEF77CFC8FE62F49E6
:109CB0002846FEF777FC1B4B8022DA611A492846BA
:109CC000FEF770FC83E600BF381701007C420010ED
:109CD000FC190100DC050010041A0100A4080010A2
:109CE00040170100781701009C170100CC170100F4
:109CF000FC1701002C1801005C18010090180100ED
:109D0000B8180100E0180100001901004019010015
:109D10007019010098190100C0190100E019010033
:109D2000241A010000C009203C1A0100441A010055
:109D3000681A01008C1A0100B41A0100BC1A010053
:109D40004C1A0100701A0100941A01007D420010A3
:109D5000DC1A0100E41A0100081B0100241B0100A9
:109D6000401B0100481B0100101B01002C1B0100BF
:109D70000020FFF78DF900231A4619463C48006879
:109D8000FCF7FAFE3B4B01221A703B492846FEF7CE
:109D900009FC1CE6F71C02223849384606F048FA4E
:109DA0000446F0B914AA3649304606F06FF9FFF7B9
:109DB0009DF9149A904201DD002A04DA31492846BF
:109DC000FEF7F0FB03E6304B03EB421302219977D9
:109DD0002E4915A804F060F815A92846FEF7E2FB05
:109DE000F5E502222A49384606F022FA0446F0B97F
:109DF00014AA2849304606F049F9FFF777F9149A72
:109E0000904201DD002A04DA1E492846FEF7CAFB0B
:109E1000DDE51D4B03EB4213012199771E4915A87F
:109E200004F03AF815A92846FEF7BCFBCFE5052259
:109E30001A49304606F0FCF90446002840F05F81DC
:109E400017492846FEF7AEFB4FF41671084B186809
:109E5000FDF762F820B913492846FEF7A3FBB6E5E3
:109E600000238DF875308DF87430A0460E4E4AE010
:109E7000DC0500107D4200103C1A01006C1B010043
:109E8000681B0100701B010080420010881B01004C
:109E9000A41B0100A01B0100A81B0100BC1B0100AA
:109EA000C41B0100E41B0100A4080010B64B1B6892
:109EB0001593B6494FEA48128F183B7F06F1010906
:109EC0001EA8034413F8243C33708B5AB7F91820AA
:109ED000B98AF88A7E8BB7F802C0CDF810C0039615
:109EE0000290019100924246A949484603F0D4FFEE
:109EF00009EB00067B7F012B00F0F580022B00F0C0
:109F0000F88008F10108FFF7F1F84045CEDC0023A6
:109F10001A4619469F480068FCF72EFEFFF7D0F856
:109F200007F0ACFA4FF0765107F010F98146FFF7D1
:109F3000CDF807F0A3FA984907F008F9974907F018
:109F4000B9F98046FFF7C8F807F098FA944907F086
:109F5000FDF88246FFF7C6F80746484607F092FA32
:109F60000022904B06F06CFDCDE90E01404607F053
:109F700089FA00228B4B06F063FD804689465046E5
:109F800007F080FA0022874B06F05AFD82468B4686
:109F90004046494606F0FAFF8046DDE90E0106F02C
:109FA000F5FF81465046594606F0F0FF00904346C3
:109FB0004A467D49304603F06FFF06443A887B8865
:109FC000B988F888B7F808C0CDF808C001900091AA
:109FD0007649304603F060FF0644388807F019F8E8
:109FE00063A3D3E9002306F02BFDCDE90E017888A9
:109FF00007F00FF85EA3D3E9002306F021FD8046A9
:10A000008946B88807F005F85BA3D3E9002306F07A
:10A0100017FD82468B46F88806F0FBFF56A3D3E96E
:10A02000002306F00DFDCDE91001388906F0F1FF9F
:10A0300053A3D3E9002306F003FDCDE91201404606
:10A04000494606F0A3FF8046DDE90E0106F09EFFBB
:10A050008146DDE9120106F099FF0290DDE9100169
:10A0600006F094FF01905046594606F08FFF00908D
:10A0700043464A464E49304603F00EFF06449DF8DB
:10A0800075309DF874204B49304603F005FF0644B7
:10A09000494F7A69C2F340124849304603F0FCFE4A
:10A0A00006447A69C2F380124549304603F0F4FE53
:10A0B00006447A69C2F3C0124249304603F0ECFE0E
:10A0C0000644FEF7F1FF0746FEF7F4FF03463A4663
:10A0D0003D49304603F0E0FE32183C49521A28460A
:10A0E000FEF7D2F973E49DF8743001338DF87430C3
:10A0F00007E79DF8753001338DF8753001E70222CE
:10A100003349384606F094F80446002840F0AB8006
:10A1100015AA3049304605F0B9FF159B632B12D1C3
:10A120004FF0FF331593FEF7E1FF8046FEF7DEFFA9
:10A13000159B984202DDB3F1FF3F07DA2649284616
:10A14000FEF730FA43E44FF00108EFE723492846D1
:10A15000FEF728FA4FF416710E4B1868FCF7DCFE78
:10A1600000283FD11E492846FEF71CFA2FE400BF05
:10A1700049F59D5F94A0B73F8B8862F20698B93F7E
:10A1800030B8E68EFE97C93F3417010080420010B8
:10A19000041C0100DC0500100805253C00002042DD
:10A1A0001004C83B000024402C1C0100441C01008A
:10A1B000681C0100841C010000C00920A41C0100CF
:10A1C000B01C0100BC1C0100C81C0100A408001048
:10A1D000F01C0100EC1C0100701B0100F41C0100CC
:10A1E000E41B01001598FFF795F88146159BB3F124
:10A1F000FF3F01D100231593159E894F159B4344C2
:10A20000B3420DDC00231A46194686480068FCF765
:10A21000B3FC83497A1A2846FEF736F9FFF7D7BB15
:10A22000330109EB030239F8033051889088B2F802
:10A2300006C0B2F808E0B2F80AA0B2F80CB0D289B1
:10A240000692CDF814B0CDF810A0CDF80CE0CDF802
:10A2500008C00190009132467349384603F01CFE55
:10A2600007440136CAE705227049304605F0E0FF91
:10A270000446002840F0D1804FF41671694B1868ED
:10A28000FCF74AFE002840F0B98069492846FEF7ED
:10A2900089F9FFF79CBB674B03EB4613988A584537
:10A2A00000D283460E9B984200D90E90B8B18244EA
:10A2B00007F0E4F812905F4B03EB4613B3F9180074
:10A2C00007F0D3F8129906F041FF5B4906F096FFBC
:10A2D0000146109807F05EF8109009F10109554BFE
:10A2E00003EB4613DB8A03B19844524B03EB46134E
:10A2F000B3F918301F440136FEF7F8FEB042CADC4D
:10A3000000231A46194647480068FCF735FC5846B2
:10A3100007F0B4F8494906F071FF06460E9807F0B9
:10A32000ADF8464906F06AFF0E90504607F09DF8DA
:10A330008246484607F099F881460146504606F0A5
:10A340005DFF3E4906F05AFF8346404607F08DF810
:10A35000494606F053FF394906F050FF804638461B
:10A3600007F083F8354906F049FF0746FEF7AEFED1
:10A3700007F084F8324906F0E9FE324906F09AFF08
:10A380008146FEF7A9FE07F079F82F4906F0DEFEB8
:10A390008246304607F076F8CDE91201204E50464D
:10A3A00007F070F8CDE90C01484607F06BF8CDE9ED
:10A3B0000A01109807F066F8CDE90801384607F061
:10A3C00061F8CDE90601404607F05CF8CDE90401EB
:10A3D000584607F057F8CDE902010E9807F052F8F9
:10A3E000CDE90001DDE912231849304603F054FDA0
:10A3F00031462846FEF7D6F8FFF7E9BAA046A2464E
:10A400002746A14626460023109300230E934FF6BD
:10A41000FF7B71E70124FFF7DABA0024FFF7D7BA10
:10A42000A4080010DC0500101C1D01004C1D0100DB
:10A43000E41B0100804200100024744900007A44AB
:10A440000805253C000020421004C83B541D0100B3
:10A450002DE9F04F95B0466B01F1080306EB83033D
:10A460005D688B1D50F82340836A012A02DD1F7846
:10A47000FF2F41D0002A03DD1F78FF2F00F0EF856A
:10A4800003EB020900279F54002D3CD08B46069019
:10A49000083106EB8101496891F8018011461846A0
:10A4A000FFF7B2F90746002800F0DB8505F09BFEB8
:10A4B00007EB000AA9EB0A090022B5493846FFF765
:10A4C000D5F938BBB8F1000F00F09780B8F1000F54
:10A4D00000F0F680B8F1000F40F0A4810022AD49F1
:10A4E0003846FFF7C3F9002800F09C81AA4B0027EB
:10A4F0001F709846A1463EE15F78EC2FBAD14FF02D
:10A50000FF3300F0AFBD01F1080506EB850568607B
:10A510000546BBE7A04EAA1CA049304603F0BCFC90
:10A520003518B8F1010F48D0B8F1020F5FD09C493F
:10A53000284603F0B1FC05449A49284603F0ACFCD8
:10A5400005449949284603F0A7FC05449749284645
:10A5500003F0A2FC05449649284603F09DFC0544FF
:10A560009449284603F098FC05449349284603F093
:10A5700093FC05449149284603F08EFC054490491C
:10A58000284603F089FC05448E49284603F084FCE4
:10A5900005448D49284603F07FFC05448B49284635
:10A5A00003F07AFC8A49284403F076FC7A49204675
:10A5B000FDF7F8FF002300F055BD8649284603F05B
:10A5C0006BFC05448449284603F066FC0544834936
:10A5D000284603F061FC05448149284603F05CFCF1
:10A5E00005448049284603F057FC0544D1E77E49DD
:10A5F000284603F051FC0544CBE700227B4938464E
:10A60000FFF734F900283FF461AF49465046FFF7A1
:10A6100010F9074668B10025336AAB4243DD56F8AE
:10A6200025100231384605F09BFD034690B30135F5
:10A63000F2E7594D6E49284603F02EFC05440027E9
:10A6400014E056F827305B78012B19D0022B1CD070
:10A6500068490EA805F0A6FD56F827200EAB023279
:10A660006549284603F018FC05440137336ABB42AC
:10A67000E7DC49492046FDF795FF002300F0F2BCD6
:10A680005E490EA805F08EFDE6E75D490EA805F0CF
:10A6900089FDE1E756F825100BF1080206EB82066A
:10A6A000716000F0DFBC3C4D3A465649284603F045
:10A6B000F3FB29462046FDF775FF002300F0D2BCCE
:10A6C000002251493846FFF7D1F800283FF402AF85
:10A6D0004E492046FDF766FFFA2000F0FFFE2046B7
:10A6E00000F02CFF4A4B1B7843B14FF0804301220E
:10A6F0005A60AA229A6055229A60FEE70020FDF770
:10A7000067FEFAE743490BA805F04CFD0BAB00933D
:10A710000EAB52464049404603F0BEFB8044013533
:10A72000022D27DC7B1C03EB83035A0002EB050A96
:10A7300056F82730AA1D53F82240002CEFD009A963
:10A740002046FAF7AEF90A9A130E0193C2F30743B3
:10A750000093C2F30723D2B230490EA803F09CFB4A
:10A76000A145CFD056F8272002322D490BA803F07F
:10A7700093FBCBE70137336ABB4201DD0025CFE70E
:10A7800005494846FDF70EFF002300F06BBC00BFF3
:10A79000181E0100D4210100A4080010201E010091
:10A7A000601F01007C1F0100A41F0100DC1F0100CD
:10A7B000142001005020010088200100B020010079
:10A7C000DC200100FC2001001C21010054210100BB
:10A7D000E01B0100341E0100641E0100A81E0100E0
:10A7E000CC1E01000C1F0100341F01007421010068
:10A7F00078210100A01601009021010088210100AC
:10A80000B81601009C210100B8210100C0210100FF
:10A8100074420010E8210100F8210100DC21010050
:10A82000F02101000022C1493846FFF71FF80790C8
:10A8300000284AD1B8F1000F00F0CF80B8F1000F26
:10A8400000F0FC80B8F1000F00F02981B8F1000F92
:10A8500000F05681B8F1000F00F0CE81B8F1000F82
:10A8600007D10022B2493846FFF700F8002840F02F
:10A870004F82B8F1010F00F06B82B8F1010F00F0C8
:10A880007982B8F1010F00F0B682B8F1010F00F043
:10A890003A83B8F1010F00F08783B8F1020F00F09E
:10A8A000C1830022A3493846FEF7E0FF002800F0EC
:10A8B000D0830BF1080306EB830600237360069B2D
:10A8C0009D4200F0C3830023CCE349465046FEF787
:10A8D000B0FF804628B998492046FDF763FE002363
:10A8E000C0E305F031FC0746421E4FF6FE739A4264
:10A8F0000DD8AB8C834216D00022336A93422BDDF5
:10A9000056F82230998CB94219D00132F5E78B4DB7
:10A9100042468B49284603F0BFFA29462046FDF7F8
:10A9200041FE00239EE3854D02468649284603F0FA
:10A93000B3FA29462046FDF735FE002392E37F4D0A
:10A9400002333A468049284603F0A6FA29462046B3
:10A95000FDF728FE002385E3784E3A467B493046D2
:10A9600003F09AFA31462046FDF71CFE0024022C23
:10A9700012DCA31D55F8230060B100F0DFFD2B6B46
:10A98000A61D0522996A55F82600F9F7F0FB002369
:10A9900045F826300134EAE7642000F09FFD68693D
:10A9A00000F0CCFD2B6B0522996A6869F9F7DFFB93
:10A9B000BFB2AF843846FDF737FD68612B6B0522C7
:10A9C000996AF9F7AFFB2B78614A0C2101FB03234D
:10A9D0005F87FDF763FE002344E300225D493846AC
:10A9E000FEF744FF00283FF429AF00230E934946A9
:10A9F0005046FEF71EFF28B94F492046FDF7D2FD0D
:10AA000000232FE30EA9FEF753FFB0F1FF3F04D15F
:10AA100051492046FDF7C6FDF2E70E994F4805F073
:10AA2000C1FBFDF73BFE454D0E9A4D49284603F00C
:10AA300033FA29462046FDF7B5FDE1E700224949F2
:10AA40003846FEF713FF00283FF4FCAE00230E93B8
:10AA500049465046FEF7EDFE28B937492046FDF736
:10AA6000A1FD0023FEE20EA9FEF722FFB0F1FF3F99
:10AA700004D139492046FDF795FDF2E70E993A4891
:10AA800005F090FBFDF70AFE2C4D0E9A374928463B
:10AA900003F002FA29462046FDF784FDE1E7002293
:10AAA00033493846FEF7E2FE00283FF4CFAE0023DC
:10AAB0000E9349465046FEF7BCFE28B91E49204673
:10AAC000FDF770FD0023CDE20EA9FEF7F1FEB0F117
:10AAD000FF3F04D127492046FDF764FDF2E70E99B8
:10AAE000254805F05FFBFDF7D9FD144D0E9A23496B
:10AAF000284603F0D1F929462046FDF753FDE1E74A
:10AB000000221F493846FEF7B1FE059000283FF4A9
:10AB1000A1AE49465046FEF78CFE064690BB06495C
:10AB20002046FDF73FFD00239CE200BF0822010004
:10AB30009C240100A026010010220100A40800109E
:10AB40002822010040220100642201008C22010021
:10AB500080060010C0220100C422010086060010F9
:10AB6000E02201000C2301009606001010230100D2
:10AB70004023010044230100A60600105C230100CD
:10AB80008423010005F02FFB112804D0A44920469E
:10AB9000FDF708FDC7E70025052D17DC05EB45008F
:10ABA000831CF25C042D03DC2D2A01D03A2A0FD13C
:10ABB0000021F1541022304405F088FAFF2807D80C
:10ABC00014AB2B4403F8180C0135E5E7079B0593FC
:10ABD000059B002BDAD106220EA9924803F01DF93D
:10ABE000FDF75CFD904D9149284603F055F9294643
:10ABF0002046FDF7D7FC96E700228D493846FEF740
:10AC000035FE00283FF42AAE874EAA8C894930468B
:10AC100003F042F93518884E32468849284603F039
:10AC20003BF905443146864805F09AFA002858D089
:10AC3000834A8449284603F02FF90544824E324660
:10AC40008249284603F028F905443146804805F03A
:10AC500087FA00284BD07E4A7A49284603F01CF92F
:10AC600005447C4E32467C49284603F015F90544DC
:10AC700031467A4805F074FA00283ED0774A714987
:10AC8000284603F009F90544754E32787378B17897
:10AC9000F078377996F805C0CDF80CC0029701908E
:10ACA00000917049284603F0F7F805440622314622
:10ACB0005C4803F037FE30B35A490A784B788878FD
:10ACC000CE780F79497903910297019600906649F1
:10ACD000284603F0E1F854492046FDF763FC0023C1
:10ACE000C0E16249284603F0D7F80544A6E75F496A
:10ACF000284603F0D1F80544B3E75C49284603F041
:10AD0000CBF80544C0E75949284603F0C5F8E2E707
:10AD1000454D574A5749284603F0BEF805440422DA
:10AD20005549564B186805F083FA60B9534B1A68B9
:10AD300004325349284603F0AFF83B492046FDF75B
:10AD400031FC00238EE14F49284603F0A5F8F4E7D3
:10AD500002224D493846FEF789FD00283FF48DADAB
:10AD60006D6B4A492046FDF71DFC287900F02AFA50
:10AD7000002377E1022246493846FEF777FD002896
:10AD80003FF47FAD49465046FEF753FD074628B9CC
:10AD900040492046FDF706FC002363E105F0D4F9A5
:10ADA000061E0ADC3A463C491F4803F075F81E4966
:10ADB0002046FDF7F7FB002354E1686B0022009268
:10ADC000194B314600F032FA0028F0D132463349AF
:10ADD000154803F061F82B7812490C2202FB03128C
:10ADE000D26BB242E3D00A460C2101FB0323DE639F
:10ADF000FDF754FCDBE7002229493846FEF736FD13
:10AE000000283FF442AD49465046FEF712FD064683
:10AE1000002847D11F492046FDF7C4FB002321E14C
:10AE20008823010080060010A4080010C023010040
:10AE3000EC230100F42301006C0000100824010041
:10AE4000860600101C2401007C0000102424010050
:10AE5000A60600105C0000103824010096060010C1
:10AE60008C0000104C24010078240100E01B01003C
:10AE7000D0160100A4240100B8240100980000109D
:10AE8000C0240100D4240100E8240100F0240100C2
:10AE900004250100102201000C25010044250100B9
:10AEA00060250100686B00230093704B32464FF021
:10AEB000FF3100F0BBF900BB32787378B1780091B4
:10AEC0006B496A4802F0E8FF2A780C2303FB02F37F
:10AED0004033032231466748184405F0A9F960B1B0
:10AEE0002A780C2303FB02F34033032231466148E6
:10AEF000184405F0C8F9FDF7D1FB5C492046FDF781
:10AF000051FB0023AEE000225B493846FEF7AEFC61
:10AF100000283FF4BEAC6E6B49465046FEF789FCF4
:10AF2000074628B955492046FDF73CFB002399E028
:10AF300005F059F9012805D83A78A2F13003DBB2BF
:10AF4000012B0AD93A464E49484802F0A5FF474925
:10AF50002046FDF727FB002384E04A49434802F0DE
:10AF60009BFF3B78302B10D12B78424A0C2101FB00
:10AF7000032393F8382022F0100283F838200023AE
:10AF800086F85830FDF78AFBE1E72B78394A0C2127
:10AF900001FB032393F8382042F0100283F8382095
:10AFA000012386F85830EDE7002237493846FEF78E
:10AFB0005DFC00283FF471AC6F6B2C4EAA8C3349BA
:10AFC000304602F069FF351807F10C03BA683049C2
:10AFD000284602F061FF054497F85830E3B92D493F
:10AFE000284602F059FF0544D7E906232A49284696
:10AFF00002F052FF0544D7E904232849284602F00D
:10B000004BFF3A6A2649284402F046FF174920467A
:10B01000FDF7C8FA002325E02249284602F03CFF4C
:10B020000544E1E7002218493846FEF71FFC0028D6
:10B030003FF437AC0D4EAA8C1B49304602F02CFF72
:10B0400031462046FDF7AEFA00230BE04FF0FF3308
:10B0500008E016492046FDF7A5FA002302E0012387
:10B0600000E00023184615B0BDE8F08FA4080010DA
:10B0700068250100800600108425010010220100CF
:10B080008C250100B8250100EC230100D825010022
:10B09000F02501000C260100402601005826010081
:10B0A000702601002426010088260100A826010040
:10B0B00008B5034A034B1A6000F0EBFC08BD00BF63
:10B0C0000020000008ED00E010B50446006802F022
:10B0D0004DFD236881229A60206802F083FD4FF4C1
:10B0E00000630122216D04F1280002F059F94FF4A8
:10B0F00000730122616D04F13C0002F051F92368F4
:10B10000C7229A602268536843F00503536094F99C
:10B110000530002B11DB03F1604303F56143082286
:10B1200083F8002394F9053003F01F015B09012225
:10B130008A40054941F8232010BD03F00F03034A5C
:10B140001A4408231376EDE700E100E0FCEC00E090
:10B1500030B585B00446C36A426B816B521A9B1AA4
:10B1600003EB83035A0002F2FF7240F6FE739A4229
:10B170000ED8056ACC3508E01022694604F1280093
:10B1800002F018FA236A18442062236AAB42F3D310
:10B1900004F13C0204F12801206802F0EAFD05B048
:10B1A00030BDFFFF08B50248FFF7D2FF08BD00BF62
:10B1B0008007001008B50248FFF7CAFF08BD00BFAE
:10B1C000180800102DE9F04383B018B1032826D1E8
:10B1D000002600E00226DFF85080002500950823B5
:10B1E00032462946404602F01AF80E4C23684FF0CA
:10B1F000010909FA06F73B432360E3693B43E36136
:10B2000040F2DC5000F06AF9A3693B43A361CDF83A
:10B210000090082332462946404602F000F803B069
:10B22000BDE8F08300C0092000C002402DE9F047CE
:10B2300082B0074615469A469DF828800023ADF84F
:10B24000063038238DF804304E238DF80530312335
:10B250008DF806300E1E19DDB6F5965F25D01BDD84
:10B26000B6F5964F21D037DDB6F5614F1DD0B6F556
:10B27000E13F1AD0B6F5164F17D0B8F1000F32D013
:10B280004FF41653BB604FF0000911E0B8F1000F06
:10B29000E2D14FF000090BE0B6F5167F05D014DCC3
:10B2A0006E2E02D0B6F5967FE7D1BE604FF0000952
:10B2B00025B30024284604F096FFA04225D92A1978
:10B2C0002B5D202B1FD90134F4E7B6F5966FECD037
:10B2D000B6F5166FD1D1E8E7B6F5165FE5D0B6F54D
:10B2E000615FCAD1E1E75249504602F0D5FD5046B0
:10B2F00004F079FF82444FF00109D9E7B8F1000F5B
:10B3000033D100245CE000231370284604F06BFF67
:10B31000022803D8B8F1000F29D001AD2A78A2F194
:10B320003004E4B2A2F13503DBB2032B26D83A7322
:10B33000053C6B78453B2A2B5FD8DFE803F0545E71
:10B340005E5E5E5E5E5E5E2F595E5E5E5E5E5E5E51
:10B350005E5E5E5E5E5E5E5E5E5E5E5E5E5E545E17
:10B360005E5E5E5E5E5E5E2F59000024A2E731499C
:10B37000504602F091FD4FF0010930E0B8F1000FA6
:10B3800003D038233B730324D3E72B49504602F004
:10B3900083FD824400244FF00109CAE74E237B73EA
:10B3A000AA78A2F13103DBB2012B34D9B8F1000F36
:10B3B00033D03123BB73BB7B322B01D144F0040467
:10B3C000B9F1000F0BD1002E02DCB8F1000F03D051
:10B3D000B968386802F01EFC35B33B68DC6048464B
:10B3E00002B0BDE8F08745237B7344F01804D7E72B
:10B3F0004F237B7344F00804D2E7B8F1000F02D06A
:10B400004E237B73CCE70D49504602F045FD824444
:10B410004FF00109C4E7BA73CDE70949504602F07D
:10B420003BFD4FF00109C6E7B8F1000FD5D1D6E7D3
:10B43000B42601002C270100542701008C270100AD
:10B44000BC270100F0B583B004460E4617466022C3
:10B45000002102F0E6FC052363710A4B23600025FE
:10B460002571094B2365094B63652046FFF72CFEC8
:10B47000012300932B463A4631462046FFF7D6FE7D
:10B4800003B0F0BD00C00040184D0010185D001062
:10B4900070B582B004460D4616466022002102F0C7
:10B4A000C0FC082363710A4B236003232371094BFB
:10B4B0002365094B63652046FFF706FE01230093D1
:10B4C0000023324629462046FFF7B0FE02B070BD89
:10B4D00000C0094018550010185F001008B5034B54
:10B4E000A3FB0030C008FCF751F908BDCDCCCCCC93
:10B4F00082B04FF47A7303FB00F000900D4B1A6892
:10B500000D4BA3FB0232D20C009B4BB9009B0133C5
:10B51000009305E0019B01330193019B9A42F9D806
:10B52000009B013B009313B100230193F5E702B0A8
:10B53000704700BF98630010819F5E1630B591B0D0
:10B5400005460221F9F7DCF9002400234022694670
:10B550002846F9F759F8002808DB0220FCF716F90D
:10B56000631CDBB2182C01D81C46EEE72846F8F71E
:10B57000FBFE11B030BD80B582B000AF78600F2007
:10B5800000F04AFD00BF0837BD4680BD80B483B0DF
:10B5900000AF78600B46FB701346BB70FA787B688F
:10B5A0001A3253F82210BB78012202FA03F3FA7818
:10B5B00019437B681A3243F8221000BF0C37BD468E
:10B5C00080BC704780B483B000AF78600B46FB70DE
:10B5D000FA787B68DA6700BF0C37BD4680BC7047DD
:10B5E00080B582B000AF78600F2000F015FD00BF7D
:10B5F0000837BD4680BD80B483B000AF7860084690
:10B6000011461A460346FB700B46BB7013467B700F
:10B610007B78002B0ED0FB785B017A681344996924
:10B62000BB7801229A40FB785B01786803440A43A7
:10B630009A610DE0FB785B017A681344D969BB78A5
:10B6400001229A40FB785B01786803440A43DA617F
:10B6500000BF0C37BD4680BC704780B584B000AFDA
:10B66000F860B96011461A460B46FB711346BB7170
:10B67000BB68D9B2BB79FA79F868FFF7BCFF00BFA5
:10B680001037BD4680BD80B483B000AF78600B46F4
:10B69000FB701346BB70FB785B017A681344196832
:10B6A000BB7801229A40FB785B01786803440A4327
:10B6B0001A6000BF0C37BD4680BC704780B483B0B1
:10B6C00000AF78600B46FB701346BB70FB785B01E4
:10B6D0007A6813441968BB78012202FA03F3DA434B
:10B6E000FB785B01786803440A401A6000BF0C379E
:10B6F000BD4680BC704780B582B000AF7860084618
:10B7000011461A460346FB700B46BB7013467B700E
:10B710007B78002B06D0BA78FB7819467868FFF75B
:10B72000B2FF05E0BA78FB7819467868FFF7C6FFE4
:10B7300000BF0837BD4680BD80B582B000AF7860DD
:10B74000084611461A460346FB700B46BB7013466B
:10B750007B707B78BA78F9787868FFF7CCFF00BF08
:10B760000837BD4680BD80B483B000AF78600B461B
:10B77000FB70FA787B681A6000BF0C37BD4680BC4E
:10B78000704780B483B000AF78607B681B68DBB221
:10B7900018460C37BD4680BC704780B483B000AFFC
:10B7A000786039607B683A68DA6000BF0C37BD4664
:10B7B00080BC704780B483B000AF78607B685B6901
:10B7C00018460C37BD4680BC704780B586B000AFC8
:10B7D000F860B9607A6000237B6109E0BA687B6930
:10B7E00013441B78184600F085F87B6901337B61B0
:10B7F0007B687A699A42F1D37B6818461837BD4650
:10B8000080BD80B582B000AF00F08EF80346FB71BA
:10B81000FB7918460837BD4680BDFFFF80B500AFF5
:10B820000123122201210548FFF786FF01231A2276
:10B8300003210248FFF780FF00BF80BD00C0092040
:10B8400080B582B000AF03460A46FB711346BB7158
:10B85000FB79002B02D0012B12D023E0BB79002B07
:10B8600014BF01230023DBB283F00103DBB203F03A
:10B870000103DBB2122201210C48FFF7EEFE11E0BA
:10B88000BB79002B14BF01230023DBB283F001033B
:10B89000DBB203F00103DBB21A2203210348FFF7F6
:10B8A000DCFE00BF00BF0837BD4680BD00C00920D8
:10B8B00080B483B000AF786000BF0C37BD4680BC59
:10B8C0007047FFFF80B500AF0948FFF7F1FF084858
:10B8D00002F04CF94FF4E131054802F09BF90321E5
:10B8E0000348FFF75AFF024802F07CF900BF80BD11
:10B8F00000C0094080B582B000AF0346FB7100BFB5
:10B900000848FFF757FF034603F02003002BF7D04A
:10B91000FB7919460348FFF726FF00BF0837BD46ED
:10B9200080BD00BF00C0094080B500AF0848FFF7E8
:10B9300041FF034603F00103002B04D00448FFF746
:10B9400020FF034601E04FF0FF33184680BD00BFE3
:10B9500000C0094080B500AFFFF7B4FF0448FFF70F
:10B960003FFE0448FFF707FEFFF758FF00BF80BD0A
:10B9700000C0092000C0024080B584B002AF034679
:10B98000FB71FB79012B19D0022B32D0002B00D098
:10B990004AE00123009308231B220021244801F0E0
:10B9A0003EFC0123009308231C220021204801F0C3
:10B9B00036FC00211E48FFF705FE35E00223009308
:10B9C0000823132200211A4801F029FC02230093C6
:10B9D000082314220021164801F021FC1322002123
:10B9E0001348FFF7D3FD142200211148FFF7CEFDC5
:10B9F0001AE00223009308230A2200210C4801F0D8
:10BA00000EFC0223009308230B220021084801F0BA
:10BA100006FC0A2200210648FFF7B8FD0B22002190
:10BA20000348FFF7B3FD00BF00BF0837BD4680BD28
:10BA300000C0024080B485B000AF0346FB71084BE4
:10BA40001B68C3F30B03FB60FB791B031946044A15
:10BA5000FB680B43136000BF1437BD4680BC7047C2
:10BA600000C00F4080B500AF11220349034801F028
:10BA700020FC00BF80BD00BFFC27010000C00240C9
:10BA800080B500AF01F0E4FE0420FFF7D3FF00BF54
:10BA900080BD80B500AFFFF7E5FFFFF7F1FF00BF06
:10BAA00080BD80B483B000AF78607B685B6B03F0CF
:10BAB0000103002B14BF01230023DBB218460C370F
:10BAC000BD4680BC7047FFFF80B584B000AF034621
:10BAD0000A46FB711346BB800023FB73FA23BB604D
:10BAE000BA88FB7919464FF0A04000F059FC12E0EB
:10BAF0004FF0A040FFF7D5FF0346002B07D0BB68EF
:10BB0000013BBB60084B1B680120984703E0002302
:10BB1000BB600123FB73BB68002BE9DCFB7B184691
:10BB20001037BD4680BD00BF2461001080B584B0D1
:10BB300000AF03463960FB710023FB73FA23BB603F
:10BB4000FB7919464FF0A04000F048FC1DE04FF093
:10BB5000A040FFF7A6FF034683F00103DBB2002BF2
:10BB60000CD00023BB604FF0A04000F04FFC034618
:10BB70001A463B681A800123FB7306E0BB68013B51
:10BB8000BB60064B1B6801209847BB68002BDEDCBE
:10BB9000FB7B18461037BD4680BD00BF24610010F6
:10BBA00080B483B000AF03460A46FB801346BB80D7
:10BBB000FB8803F00403002B06D0314B1B6843F0D5
:10BBC00008032F4A136005E02D4B1B6823F0080380
:10BBD0002B4A1360BB8803F01C03082B1DD0142BC9
:10BBE0000ED0042B26D0264B1B6843F01003244AAA
:10BBF0001360234B1B6843F02003214A136026E0A7
:10BC00001F4B1B6823F010031D4A13601C4B1B685D
:10BC100043F020031A4A136019E0194B1B6843F0E4
:10BC20001003174A1360164B1B6823F02003144AB5
:10BC300013600CE0124B1B6823F01003104A1360D2
:10BC40000F4B1B6823F020030D4A136000BF0C4B01
:10BC50001A680C4B1B68534003F03803002B09D0C3
:10BC6000074B1B68074A1360054B1B6843F004032E
:10BC7000034A136000BF0C37BD4680BC704700BF4D
:10BC8000186100101C61001080B586B000AFB9606B
:10BC90007A603B600346FB7300237B822E4ABB68BD
:10BCA00013602E4B00221A602D4B00221A602C4B81
:10BCB0001B682C4A13604FF400410020FFF704FF7B
:10BCC0000346012B01D0002341E04FF4C8737B6190
:10BCD0001AE0214B1B680120984707F11003194611
:10BCE0000020FFF723FF0346012B01D000232EE0A5
:10BCF0003B8A03F40843002B03D14FF0FF337B61F1
:10BD000002E07B69013B7B617B69002BE1DC7B69A5
:10BD1000002B01D100231AE07B68642B03D17B8ABE
:10BD200043F400537B827B68002B03D17B8A43F46E
:10BD300090537B823B68002B03D07B8A43F4807353
:10BD40007B827B8A19460020FFF7BEFE012318463E
:10BD50001837BD4680BD00BF24610010206100106F
:10BD6000186100101C61001098B500AF2D4B1B68C6
:10BD7000012B16D0022B2FD001214FF0A04000F054
:10BD80002DFB294B1B6823F00403274A1360264B25
:10BD90001B6843F00203244A1360224B01221A60FD
:10BDA0003CE04FF0A040FFF77CFE034683F0010328
:10BDB000DBB2002B2FD04FF0A04000F027FB034652
:10BDC0001A461A4B1A801F214FF0A04000F006FBC4
:10BDD000144B02221A601EE04FF0A040FFF761FEF4
:10BDE000034683F00103DBB2002B16D00E4B1B6819
:10BDF00023F002030C4A13600C4B1C884FF0A04048
:10BE000000F004FB034619462046FFF7C9FE054B28
:10BE100000221A6001E000BF00E000BF024B1B6877
:10BE2000184698BD206100101861001028610010AC
:10BE300080B500AF00F0D8F90246024B1A6000BF8F
:10BE400080BD00BF9863001080B400AF064BD3F8EC
:10BE5000883003F08073002B14BF01230023DBB272
:10BE60001846BD4680BC704700C00F4080B400AF8C
:10BE7000064BD3F8883003F00073002B14BF012366
:10BE80000023DBB21846BD4680BC704700C00F409F
:10BE900080B483B000AF0346FB71094AFB795B01B4
:10BEA00013448C33AA221A60054AFB795B011344C0
:10BEB0008C3355221A6000BF0C37BD4680BC7047DA
:10BEC00000C00F4080B400AF054BD3F80C31DBB29B
:10BED00003F00303DBB21846BD4680BC704700BFC9
:10BEE00000C00F4080B400AF024B1B681846BD462F
:10BEF00080BC7047F427010080B400AF024B1846A5
:10BF0000BD4680BC704700BF00093D0080B400AF53
:10BF1000024B1B681846BD4680BC7047F8270100DD
:10BF200080B500AF00F008F90346184680BDFFFF5A
:10BF300080B584B000AF03463960FB710C4AFB79D1
:10BF400004335B0113441B68FB60FA683B681343CE
:10BF5000FB60074AFB7904335B011344FA681A60FB
:10BF6000FB791846FFF794FF00BF1037BD4680BD30
:10BF700000C00F4080B584B000AF03463960FB714C
:10BF80000D4AFB7904335B0113441B68FB603B687B
:10BF9000DB43FA681340FB60074AFB7904335B011B
:10BFA0001344FA681A60FB791846FFF771FF00BF67
:10BFB0001037BD4680BD00BF00C00F4080B586B0C1
:10BFC00000AF0346B9607A60FB73FB7B002B05D1A1
:10BFD0007B681B04BA6813437B6104E07B685B01E8
:10BFE000BA6813437B610B4AFB7B04335B01134448
:10BFF00004337A691A60074AFB7B04335B011344FC
:10C0000001221A60FB7B1846FFF742FF00BF18377A
:10C01000BD4680BD00C00F4080B485B000AF034670
:10C02000FB71FB79FB60084BD3F8C4300121FA683F
:10C0300001FA02F21146044A0B43C2F8C43000BFB1
:10C040001437BD4680BC704700C00F4080B582B039
:10C0500000AFFFF70BFF0346002B02D00123FB715B
:10C0600001E00023FB71FB7918460837BD4680BD0F
:10C0700080B483B000AF7860044A7B68C2F80431B2
:10C0800000BF0C37BD4680BC704700BF00C00F40EA
:10C0900080B400AF044BD3F80431DBB2013318464F
:10C0A000BD4680BC704700BF00C00F4080B487B061
:10C0B00000AF0346FB7101237B61FB795B003B61B1
:10C0C0003B6903F01F03FB603B695B093B61194A55
:10C0D0003B696A3352F823307B617A69FB6822FA44
:10C0E00003F303F003037B617B69002B02D104237C
:10C0F0007B6119E07B69012B02D101237B6113E095
:10C100007B69022B02D102237B610DE0FB790D2BB1
:10C1100005D0FB790E2B02D0FB790F2B02D1062321
:10C120007B6101E008237B617B6918461C37BD46B3
:10C1300080BC704700C00F4080B500AFFFF7C2FE63
:10C140000346012B07D0022B09D0002B0BD1FFF7A0
:10C15000D3FE034608E0FFF7C5FE034604E0FFF701
:10C16000D5FE034600E00023184680BD80B584B0AC
:10C1700000AF0023FB60FFF767FE0346002B18D0DB
:10C180000E4BD3F88430C3F30E030133BB600B4B6B
:10C19000D3F884301B0CDBB201337B60FFF7C0FEA9
:10C1A0000246BB6803FB02F35A007B68B2FBF3F361
:10C1B000FB60FB6818461037BD4680BD00C00F40CD
:10C1C00080B500AFFFF742FF0346002B05D0012BDF
:10C1D00007D1FFF7CBFF034604E0FFF7ADFF0346AF
:10C1E00000E00023184680BD98B500AFFFF7E8FFD8
:10C1F0000446FFF74DFF0346B4FBF3F3184698BD22
:10C2000090B583B000AF0346FB71FFF7EDFF044626
:10C21000FB791846FFF74AFF0346B4FBF3F31846D1
:10C220000C37BD4690BD80B500AFFFF7DDFF03467C
:10C23000184680BD80B483B000AF78607B684FF44F
:10C240004F421A607B687822C3F8002100BF0C3788
:10C25000BD4680BC704780B584B000AF7860786818
:10C26000FFF7E8FF0023FB6002E0FB680133FB609F
:10C27000FB68632BF9D900BF1037BD4680BD80B580
:10C2800082B000AF78600B46FB701E20FFF7C4FE43
:10C290007868FFF7E0FF7B6802221A607B68312232
:10C2A0005A60FB78002B05D07B684FF4C862C3F856
:10C2B000002104E07B684FF48862C3F800217B68AA
:10C2C00015229A607B681222DA607B684FF48072D4
:10C2D0009A617B684FF4C0625A617B6843F20F72C7
:10C2E0001A617B68D3F8003143F080027B68C3F8A1
:10C2F00000217B684FF6FF72C3F8E82F7B680022AD
:10C30000C3F8E42F00BF0837BD4680BD80B485B0B8
:10C3100000AFF860B9601346FB71FB791B0203F4B0
:10C32000F8530A4A1360BB689B0003F03C0343F4D4
:10C330000042FB681A62FB681B6A23F40042FB6838
:10C340001A6200BF1437BD4680BC70472C610010D4
:10C3500080B584B000AF786039600023FB60FFF7E0
:10C3600062FF02463B68B2FBF3F3BB600023FB6055
:10C370000CE00A4AFB6813441B781A46BB689342D8
:10C3800001D8FB6806E0FB680133FB60FB680E2BFD
:10C39000EFD90E2318461037BD4680BD4028010056
:10C3A00080B483B000AF78600B46FB7013463B80CF
:10C3B0007B6800225A62FB7803F01F02064B1B6861
:10C3C0001A437B689A623A887B68DA6200BF0C374E
:10C3D000BD4680BC704700BF2C61001080B483B0A4
:10C3E00000AF78600B46FB70FB7803F01F02064B32
:10C3F0001B681A437B689A627B6801225A6200BFFD
:10C400000C37BD4680BC70472C61001080B483B0EF
:10C4100000AF78607B6800225A627B681B6B9BB21E
:10C4200018460C37BD4680BC704780B483B000AF5F
:10C4300078607B685B6843F001027B685A607B68C8
:10C44000D3F8003143F480627B68C3F800217B6835
:10C4500015229A6000BF0C37BD4680BC704780B47F
:10C4600083B000AF78607B685B6823F001027B6873
:10C470005A607B68D3F8003123F480627B68C3F88C
:10C4800000217B6812229A6000BF0C37BD4680BC39
:10C49000704780B485B000AFF860B9607A603B60E7
:10C4A000BA68FB68C3F81C213B685A1EFB68C3F8D6
:10C4B00024217A68FB68C3F82021FB680022C3F8B6
:10C4C000282100BF1437BD4680BC704780B485B0BA
:10C4D00000AFF860B9607A603B60BA68FB68C3F887
:10C4E00008213B685A1EFB68C3F810217A68FB6874
:10C4F000C3F80C21FB680022C3F8182100BF1437D1
:10C50000BD4680BC704780B485B000AFF860084677
:10C5100011461A4603467B810B463B811346FB803E
:10C520003A897B899A4201D1002311E03B89002B93
:10C5300006D17A89FB88013B9A4201D1022307E0A8
:10C540003A897B8901339A4201D1022300E0012319
:10C5500018461437BD4680BC704780B485B000AF24
:10C5600078607B68D3F82831FB60FB680133FB609F
:10C570007B68D3F82431FA689A4201D90023FB6022
:10C580007B68FA68C3F82821FB689BB21846143709
:10C59000BD4680BC704780B485B000AF78607B68D2
:10C5A000D3F81831FB60FB680133FB607B68D3F87C
:10C5B0001031FA689A4201D90023FB607B68FA685F
:10C5C000C3F81821FB689BB218461437BD4680BCDF
:10C5D0007047FFFF80B582B000AF0346FB71FA7968
:10C5E00007491346DB009B1A9B000B4404331B785E
:10C5F0001846FFF711FD00BF0837BD4680BD00BFDC
:10C600009C00001080B582B000AF0346FB71FB793F
:10C61000044AD35C1846FFF7F3FD03461846083773
:10C62000BD4680BD5028010080B483B000AF786063
:10C630007B683C229A617B6860221A6000BF0C37DD
:10C64000BD4680BC704780B483B000AF78607B6823
:10C6500038229A617B6844221A6000BF0C37BD46BD
:10C6600080BC704780B483B000AF78607B681B6883
:10C6700003F01003002B0CBF01230023DBB218468C
:10C680000C37BD4680BC704780B483B000AF786083
:10C690007B685B6803F0F80318460C37BD4680BC26
:10C6A000704780B582B000AF78607868FFF7ECFF24
:10C6B00003465F2BD4BF01230023DBB218460837A3
:10C6C000BD4680BD80B483B000AF0346FB710B460E
:10C6D000BB7113467B717B7943F001037B71FA795F
:10C6E000BB795340DBB21A467B79DB431340002B06
:10C6F0000CBF01230023DBB218460C37BD4680BCBB
:10C70000704780B582B000AF78600B46FB70FB7855
:10C710005B08DBB2002B01D100233CE07B68DB68C7
:10C72000D8B27B681B6BDAB2FB781946FFF7CAFFF9
:10C730000346002B01D001232DE07B681B6AD8B291
:10C740007B685B6BDAB2FB781946FFF7BBFF0346E9
:10C75000002B01D002231EE07B685B6AD8B27B68A5
:10C760009B6BDAB2FB781946FFF7ACFF0346002B50
:10C7700001D003230FE07B689B6AD8B27B68DB6B38
:10C78000DAB2FB781946FFF79DFF0346002B01D074
:10C79000042300E0002318460837BD4680BDFFFF94
:10C7A00080B584B000AF786039603C23FB60786866
:10C7B000FFF76AFF0346582B00F2158101A252F8D9
:10C7C00023F000BFD5C90000E7C90000E7C9000099
:10C7D000E7C90000E7C90000E7C90000E7C9000099
:10C7E000E7C9000029C90000E7C90000E7C9000047
:10C7F000E7C90000E7C90000E7C90000E7C9000079
:10C80000E7C9000029C90000E7C90000E7C9000026
:10C81000E7C90000E7C90000E7C90000E7C9000058
:10C82000E7C9000047C90000E7C90000E7C90000E8
:10C83000E7C90000E7C90000E7C90000E7C9000038
:10C84000E7C90000BDC90000E7C90000E7C9000052
:10C85000E7C90000E7C90000E7C90000E7C9000018
:10C86000E7C9000047C90000E7C90000E7C90000A8
:10C87000E7C90000E7C90000E7C90000E7C90000F8
:10C88000E7C90000BDC90000E7C90000E7C9000012
:10C89000E7C90000E7C90000E7C90000E7C90000D8
:10C8A000E7C90000CDC90000E7C90000E7C90000E2
:10C8B000E7C90000E7C90000E7C90000E7C90000B8
:10C8C000E7C90000ABC90000E7C90000E7C90000E4
:10C8D000E7C90000E7C90000E7C90000E7C9000098
:10C8E000E7C90000BDC90000E7C90000E7C90000B2
:10C8F000E7C90000E7C90000E7C90000E7C9000078
:10C90000E7C900008FC90000E7C90000E7C90000BF
:10C91000E7C90000E7C90000E7C90000E7C9000057
:10C92000E7C9000087C900003B681B785B003A68D4
:10C930009268002A0CBF01220022D2B213431A4689
:10C940007B689A604FE03B689B68002B0CD13B688A
:10C950001B69002B02D06FF0200301E06FF0100381
:10C96000FA681340FB603EE03B685B68591C3A681C
:10C9700051601B781A467B689A603B689B685A1E18
:10C980003B689A602FE0FB6823F01003FB607B6834
:10C9900098683B68DB68591C3A68D160C2B21A706B
:10C9A0003B681B695A1E3B681A613B681B69012B77
:10C9B00018DDFB6823F00403FB6013E03B680122F1
:10C9C0001A75FB6823F01003FB600CE03B68022241
:10C9D0001A7508E03B6803221A75FB6823F0100300
:10C9E000FB6000E000BFFB6883F03C027B681A60DC
:10C9F0007B68FA689A61FB6803F01003002B03D090
:10CA00003B681B7D022B08D13B681B7D042B02D1A8
:10CA10003B6800221A75002300E0012318461037F6
:10CA2000BD4680BD80B582B000AF78607868FFF702
:10CA30002BFE0346702B0CD0702B04DC602B08D02F
:10CA4000682B06D00EE0A82B03D0B02B01D0782B9A
:10CA500008D17B689B68DBB219467868FFF751FE06
:10CA6000034600E0002318460837BD4680BDFFFF9F
:10CA700080B584B000AF786039603C23FB60002350
:10CA8000BB603B6804221A757868FFF7FDFD03461A
:10CA9000603B682B00F23A8101A252F823F000BFFC
:10CAA00077CC00000DCD00000DCD00000DCD0000B5
:10CAB0000DCD00000DCD00000DCD00000DCD00000E
:10CAC00077CC00000DCD00000DCD00000DCD000095
:10CAD0000DCD00000DCD00000DCD00000DCD0000EE
:10CAE00077CC00000DCD00000DCD00000DCD000075
:10CAF0000DCD00000DCD00000DCD00000DCD0000CE
:10CB000077CC00000DCD00000DCD00000DCD000054
:10CB10000DCD00000DCD00000DCD00000DCD0000AD
:10CB200045CC00000DCD00000DCD00000DCD000066
:10CB30000DCD00000DCD00000DCD00000DCD00008D
:10CB4000DBCC00000DCD00000DCD00000DCD0000B0
:10CB50000DCD00000DCD00000DCD00000DCD00006D
:10CB600045CC00000DCD00000DCD00000DCD000026
:10CB70000DCD00000DCD00000DCD00000DCD00004D
:10CB8000DBCC00000DCD00000DCD00000DCD000070
:10CB90000DCD00000DCD00000DCD00000DCD00002D
:10CBA000DBCC00000DCD00000DCD00000DCD000050
:10CBB0000DCD00000DCD00000DCD00000DCD00000D
:10CBC00099CC00000DCD00000DCD00000DCD000072
:10CBD0000DCD00000DCD00000DCD00000DCD0000ED
:10CBE00099CC00000DCD00000DCD00000DCD000052
:10CBF0000DCD00000DCD00000DCD00000DCD0000CD
:10CC0000A9CC00000DCD00000DCD00000DCD000021
:10CC10000DCD00000DCD00000DCD00000DCD0000AC
:10CC2000DBCC00000DCD00000DCD00000DCD0000CF
:10CC30000DCD00000DCD00000DCD00000DCD00008C
:10CC4000DBCC00007B6898683B68DB68591C3A685D
:10CC5000D160C2B21A703B681B695A1E3B681A61E8
:10CC60000523BB603B681B69012B4ADDFB6823F091
:10CC70000403FB6045E07B689B68DBB223F00103A3
:10CC8000DAB23B681A703B681B69012B3BDDFB681D
:10CC900023F00403FB6036E07B689B68DBB223F083
:10CCA0000103DAB23B681A703B685B68591C3A684A
:10CCB00051601B781A467B689A603B689B685A1ED5
:10CCC0003B689A603B689B68002B03DDFB6823F0A0
:10CCD0000403FB600623BB6018E00223BB60FB6813
:10CCE00023F00403FB603B6800221A753B681B7845
:10CCF00003F00103002B08D0FB6823F02003FB6046
:10CD000003E000BF02E000BF00E000BFFB6883F06B
:10CD10003C027B681A607B68FA689A61BB681846B7
:10CD20001037BD4680BD00BF80B485B000AF03465C
:10CD30000A46FB711346BB71FA791346DB009B1A56
:10CD40009B000B4A1344FB60BB79012B0AD1FB68A3
:10CD50001B691433BB6000BFBB681B78DBB2042BBC
:10CD6000FAD000E000BF1437BD4680BC704700BF5A
:10CD70009C00001080B584B000AF03460A46FB71EA
:10CD80001346BB71FA791346DB009B1A9B00104ACD
:10CD90001344FB60BB79012B15D1FB681B6914336D
:10CDA000BB600AE0FB79184600F002FA0346002B4C
:10CDB00003D0FB79184600F06BF9BB681B78DBB237
:10CDC000042BEFD000E000BF1037BD4680BD00BF90
:10CDD0009C00001080B582B000AF0346FB71FB7968
:10CDE0001846FFF7F7FBFA7906491346DB009B1A52
:10CDF0009B000B441B686C229A6100BF0837BD463C
:10CE000080BD00BF9C00001080B584B000AF034619
:10CE10003960FB71FB791846FFF7F4FB02463B686B
:10CE2000B2FBF3F3FB60FA7910491346DB009B1A5F
:10CE30009B000B441B68FA6852081A61FA790B4987
:10CE40001346DB009B1A9B000B441B681969FA7997
:10CE500006481346DB009B1A9B0003441B68FA68D4
:10CE6000521A5A6100BF1037BD4680BD9C000010A9
:10CE700080B485B000AF03463960FB71FA79134680
:10CE8000DB009B1A9B000B4A1344FB60FB681B6989
:10CE9000002B02D1FB683A689A60FB689B683A688D
:10CEA0009A420CBF01230023DBB218461437BD465B
:10CEB00080BC70479C00001080B584B000AF034672
:10CEC0003960FB71FA791346DB009B1A9B00204AFC
:10CED0001344FB60FB689B68FA790321104698476E
:10CEE0003B6804221A75FB683A681A61FB685B6943
:10CEF000002B04D1FB681B681846FFF795FBFB6805
:10CF00009B68FA79012110469847FB6800221A6154
:10CF100000BFFB681B681846FFF7A4FB0346002B05
:10CF2000F7D0FB689B6903F47F43002B04D0FB68B8
:10CF30001B681846FFF787FBFB689B68FA7904219A
:10CF4000104698473B681B7D18461037BD4680BD8C
:10CF50009C00001080B588B000AF3A601A460346C6
:10CF6000FB710B46BB7113467B7107F1080300226E
:10CF70001A605A609A60DA601A615A61BB793B7232
:10CF80003B68FB607B793B6100BF07F10802FB79DE
:10CF900011461846FFF790FF0346022BF5D07A7929
:10CFA0003B69D31A18462037BD4680BD80B588B08E
:10CFB00000AF3B600346FB710B46BB7113467B71B0
:10CFC00007F1080300221A605A609A60DA601A6159
:10CFD0005A61BB793B727B1DFB6001233B613B685F
:10CFE0007B61BB6ABB6100BF07F10802FB79114698
:10CFF0001846FFF761FF0346022BF5D0BB69BA6AFA
:10D00000D31A18462037BD4680BD80B58AB000AF20
:10D01000BA607B600346FB730B46BB7307F11003DA
:10D0200000221A605A609A60DA601A615A61BB7B0A
:10D030003B74BB68FB617B683B6200BF07F1100279
:10D04000FB7B11461846FFF737FF0346022BF5D04E
:10D050003B6A7A68D31A18462837BD4680BDFFFF61
:10D0600080B582B000AF0346FB71FA7907491346D9
:10D07000DB009B1A9B000B441B681846FFF711FB53
:10D08000034618460837BD4680BD00BF9C0000100F
:10D0900080B582B000AF0346FB71FA79134913469D
:10D0A000DB009B1A9B000B441868FA790F49134662
:10D0B000DB009B1A9B000B4410331B681946FFF7DB
:10D0C0006FFB0346002B0CD1FA7908491346DB00AD
:10D0D0009B1A9B000B4408331B68FA790221104607
:10D0E000984700BF0837BD4680BD00BF9C000010B8
:10D0F00080B586B000AF0346FB71FA791346DB00BA
:10D100009B1A9B00284A13447B617B695B69002B57
:10D1100018D17B691B681846FFF784FC0346FB7433
:10D12000FA79F97C13469B0013440B44DB001F4A39
:10D130001344FB60FB681A687B695A61FB685A6894
:10D140007B69DA607B695B691B785AB27B691B6912
:10D15000002B14BF01230023DBB25BB213435AB28E
:10D160007B695B69D2B21A707B691A687B695B69FB
:10D1700019461046FFF77CFCB860BB68002B0ED048
:10D180007B695B691B7D002B02D17B6900225A61A0
:10D190007B69DB68BA68D1B2FA791046984700BF5C
:10D1A0001837BD4680BD00BF9C00001030610010E4
:10D1B00080B483B000AF0346FB71FA790949134686
:10D1C000DB009B1A9B000B441B681B6803F00803E1
:10D1D000002B14BF01230023DBB218460C37BD46D9
:10D1E00080BC70479C00001080B586B002AFF8602C
:10D1F0007B600B46FB721346BB727B6898087B68AA
:10D20000DBB203F00303DBB2BA7AF97A0093034688
:10D21000F86800F004F800BF1037BD4680BD80B448
:10D2200087B000AFF8607B600B46FB721346BB72A1
:10D23000BB7A03F00F03DBB25B00FB75FB7A5B008C
:10D24000DAB2BB7A1B09DBB21344BB75BA7DFB684B
:10D2500053F82220FB7D032101FA03F3DB43134043
:10D260003B6197F82020FB7D02FA03F31946BA7D53
:10D270003B691943FB6843F82210BA7DFB68103202
:10D2800053F82220FB7D032101FA03F3DB43134013
:10D290003B61FB7D7A6802FA03F1BA7D3B69194371
:10D2A000FB68103243F8221000BF1C37BD4680BC1B
:10D2B000704780B586B000AFF860B9607A6000232F
:10D2C0007B611FE07B699B00BA6813441B78C3F342
:10D2D0000203DBB219467B699B00BA6813441B78D2
:10D2E000C3F3C403DBB218467B699B00BA681344DE
:10D2F0001B68C3F317230246F868FFF775FF7B69C5
:10D3000001337B617A697B689A42DBD300BF1837AF
:10D31000BD4680BD80B483B000AF78607B680C33BD
:10D320001A687B6810331B68D31A18460C37BD4641
:10D3300080BC704790B583B000AF78607B685C6854
:10D340007868FFF7E7FF0346E31A18460C37BD4637
:10D3500090BD80B582B000AF78607868FFF7DAFFE3
:10D3600002467B685B689A42ACBF01230023DBB2B4
:10D3700018460837BD4680BD80B483B000AF7860E2
:10D380007B680C331A687B6810331B689A420CBFA9
:10D3900001230023DBB218460C37BD4680BC704722
:10D3A00080B485B000AFF860B9607A603B60FB681C
:10D3B000BA681A60FB683A685A60FB687A689A60D3
:10D3C000FB6800221A61FB681A69FB68DA600123B6
:10D3D00018461437BD4680BC704780B584B000AF96
:10D3E000786039607B681B68FB607868FFF7B1FF85
:10D3F0000346002B01D0002319E07B68DB687A68C4
:10D400005268013A13407A68926802FB03F3FA68A3
:10D410001344FB607B689B681A463968F86800F023
:10D42000FCFC7B68DB685A1C7B68DA6001231846C9
:10D430001037BD4680BD80B588B000AFF860B960D8
:10D440007A60FB681B68BB61F868FFF782FF0346E0
:10D45000002B01D000237BE0F868FFF76BFF7861B9
:10D460007B69FB61FB68DB68FA685268013A1A4025
:10D47000FB691344FA68526893420AD3FB685B68FD
:10D480001946FB68DB68FA685268013A1340CB1A08
:10D49000FB617A69FB69D31A7B61FA697B68934205
:10D4A000A8BF1346FB617A68FB69D31A7B607A696F
:10D4B0007B689342A8BF13467B617A687B69D31A65
:10D4C0007B60FB68DB68FA685268013A1340FA68CF
:10D4D000926802FB03F3BA691344BB61FB689B6863
:10D4E000FA6902FB03F31A46B968B86900F095FCC3
:10D4F000FB68DA68FB691A44FB68DA60FB681A6843
:10D50000FB68DB68F968496801390B40F96889688C
:10D5100001FB03F31344BB61FB689B68FA6902FBE0
:10D5200003F31A46BB681344BB60FB689B687A69C7
:10D5300002FB03F31A46B968B86900F06EFCFB6899
:10D54000DA687B691A44FB68DA60FA697B6913441C
:10D5500018462037BD4680BD80B584B000AF7860E6
:10D5600039607B681B68FB607868FFF705FF03463E
:10D57000002B01D0002319E07B681B697A68526890
:10D58000013A13407A68926802FB03F3FA68134485
:10D59000FB607B689B681A46F968386800F03DFCC0
:10D5A0007B681B695A1C7B681A6101231846103777
:10D5B000BD4680BD80B588B000AFF860B9607A60C4
:10D5C000FB681B68BB61F868FFF7D6FE0346002BBB
:10D5D00001D000237BE0F868FFF79CFE78617B694F
:10D5E000FB61FB681B69FA685268013A1A40FB69E3
:10D5F0001344FA68526893420AD3FB685B68194681
:10D60000FB681B69FA685268013A1340CB1AFB6148
:10D610007A69FB69D31A7B61FA697B689342A8BF78
:10D620001346FB617A68FB69D31A7B607A697B6871
:10D630009342A8BF13467B617A687B69D31A7B60EB
:10D64000FB681B69FA685268013A1340FA689268ED
:10D6500002FB03F3BA691344BB61FB689B68FA6978
:10D6600002FB03F31A46B969B86800F0D6FBFB6801
:10D670001A69FB691A44FB681A61FB681A68FB683F
:10D680001B69F968496801390B40F968896801FB31
:10D6900003F31344BB61FB689B68FA6902FB03F365
:10D6A0001A46BB681344BB60FB689B687A6902FB3F
:10D6B00003F31A46B969B86800F0AFFBFB681A6952
:10D6C0007B691A44FB681A61FA697B69134418463E
:10D6D0002037BD4680BD80B483B000AF786039602C
:10D6E0007B683A681A6000BF0C37BD4680BC704743
:10D6F00080B483B000AF786039607B689A683B681B
:10D700001A437B689A6000BF0C37BD4680BC7047E7
:10D7100080B582B000AF78601020FEF77DFC7B689A
:10D720004FF0FF321A607B6800225A607B680C223F
:10D730009A607B680022DA6000BF0837BD4680BD72
:10D7400080B584B000AF786039601D20FEF758FDC9
:10D7500002460A4BA3FB02239A093B6802FB03F330
:10D76000FB60F9687868FFF7B6FF02217868FFF779
:10D77000BFFF00BF1037BD4680BD00BFD34D621054
:10D7800080B400AF064BD3F8883003F08073002BD1
:10D7900014BF01230023DBB21846BD4680BC70478E
:10D7A00000C00F4080B400AF064BD3F8883003F0C0
:10D7B0008063002B14BF01230023DBB21846BD4653
:10D7C00080BC704700C00F4080B400AF064BD3F858
:10D7D000883003F00073002B14BF01230023DBB259
:10D7E0001846BD4680BC704700C00F4080B400AFF3
:10D7F000054BD3F8A031044A43F02003C2F8A0310E
:10D8000000BFBD4680BC704700C00F4080B400AF71
:10D81000064BD3F8A03103F04003002B14BF0123C3
:10D820000023DBB21846BD4680BC704700C00F40E5
:10D8300080B483B000AF0346FB71044AFB79C2F8A1
:10D840000C3100BF0C37BD4680BC704700C00F4094
:10D8500080B500AFFFF7B8FF0346002B03D00221CD
:10D860000020FEF787FBFFF78BFF0346002B03D05A
:10D8700001210020FEF77EFBFFF7C8FF034683F07F
:10D880000103DBB2002B01D0FFF7B0FF00BFFFF7B1
:10D89000BDFF034683F00103DBB2002BF7D100206C
:10D8A000FEF7E6FB0120FFF7C3FF00220F21002057
:10D8B000FEF784FB01210020FEF73AFB0320FEF770
:10D8C000D7FB00BFFFF76EFF034683F00103DBB217
:10D8D000002BF7D102210020FEF72AFB00BF80BDFC
:10D8E00080B483B000AF78607B680C331A687B68C3
:10D8F00010331B689A420CBF01230023DBB2184689
:10D900000C37BD4680BC704780B483B000AF7860F0
:10D910000B46FB70FA787B681A6000BF0C37BD4677
:10D9200080BC704780B483B000AF78607B681B68B0
:10D93000DBB218460C37BD4680BC704780B483B05C
:10D9400000AF786039607B685A683B681A437B682F
:10D950005A6000BF0C37BD4680BC704780B483B0AE
:10D9600000AF786039607B685A683B68DB431A40D7
:10D970007B685A6000BF0C37BD4680BC704780B4DE
:10D9800083B000AF78607B689B6818460C37BD4653
:10D9900080BC704780B483B000AF786039607B682A
:10D9A0003A689A6000BF0C37BD4680BC704780B4AF
:10D9B00083B000AF786039607B683A68DA6000BF96
:10D9C0000C37BD4680BC704780B483B000AF786030
:10D9D0007B68DB6843F080027B68DA6000BF0C374D
:10D9E000BD4680BC704780B483B000AF78607B6870
:10D9F000DB6823F080027B68DA6000BF0C37BD462D
:10DA000080BC704780B483B000AF78600B46FB7079
:10DA10001346BB70FA787B681A60BA787B685A60E4
:10DA200000BF0C37BD4680BC704780B483B000AFE8
:10DA300078607B685B6918460C37BD4680BC7047D0
:10DA400080B483B000AF786039607B681A6A3B6845
:10DA50001A437B681A6200BF0C37BD4680BC704712
:10DA600080B485B000AF78607B680E4A934202D1E3
:10DA70000423FB730FE07B680B4A934202D1182307
:10DA8000FB7308E07B68094A934202D11923FB73B8
:10DA900001E00323FB73FB7B18461437BD4680BCB3
:10DAA000704700BF000001400080094000C00940ED
:10DAB00080B582B000AF78607868FFF760FF0346FA
:10DAC00003F48073002B11D04FF480717868FFF756
:10DAD000B7FF4FF480717868FFF740FF0E4B1B785B
:10DAE000DBB2002B02D10C4B01221A707868FFF7D1
:10DAF00046FF034603F40073002B09D04FF4007176
:10DB00007868FFF79DFF4FF400717868FFF726FFF4
:10DB100000BF0837BD4680BDA861001080B485B045
:10DB200000AF78607B680E4A934202D10423FB73F6
:10DB30000FE07B680B4A934202D11823FB7308E085
:10DB40007B68094A934202D11923FB7301E0032346
:10DB5000FB73FB7B18461437BD4680BC704700BF83
:10DB6000000001400080094000C0094080B584B039
:10DB700000AF78607868FFF773FF03461846FEF73A
:10DB80004BFA07217868FFF705FF786800F036F850
:10DB90007B6800225A607B680022DA607B68002282
:10DBA0001A627B680022DA647B6800225A657B680F
:10DBB00000221A657B680A4A934205D17B680022DD
:10DBC0001A617B689B69FB6003217868FFF7EFFEB1
:10DBD0007B6810229A6200BF1037BD4680BD00BF2F
:10DBE0000000014080B483B000AF78607B68802281
:10DBF0001A6300BF0C37BD4680BC704780B483B049
:10DC000000AF78607B6800221A6300BF0C37BD4606
:10DC100080BC704780B586B000AF786039607868A6
:10DC2000FFF77CFF03461846FEF7EAFA78613B6887
:10DC30001B017A69B2FBF3F33B613B691B0AFB6092
:10DC4000FB681B023A69D31ABB607868FFF7BCFE19
:10DC5000BB68DBB2FA68D2B219467868FFF7D2FE29
:10DC60007868FFF7C0FE7A693B69B2FBF3F31846A8
:10DC70001837BD4680BD80B584B000AF786039608C
:10DC80000AE07868FFF74EFE0346FB7307F10F03C7
:10DC900019463868FFF7A1FB7868FFF7C6FE034610
:10DCA00003F00103002BECD100BF1037BD4680BD4F
:10DCB00080B584B000AF7860396004E0FB7B194622
:10DCC0007868FFF721FE7868FFF7AFFE034603F0A0
:10DCD0002003002B08D007F10F0319463868FFF71F
:10DCE0003BFC0346002BE9D100BF1037BD4680BD89
:10DCF00080B586B000AFF860B9607A603B607B6841
:10DD00007B610221F868FFF729FE3A687969B868F3
:10DD1000FFF791FB03463B61B968F868FFF7C8FF5E
:10DD20007A693B69D1183A683B69D31A1A46B868D0
:10DD3000FFF781FB03461A463B6913443B6102210E
:10DD4000F868FFF7FBFD3B6918461837BD4680BDF4
:10DD500080B584B000AFF860B9607A603B603A6823
:10DD60007968B868FFF726FC034618461037BD46A9
:10DD700080BD80B584B000AFF860B9607A60FB68A0
:10DD80005B6803F00203002B0DD07968F868FFF799
:10DD90008FFF7868FFF7A4FD0346002B03D0022114
:10DDA000F868FFF7DBFDB968F868FFF764FFF8680B
:10DDB000FFF77EFE00BF1037BD4680BD80B483B044
:10DDC00000AF78607B6800221A607B68FF225A608F
:10DDD00000BF0C37BD4680BC704780B483B000AF35
:10DDE000786039603B6803F00403002B05D07B6842
:10DDF0001B6803F01B027B681A603B6803F0080392
:10DE0000002B05D07B681B6843F008027B681A6012
:10DE100000BF0C37BD4680BC704703F04FBB03F01A
:10DE200067BB03F073BB10B5425C4318342A01DCB6
:10DE3000002010BD352A06D1194611F8012F302ACD
:10DE4000FBD0002AF4D01A46302412F8011D3929DB
:10DE500001D11470F9E7013111700278302AE7D04E
:10DE60001A1A002A01DA0120E3E713F801299A704F
:10DE7000F6E730B50A258C1FA14200D130BD90FBDA
:10DE8000F5F3C3EB4312C3EB8202303000EB4200E8
:10DE900001F801091846EFE70EB430B594B017AB9E
:10DEA00053F8044B05463C22002105A80493FFF7D4
:10DEB000B8FF0A2308936FF000430793104B4FF00D
:10DEC000FF320293049B05A8CDE900436FF00043A5
:10DED000059500F049FD079B0446013B002B079385
:10DEE00008DB0022059B1A70204614B0BDE83040C4
:10DEF00003B0704705A9002002F0FAFAF4E700BF6A
:10DF000009DF0000FFFFFFFF2DE9F04F9DB00493F4
:10DF10000B68144606934B6881460593079347F6B2
:10DF2000F073059ADDF89CA033EA12432AD100234E
:10DF3000E370C2F31303069A13434FF06E031BD131
:10DF4000637066236922A370059B2270002B07DA99
:10DF5000AB4B0325269A136028461DB0BDE8F08F11
:10DF6000049B980706D4A74A13F0040FA64B18BFCA
:10DF70001346EEE7A54BECE761222370A3706270B5
:10DF8000A14BE6E720F02003412B00F0A982DDE958
:10DF900006010022002303F05BF8069E00283FD014
:10DFA000079B03F1004501230C9300220023304618
:10DFB000294603F037F8002840F08C8240F22D1BF0
:10DFC0000FAA3046294602F05CFB4FF47A730F9A91
:10DFD000CDE910010BFB02FBABF5AB5BABF11C0B0E
:10DFE0009BFBF3FB0020ABEB0202894902F074FBC0
:10DFF000BBF1000FCDE91A0115DA7BA3D3E90023A9
:10E00000CDE91623CBF10005E90714D4DDE91601AB
:10E01000DDE9162302F014FD6D10CDE91601F3E7DA
:10E02000059D0C90C1E74FF000027A4BCDE9162315
:10E030000BD05D46E8E7DDE91601DDE91A2302F0C1
:10E04000FFFC012DCDE91A01E0D1DDE91001DDE988
:10E050001A2302F07BFD0026CDE912016E4FDDE9A7
:10E06000120163A3D3E9002302F0F2FF002840F07D
:10E0700095800026684FDDE912015FA3D3E90023F4
:10E0800003F03AF8002840F09C80DDE9120102F02C
:10E090007DFF05468BEAEB73A3EBEB730D930F9AB1
:10E0A0002846ABEB020602F0B4FF324602F014FB46
:10E0B00000220023BBF1000FCDE91201CDE91423AA
:10E0C00080F2AC8048A3D3E90023CDE916230022D7
:10E0D0000023CDE91823DDE91667DDE916010026E6
:10E0E000DDE91823CDE9082332463B4602F0C6FDA0
:10E0F000DDE9082302F09AFECDE91801CDE91667A3
:10E10000DDE916010022434B02F09AFC02460B4661
:10E1100000203F4902F0B2FD00223E4B02F016FD06
:10E12000CDE91801DDF8348018F0010F40F08D8042
:10E13000DDE91623DDE91801DDE91867CDE90801FD
:10E140001046194602F072FEDDE9082302F06EFE69
:10E1500032463B4602F074FCCDE91801DDE91601B8
:10E16000DDE9162302F06CFCCDE91601DDE9166746
:10E17000DDE916010026DDE91823CDE90823324642
:10E180003B4602F07BFDDDE9082302F04FFE4FEA3B
:10E190006808CDE91801CDE91667C5E7DDE9120188
:10E1A00032463B4602F04CFCCDE91201DDE91A0192
:10E1B00032463B4602F0CAFC0BF1FF3BCDE91A01A7
:10E1C0004DE7DDE9120132463B4602F0BFFCCDE9E6
:10E1D0001201DDE91A0132463B4602F031FC0BF137
:10E1E000010BCDE91A0146E79A9999999999C93F86
:10E1F00000000000006AF8400000000080842E410A
:10E200008528010055280100D72801005328010066
:10E210000000F03F00001440000024404FF00002D6
:10E22000B94BCDE916234FF000024FF00003CDE9C2
:10E2300018237FF477AFDDE91201DDE9102302F046
:10E2400031FF002847D1013D29E7DDE91223CDE95F
:10E250000823DDE91823DDE91601CDE90A23DDE90C
:10E260001823DDE9146702F0E1FD32463B4602F077
:10E27000E7FBDDE90A2306460F46DDE9080102F067
:10E28000DFFB02460B463046394602F0CFFDCDE9B2
:10E290001401DDE91601DDE9122302F0D1FBCDE91D
:10E2A0001201DDE91267DDE912010026DDE9142320
:10E2B000CDE9082332463B4602F0E0FCDDE90823C5
:10E2C00002F0B4FDB8F1010FCDE91401CDE91267F8
:10E2D0007FF42EAFAFE7DDE91223DDE9100102F094
:10E2E000CDFCCDE91001DDE91423DDE9100102F0D8
:10E2F000C5FCCDE91001DDE91A23DDE9100102F0CA
:10E3000025FC7FA3D3E90023CDE91001DDE910014D
:10E3100002F096FBCDE91001DDE9100102F036FEB6
:10E32000DDE91067804602F074FE02460B46304677
:10E33000394602F0A3FC72A3D3E9002302F080FB6C
:10E34000CDE91001DDE9100102F020FE0646002EA5
:10E35000C0F28C806D4B9E4200F38F80B8F1000FAD
:10E36000C0F29280694B984500F39480684A9542C8
:10E3700000F39680674B0A2198FBF3F296FBF3F3C8
:10E38000654801FB052500FB028800FB036601FBD5
:10E3900008384E430BF1FF3B21463027284601F851
:10E3A000067BFFF766FD04F10C014046FFF761FDB7
:10E3B00004F112013046FFF75CFD002323750C9B2E
:10E3C0000BF1050BE77443EA8B0B1BF0010F00F018
:10E3D0008A80524B269A2BF0010B13600423B9F16B
:10E3E000610F9BFBF3FBDAF800500DD000F3A48023
:10E3F000B9F1450F00F0AC80B9F1470F00F0E781AB
:10E40000B9F1410F40F0E181059B0027C3F31301EF
:10E41000069B00201E461A46059B0F43C3F30A5174
:10E420000643002900F00A81A1F2FF30002D40F0E0
:10E430000B81049B1B0700F1078100290346384923
:10E44000384814BF31223022B9F1610F18BF01469C
:10E450002046FFF721FD314A079B3349054612EA62
:10E46000230338BF0B46269A136075E506F574261C
:10E4700006F5107608F1FF3869E7A6F57426A6F5CB
:10E48000107608F1010866E708F5742808F5107899
:10E49000013D63E7A8F57428A8F51078013562E717
:10E4A0009D427FF779AF0A226FF0090395FBF2F1E5
:10E4B00003FB01551D480BF1010B00FB058595FB86
:10E4C000F2F803FB085300FB0366053696FBF2F6F1
:10E4D0000D4661E700266FF0040BB04635465BE75A
:10E4E0004FF0000B71E7049B9A0706D4104A13F013
:10E4F000040F0D4B18BF13466CE70E4B6AE700BFC5
:10E500000000000080842E41000014403F420F00B4
:10E510009F860100A08601006079FEFF852801002A
:10E52000572801005F280100D728010040420F0052
:10E530005528010053280100B9F1660F00F06681EB
:10E54000B9F1670F00F04381B9F1650F40F03D81EB
:10E55000DAF80030112B05DD299A113B13601123E5
:10E56000CAF80030049BDAF8005013F4006605F195
:10E57000020504D129462046FFF755FC8344637801
:10E580002370DAF8003023B940F60803049A1A42DF
:10E590006CD02E236370299B1B68002BC2BF3E23C7
:10E5A0006355013576B1049B19070BD46219151B0D
:10E5B00012F8013D302BFAD03E2BF8D02E2B08BF9D
:10E5C00005F1FF35BBF1000FB6BF2D212B21CBF19B
:10E5D000000B6A1CBBF57A7F04F8059005F1020375
:10E5E000A1540ADB4FF47A729BFBF2F202F1300184
:10E5F000E1549C4B03FB02BBEB1CBBF1630F0ADD38
:10E6000064229BFBF2F202F13001E1546FF06301EE
:10E6100001FB02BB01330A229BFBF2F2D2B202F1F0
:10E620003001E1549D1C1C44C2EB4213C2EB830237
:10E630000BF1300B0BEB420262708DE456EA0703DC
:10E64000894808BF0020F1E60029029087498848E0
:10E6500014BF31223022CDE90067B9F1610F18BF34
:10E6600001462B462046FFF717FCF4E6012592E70A
:10E670005B449D1C122DC1BF299A113B13601325C9
:10E6800076B929462046FFF7CEFB48B17FEA0B0753
:10E6900005F1010504D1637823702E236370CDE06A
:10E6A000012F04EB05030CD11A1B002A02DC0135F3
:10E6B0003023F1E713F801299A70F5E713F80129DF
:10E6C000DA701A1B002AF9DC302323702E236370C2
:10E6D0003C23A370289B013F02351F60AEE00BEB8B
:10E6E0000307BD1C122D51DD8EBB13212046FFF701
:10E6F0009AFB60B314250BF1010B6A1E5A452346A1
:10E7000027DD5A7803F8012B1A1B9345F9DA2E22DC
:10E7100004EB0B035A70DAF80030299A5B44113B82
:10E720001360002B40F08F80002E44D0049B1A070A
:10E730003FF512AC6219151B12F8013D302BFAD0CF
:10E740003E2BF8D02E2B7FF407AC013D04E41325BB
:10E75000D3E7597803F8011B191B8A42F9DC3C22E4
:10E76000631903F8012CABEB050B289A0BF102039C
:10E7700013602E226255DAF800206B1C002A6CD040
:10E78000299902350A603E22E254CDE73EB9294676
:10E790002046FFF748FB10B10BF1010BFD1C23468F
:10E7A0005A7803F8012B1A1B9345F9DA2E23A34458
:10E7B0008BF80130B8E7DAF80030002B7FF4CCABEF
:10E7C000049B1B073FF5C8ABBFE74FF06709049BED
:10E7D000002D43F400630493DCBF0123CAF800302A
:10E7E000DAF8001020461129A8BF11210131FFF7E6
:10E7F0001AFBDAF8003083445B4528DD1BF1040F77
:10E8000025DB0BF101029B1ACAF80030049ABBF118
:10E81000000FDAF8003002F40066BFF660AFCBF10B
:10E8200000075A1CBA42BFF623AF302323702E23B1
:10E8300002256370DAF80030299A1360299B1B685F
:10E84000002B7FF771AF3E23635501356CE7013B29
:10E85000CAF80030A9F102097AE61D46002E7FF4BD
:10E8600065AFADE718FCFFFF01FCFFFF6728010063
:10E8700076280100F0B595B004460D4616460021F5
:10E880003C2205A81F46FFF7CCFA0A2308936FF035
:10E8900000430594002407930C4B6A1ECDE90173D5
:10E8A0000096234605A800F05FF8079B0546013B4C
:10E8B000A342079304DB059B1C70284615B0F0BDEE
:10E8C00005A9204601F014FEF7E700BF09DF0000AC
:10E8D0000FB473B506AB53F8046B0121324668469A
:10E8E0000193FFF7C7FF041E13DD651C284601F0E6
:10E8F0004FFF009068B1019B32462946FFF7BAFFEF
:10E90000074B22460099186DFCF75FFF009801F055
:10E91000A3FF204602B0BDE8704004B0704700BFBE
:10E92000B861001040EA01039B0770B50CD10446A2
:10E930000B46032A1946204606D906680D6804349A
:10E94000AE4203F1040304D00A44914203D10020F3
:10E9500008E0043AEDE710F8013B11F8014BA3423F
:10E96000F3D0181B70BDFFFF2DE9F04F9FB0CDE92C
:10E970000A23DDE92839002205460592187803F1BB
:10E98000010818B905981FB0BDE8F08F252819D0E7
:10E99000DDE90A67059B1946DA175C1C1346B1428C
:10E9A000BB4108DAAB68013B002BAB6006DB2B6890
:10E9B0005A1C2A60187005944346DFE7294601F087
:10E9C00097FDF8E7002409E02D2F04D0302F0FD158
:10E9D00044F4007401E044F00104B046464616F8E1
:10E9E000017B2B2F12D0EFD8202F12D0232F13D042
:10E9F0002A2F14D000230A21A7F13002D0B209280F
:10EA00001BD801FB032316F8017BF5E744F0020451
:10EA1000E3E744F00404E0E744F00804DDE709F12B
:10EA20000402D9F800309146002B98F80170BCBF61
:10EA30005B4284F0010408F1020623EAE3732E2FFF
:10EA40000D9334D137782A2F0FD000230A220136B4
:10EA50000693A7F13003D9B209290DD8069916F803
:10EA6000017B02FB01330693F3E7D9F80030777896
:10EA7000069309F104090236069B002B17DB44F0CC
:10EA800010046C2F0AD137786C2F03BF777844F0CD
:10EA900060040236013618BF44F020044C2F01D028
:10EAA000712F07D1377844F0600401360FE000235E
:10EAB0000693E6E7682F1FD13778682F03BF777872
:10EAC00044F480740236013618BF44F08004672F86
:10EAD0006DDC652F80F2B482472F00F0B18216DC26
:10EAE000412F00F0A782452F00F0AA82002F00F0EE
:10EAF0003881CDF83090C4E06A2F03D144F040044F
:10EB00003778D2E77A2FFBD0742FE0D1F8E7612F66
:10EB100000F0908220DC582FEBD1610640F1A781F4
:10EB200009F1070929F0070909F108030C93D9E94C
:10EB300000AB220640F1A4811FFA8AFA4FF0000BC5
:10EB4000B54B14F0080FB54A18BF1A46E00601D5B8
:10EB500024F40074B24BCEE1632F00F08D80642F5B
:10EB6000C7D1630640F14E8209F1070929F0070970
:10EB700009F108030C93D9E900AB200640F14B8260
:10EB80000FFA8AFA4FEAEA7BBAF1000F7BF1000331
:10EB900080F24782DAF1000AA24A6BEB4B0B14F0C9
:10EBA000100300F0A88124F400740023A3E1702F67
:10EBB00000F0978106DC6E2F00F0DB8000F3D5813A
:10EBC000692FCDE7752F00F0F681782F00F05E8178
:10EBD000732F8ED109F104030C93D9F800A0924B46
:10EBE000BAF1000F08BF9A46504601F0FCFA83467E
:10EBF000E00603D5069B9B45A8BF9B460D9BA3EB58
:10EC00000B0714F00103069313D1059A14F4007F47
:10EC10000CBF2023302390463C464FEAE279013C6A
:10EC200040F1C580059A27EAE7731A44013F05922F
:10EC3000FF1A059B002498464FEAE379AAEB030AE2
:10EC40005C45C0F2CF80059BBBF1000FA8BF5B44C1
:10EC50000593069B002B00F08780059B3C46984659
:10EC60004FF0200A4FEAE379013C40F1E680059B32
:10EC7000002FA8BFDB1939E009F10403D9F80070AF
:10EC80000C930D9B14F0010903F1FF3849D1059B4A
:10EC900014F4007F0CBF202430249A464FEAE37B13
:10ECA000B8F10108524623D5DDE90A01531C05934A
:10ECB00082424FEAE2738B4108DAAB68013B002BDA
:10ECC000AB6030DB2B685A1C2A601F70B9F1000F53
:10ECD0004AD0059B44469A4620274FEAE37B013CF5
:10ECE00026D5059BB8F1000FA8BF434405933BE030
:10ECF000DDE90A2392457BEB030308DAAB68013BAD
:10ED0000002BAB6008DB2B685A1C2A601C701AF1C0
:10ED1000010A4BF1000BC3E72946204601F0E8FB4E
:10ED2000F5E7059AC0E72946384601F0E1FBCDE753
:10ED3000DDE90A2392457BEB030308DAAB68013B6C
:10ED4000002BAB6008DB2B685A1C2A601F701AF17D
:10ED5000010A4BF1000BC2E72946202001F0C8FB55
:10ED6000F5E7013ECDF83090DDF83090059CB046D7
:10ED700021E609F104030C936106D9F8003005D5AA
:10ED8000059A1046D117C3E90001EDE7A20602D5A6
:10ED9000059A1A60E8E7E70503D59DF814201A7074
:10EDA000E2E72406F4D5BDF814201A80DCE7DDE99B
:10EDB0000A12884579EB020208DAAA68013A002AA9
:10EDC000AA6008DB2A68511C2960137018F1010839
:10EDD00049F1000923E718462946089301F088FB0A
:10EDE000089BF3E7DDE90A23904579EB03030BDA8F
:10EDF000AB68013B002BAB6018DB2B685A1C2A6008
:10EE00000AEB080212781A7018F1010804F10104E3
:10EE100049F1000914E700BF8E280100D72801003E
:10EE20009628010085280100872801000AEB0803C5
:10EE30002946187801F05CFBE6E7DDE90A239045F6
:10EE400079EB030309DAAB68013B002BAB6009DB0C
:10EE50002B685A1C2A6083F800A018F1010849F1B8
:10EE6000000901E72946202001F042FBF5E709F1FE
:10EE700004030C93D9F800304FF0000B9A4658E683
:10EE8000E3057FF55DAE0AF0FF0A57E661061AD585
:10EE900009F1070929F0070909F108030C93D9E9D9
:10EEA00000AB220618D51FFA8AFA4FF0000B7F4BF1
:10EEB00014F0080F7E4A18BF1A46E00601D524F464
:10EEC00000747C4B17E009F104030C93D9F800306F
:10EED0004FF0000B9A46E4E7E305E8D50AF0FF0A95
:10EEE000E3E74FF0000B09F104030C93D9F800306D
:10EEF0006E4A9A466F4B0599DDE90A89B8EB01081D
:10EF000069EBE1790699CDE90889CDE910124FF056
:10EF1000FF325521CDE91222002216A88154013278
:10EF2000202AFAD114F4826F04BF01221092672FB5
:10EF300000F3AA80652F08DA472F06D000F39A80E5
:10EF4000412F02D0452F40F0A88013AB039312ABA2
:10EF5000029310AB019311AB00933846234616AAD7
:10EF600014A92A9FB8470690BEE0610615D509F19D
:10EF7000070929F0070909F108030C93D9E900AB47
:10EF8000220613D51FFA8AFA4FF0000B484A4A4B63
:10EF900014F0080F18BF1A4601E609F104030C9398
:10EFA000D9F800304FF0000B9A46E9E7E305EDD5BC
:10EFB0000AF0FF0AE8E7600616D509F1070929F00B
:10EFC000070909F108030C93D9E900AB210614D510
:10EFD0001FFA8AFA4FF0000B14F0100302D000233E
:10EFE00024F40074324A86E709F104030C93D9F83B
:10EFF00000304FF0000B9A46E8E7E205ECD50AF046
:10F00000FF0AE7E709F104030C93D9F800309A46A8
:10F010004FEAE37BB1E5E1057FF5B6AD4FFA8AFA39
:10F02000B0E5A20704D414F0040F214A234BB1E742
:10F03000234AB4E5E3065EBF0D2344F010040693B3
:10F0400014F0100F069B08BF062309F1070929F0E9
:10F050000709069309F108030C93D9E90023CDE9C8
:10F060001423002344F480644FF0000A4FF0000B97
:10F070001A4640E7612F3FF468AF642F00F00A8121
:10F08000582F0AD100222BE0702FFBD008DC692F0B
:10F0900000F000816F2F00F09B800023069323E097
:10F0A000752F00F0F780782FEBE700BF9128010063
:10F0B000D7280100A7280100942801005528010045
:10F0C000532801000AF00F01595C16A881544FEA39
:10F0D0001A1141EA0B714FEA1B108A46834601322E
:10F0E0005AEA0B010692EDD114F480630E9300F0FE
:10F0F000D58000231093129B002BC4BF03F1FF3374
:10F100001093139B002B03DD109A013B13441093C3
:10F11000069B109F11981F4401F065F80D9B4FF05E
:10F120000008DF1B04F001030D9340F201231C4291
:10F13000A7EB000700F0DB80C2464FEAE87B119B9B
:10F140005A1C119293F80090B9F1000F40F0D6804C
:10F150000D9B83B914F4007F0CBF20233023C246DB
:10F160003C464FEAE87B013C40F1E48027EAE77344
:10F170007A1ED71A98440E9B002B00F0F68030249C
:10F18000069B4B4500F306810D9B5BB1C2463C4696
:10F190004FF020094FEAE87B013C40F19681002FB7
:10F1A000A8BFB844059B4344A0E50AF007023032EB
:10F1B00016A9CA544FEADA0242EA4B724FEADB015F
:10F1C00092468B4601335AEA0B020693EDD18BE748
:10F1D0000023F8E75FEA5B014FEA3A004FEA9A0240
:10F1E00042EA8B7210EB02084FEA9B0341EB0309E2
:10F1F0004FEA181242EA097218EB02004FEA19139B
:10F2000049EB030189464946020A42EA096280182D
:10F210004FEA112349EB03014FEA104848EA01483D
:10F2200018EB00024FEA114949EB0103002112EBF0
:10F23000030843EB01094FEAD80848EA4978A8FBDC
:10F240000C014FEAD9090CFB09111AF106024BF126
:10F250000003121A63EB0103CDE90623069B0AF1B2
:10F26000300A1809079B40EA037010EB08024FEAC6
:10F27000131141EB090302EB8201AAEB410A16A923
:10F2800001F807A09B46924601375AEA0B030697FE
:10F29000A0D129E700274FF00A0CF6E7069A109B49
:10F2A0009B1A0E9A48BF134631E7DDE908239045C3
:10F2B00079EB030309DAAB68013B002BAB6011DB90
:10F2C0002B685A1C2A6083F800B018F1010849F134
:10F2D0000009AAEB0803002BE7DA27EAE778AAEB94
:10F2E000080729E72946202001F002F9EDE74FF051
:10F2F000000907F1FF3A4FF0200BEAE7DDE90823A8
:10F3000092457BEB030308F1010809DAAB68013B86
:10F31000002BAB6009DB2B685A1C2A6083F8009035
:10F320001AF1010A4BF1000B09E72946484601F0A2
:10F33000DFF8F5E7DDE908128A457BEB020208DA1F
:10F34000AA68013A002AAA6008DB2A68511C2960D1
:10F3500013701AF1010A4BF1000B04E71846294615
:10F360000F9301F0C5F80F9BF3E7C24630244FEA34
:10F37000E87B109B013B002B10936DDAC246069C84
:10F380004FEAE87B002C00F38280069B002BA8BF8D
:10F390009844F9E616AB13F80900C2463C284FEA38
:10F3A000E87B31D03E2841D1139B013B002B1393C6
:10F3B0002FDBDDE9082392457BEB030308F101080D
:10F3C00008DAAB68013B002BAB602ADB2B685A1CC8
:10F3D0002A601C701AF1010A4BF1000BE4E7DDE929
:10F3E000082392457BEB030308F1010808DAAB68B8
:10F3F000013B002BAB600FDB2B685A1C2A601C7092
:10F400001AF1010A4BF1000B129B013B002B1293E6
:10F41000E5DA09F10109B3E62946302001F068F880
:10F42000EEE72946302001F063F8D3E7DDE9082351
:10F4300092457BEB030308F10108EADAAB68013B74
:10F44000002BAB6004DB2B685A1C2A601870E0E7C5
:10F45000294601F04DF8DCE7DDE9082392457BEB16
:10F46000030308F1010808DAAB68013B002BAB602D
:10F4700008DB2B685A1C2A601C701AF1010A4BF138
:10F48000000B76E72946302001F032F8F5E7DDE998
:10F49000082392457BEB03030CDAAB6816AA013B09
:10F4A0002244002BAB6012F8010C0ADB2B685A1CBB
:10F4B0002A6018701AF1010A04F1FF344BF1000BB5
:10F4C00060E7294601F014F8F4E7DDE908239245E6
:10F4D0007BEB030309DAAB68013B002BAB6009DB74
:10F4E0002B685A1C2A6083F800901AF1010A4BF12C
:10F4F000000B51E62946202000F0FAFFF5E700BF97
:10F500000A4B034493F880309A0605D53038884278
:10F51000A8BF4FF0FF3070471A0701D55738F6E7FC
:10F52000DB064CBF37384FF0FF30F0E7D82801003A
:10F530002DE9F84F804615460346894627491E4661
:10F5400016F8010B80B30A1892F88020D20724D451
:10F55000302829D158789E1C00F0DF02582A1ED18D
:10F5600035F0100724D110259878DE1C0024A2461F
:10F57000A3462946FFF7C4FF00281DDA0FB106F1A4
:10F58000FF38C9F80080BBF1000F24D022224FF0D1
:10F59000FF30134B1A60BDE8F88F3346CFE70127E1
:10F5A000002DE3D10825E1E725B92F460A25DDE73F
:10F5B0000127DBE70027D9E704FB0504230C0AFB3E
:10F5C000053ABAF5803FA4B228BF4FF0010B16F8F8
:10F5D000010B0127CDE744EA0A40DCE7D828010007
:10F5E000AC6100102DE9F74F0446914698464FF064
:10F5F000FF35DDF830A0654F009161686A1C013964
:10F600000029616057DB2168481C20600E78B91919
:10F6100091F88010C8074CD4711C00F0B280BAF188
:10F62000000F66DD19F0200F14D02B2E03D02D2EE5
:10F6300010D149F4007962680235013A002A62600B
:10F6400040DB2268511C21601678BAF1010B52D0C0
:10F650002A46DA46302E4CD1616849F48077013968
:10F6600000290AF1FF3B02F1010561602FDB2168EF
:10F67000481C20600E78BBF1000F34D026F020012A
:10F68000582930D138F010030FD16368AAF1020B6A
:10F69000013B002B02F1020563601FDB23685A1C4B
:10F6A00022601E784F464FF010084FF00009AB441F
:10F6B00037E01546A1E72046019200F03DFE019A91
:10F6C0000646A4E7204600F037FE0646BDE7204682
:10F6D000019200F031FE019A0646CCE7204600F088
:10F6E0002BFE0646DEE7B8F1000F08BF4FF0080812
:10F6F000DBE71546D346B8F1000F4F4608BF4FF081
:10F700000A08D2E7636847F48077013B002B09FBC6
:10F71000080905F1010563602BDB23685A1C226090
:10F720001E78ABEB0503002B05DD41463046FFF7A5
:10F73000E7FE0028E6DA2146304600F0D2FDFB0560
:10F7400021D5FE0711D4009BBC061B6807F00402FC
:10F7500003F1040103D5B80548BFC9F100090098B9
:10F7600001601B6852B1A3F80090284603B0BDE8C1
:10F77000F08F204600F0E0FD0646D2E7C3F8009087
:10F78000F3E73546F1E76FF00105EEE7D828010011
:10F7900000232DE9F04F04469BB0CDE902330F92D0
:10F7A0000D7801F1010B002D00F08880252DDFF888
:10F7B000A09347D009EB050292F880206368D60732
:10F7C00003F1FF3325D55A4612F8013B4B4493F819
:10F7D0008030D80713D46368013B002B636014DBCF
:10F7E00023685A1C2260187809EB000393F88030D4
:10F7F000D90706D4214600F074FD5946D0E7934658
:10F80000E1E7029B01330293E5E7204600F094FD17
:10F81000EAE7002B636009DB23685A1C22601E782C
:10F82000AE4208D1029B01330293E6E7204600F086
:10F8300083FD0646F4E73046214600F052FD0136CE
:10F840003CD171E14B7800272A2B06BF01F1020B56
:10F850004FF0010A4FF0000A5B460A20BB491BF833
:10F86000018B09EB080292F8802092062AD41AF044
:10F87000080F08BF6FF00047B8F16C0F2DD19BF84F
:10F8800000804AF0020A03F1020BB8F1670F00F39F
:10F89000AB80B8F1650F80F25D81B8F1580F00F0D0
:10F8A000CD832ADCB8F1450F00F05481B8F1470F41
:10F8B00000F05081B8F1250F00F0EF8003981BB0E5
:10F8C000BDE8F08F8F42F9DC00FB0788B8F1300704
:10F8D000F4D44AF0080A5B46C1E7B8F14C0F04D1F2
:10F8E0009BF800804AF0120ACDE7B8F1680FCCD13E
:10F8F0009BF800804AF0040AC5E7B8F1630F00F0F6
:10F90000E38000F31981B8F15B0FD7D19BF8005069
:10F9100000235E2D14BF002101214FF00100CDE92D
:10F920001233CDE91433CDE91633CDE918330ABFCC
:10F930009BF801500BF1010B0BF1020B002DBDD018
:10F940006A111AAB03EB820205F01F0300FA03F5FC
:10F9500052F8203C2B431BF8015B42F8203C5D2D04
:10F96000ECD149B1002312A951F82320D24341F828
:10F9700023200133082BF7D11AF0010609BF0F9B92
:10F980004FF000081A1D0F9208BFD3F8008063687B
:10F99000013B002B6360C0F2548323685A1C226031
:10F9A000187800254FF02009AF4214D0421C12D025
:10F9B00090FBF9F21AAB414203EB820201F01F0106
:10F9C00052F8202C00F01F0358BF4B4242FA03F3B9
:10F9D000DB0700F13D83214600F083FC002E40F060
:10F9E000A28288F800609EE2B8F1700F00F00583F3
:10F9F0000CDCB8F16E0F00F0EF8200F3FB82B8F17F
:10FA0000690F7FF45BAF0097002397E0B8F1750FA3
:10FA100000F01083B8F1780F00F01083B8F1730F85
:10FA20007FF44CAF4FF0FF3563680135013B002B8D
:10FA30006360C0F2E78223685A1C2260187809EBE1
:10FA4000000393F8806016F00106EDD1411C6BD0E5
:10FA50001AF0010808BF0F9B2F4402BF1A1D0F9216
:10FA60001E68BD4208D0421C06D009EB000393F883
:10FA70008030DB0740F1CA82214600F032FCB8F149
:10FA8000000F01D186F800801AF0010F02BF039B1E
:10FA900001330393029B2B44C6E66368013B002BB2
:10FAA00063600CDB23685A1C22601D78252D3FF40F
:10FAB000B9AE2146284600F014FC0135C0E62046C8
:10FAC00000F03AFC0546F1E71AF0080F08BF0127DD
:10FAD0001AF0010609BF0F9B00251A1D0F9208BFDF
:10FAE0001D68002F3FF4EAAE029B1F44029B0133C6
:10FAF00002936368013B002B636010DB23685A1C90
:10FB0000226018780EB928700135029BBB42EDD1F6
:10FB1000002E7FF472AE039B013303936DE6204603
:10FB200000F00AFC431CEDD1039B002B7FF4C6AE12
:10FB30004FF0FF330393C1E60A2300974AF02002F7
:10FB40000FA92046FFF74EFD0546ECE1CCCCCC0CCE
:10FB5000D82801004FF0FF38636808F10105013B28
:10FB6000002B6360C0F2D28023685A1C2260187890
:10FB700009EB000393F88030DE0700F1C580411CDB
:10FB8000D2D0002F00F0CC802B2800F0C3802D288D
:10FB900040F0C6804AF40076636808F10205013B34
:10FBA000002B6360C0F2B88023685A1C226018786A
:10FBB000013FB3A3D3E90023CDE9062300230022AC
:10FBC000CDE908230023B8461F460493B8F1000F7F
:10FBD00040F0A880214600F084FBDDE908010A23FB
:10FBE00003227B4393FBF2F3A7EB030842460E93F9
:10FBF00000F072FDCDE90A01049801F00AFA4246CC
:10FC000000F06AFD002FCDE9060180F252810FF26B
:10FC10007829D9E9008900229D4B4046494600F0E9
:10FC20000FFF02460B4600209A4901F027F80022F8
:10FC3000974B00F08BFFCDE904017F4200220023A7
:10FC4000CDE90823FA0738D5DDE9042340464946C3
:10FC500001F0ECF802460B46CDE90C01DDE90A01A2
:10FC600000F0EEFEDDE90823CDE90A01DDE90C0133
:10FC700000F0E6FEDDE90623CDE90801DDE9040137
:10FC800000F0DEFEDDE9082301F0D0F8DDE906230F
:10FC9000CDE908014046494600F0D2FE00220B465D
:10FCA000CDE9062300F0EAFFDDE9082301F0BEF804
:10FCB000012FCDE9080100F0038142464B46404642
:10FCC000494601F0B3F8DDE9042301F0AFF802463C
:10FCD0000B46DDE9040100F0B3FE4246CDE9040124
:10FCE0004B464046494600F0ABFE4FF000080B463D
:10FCF0004246894600F0C2FFDDE9042301F096F890
:10FD00007F10CDE904019DE7A84625E7204600F0D5
:10FD100013FB2DE756463FE7204600F00DFB47E773
:10FD2000564646E72E2811D172060FD446F04009F8
:10FD300063680135013B002B63603ADB23685A1C82
:10FD40002260187808F1FF384E463FE7524B0344D3
:10FD500093F880309B0630D5049B46F480791A4690
:10FD60004E4B06F040069A42A0F1300007DC0A2311
:10FD700003FB02030493002EDAD0013FD8E701F021
:10FD800048F9DDE9062300F05BFE02460B46DDE99B
:10FD9000080101F04BF80022CDE90801DDE9060178
:10FDA0003F4B00F0D3FECDE90601002EC0D1013754
:10FDB000BEE7204600F0C0FAC4E720F02002452A42
:10FDC00006F480737FF406AF002B3FF403AF636843
:10FDD00026F4C076013B002B63601EDB23685A1CAF
:10FDE000226018782B281ED02D281AD008F1FF3851
:10FDF00001354FF000090A22274BA844A8EB050162
:10FE0000002904DD191891F8801089061CD43106E8
:10FE10004CBFA7EB09074F44DCE6204600F08CFA04
:10FE2000E0E746F0800663680235013B002B636023
:10FE300006DB23685A1C22601878A8F10208D8E76C
:10FE4000204600F079FAF8E7616830380139002976
:10FE500046F4807602FB090905F10105616004DBC7
:10FE60002168481C20600878C8E720460A9206935B
:10FE700000F062FA0A9A069BC0E700BFAFF3008069
:10FE80009A9999999999B93F000000009999C93FA9
:10FE9000000014400000F03FD82801009F860100B8
:10FEA00000002440CDE904234FF00008DFF8D8918A
:10FEB000C4E64FF000024FF00003F3D1CDE9082370
:10FEC000DDE90823DDE90A0100F0B0FFDDE90623E2
:10FED00000F0ACFF11AA00F0D4FB119F0E9B8046EE
:10FEE0003B44B3F5806F89461F4611931FDD2222E4
:10FEF000614BD3E90078B305604B48BF08F1004877
:10FF00001A60F3057FF5DAACB00706F001092DD5CC
:10FF1000B9F1000F07D10F9B1A1D0F9219683A46CD
:10FF20004346C1E90023002DFFF6C7ADACE56FF4F1
:10FF30007F739F420ADA0022002301F073F828B988
:10FF400022224E4B07461A608046DAE73A46B7054A
:10FF50004046494605D500F0BFFB074601F1004881
:10FF6000CFE700F0B9FB07468846CAE712AA384631
:10FF7000414600F086FB129B7E33002B129313DC6C
:10FF8000002200233846414601F04CF8F8B92222FD
:10FF900000203A4B1A60B9F1000FC4D10F9B1A1D13
:10FFA0000F921B681860BEE7FE2B10DD00220023B5
:10FFB0003846414601F0A0F8314B324A002814BFC0
:10FFC0001846104622222D4B00681A60E3E7384697
:10FFD000414600F0B1FFDEE70F9B1AF0040F03F17A
:10FFE00004020F921B6815BFBDF80820029A1A8000
:10FFF0001A6002E400970823A0E5009710232AF076
:020000021000EC
:1000000006029DE5204600F097F918E5B8F1000FCB
:1000100001D13070013663680135013B002B63600C
:1000200004DB23685A1C226018781AE5204600F089
:1000300083F916E500970A23524681E500971023BD
:100040007CE5204600F078F9411C7FF4AAAC6BE512
:100050001EB988F8000008F1010863680135013B0A
:10006000002B636004DB23685A1C226018789BE431
:10007000204600F061F997E4B8280100AC61001057
:10008000F4000010F0000010000014400EB430B571
:1000900090B013AB53F8045B04463C22002101A846
:1000A0000093FDF7BEFE09232046CDE904340194F8
:1000B00000F099F8009A0290294601A8FFF768FB22
:1000C00010B0BDE8304003B07047FFFFF7B50746FA
:1000D0000E4601461A480D4615F8014B1CB303198C
:1000E00093F8803013F001031BD12B2C02D02D2C60
:1000F0001BD00D461C4601A92846FFF719FA26B168
:10010000019BAB4208BF3B4633608CB10028BDBFAA
:1001100022224FF000400B4B4042B8BF1A6003B0A0
:10012000F0BD2946D7E70D46E5E74FF40074E2E756
:100130000028BFBF2222034B6FF000401A60EEE799
:10014000D8280100AC61001038B5044C0A2225689B
:100150000021FFF7BBFF256038BD00BFAC61001078
:1001600040EA01039B0730B510D105460C462846EE
:100170002146036854F8042B04359A4206D1A2F1B3
:10018000013323EA020313F0803FF0D010F8013B63
:1001900011F8012B934201D0981A30BD002BF5D1F4
:1001A0001846FAE740EA01039B0710B513D102464F
:1001B000043951F8043FA3F1013424EA030414F094
:1001C000803F05D0D9B202F8011B59B11B12F9E7E3
:1001D00042F8043BEDE7421E11F8013B02F8013FF3
:1001E000002BF9D110BD10B5421C830716D1034670
:1001F00050F8041BA1F1013424EA010414F0803FFB
:10020000F5D011F0FF0F11D011F47F4F0CD011F485
:100210007F0F14BF03460333981A04E010F8013B24
:10022000002BE2D1801A10BD0233F5E70133F3E76A
:1002300040EA01039B0770B512D105460E46032A1A
:10024000314628460CD956F8044B036804359C42C5
:1002500006D1A4F1013323EA040313F0803F04D054
:100260000A44914203D1002008E0043AE7E710F87D
:10027000013B11F8014BA34201D0181B70BD002BAC
:10028000EFD11846FAE740EA010370B59D0724D183
:100290000E460346032A314608D956F8045BA5F1F9
:1002A000013424EA050414F0803F0FD0013A0139EB
:1002B000013B541C09D011F8014F9D1C561E03F838
:1002C000014F64B92A44954204D170BD43F8045BE0
:1002D000043ADFE705F8014BF5E70346E6E7324667
:1002E000E7E7431C15D0CB6813F402220FD123F4A7
:1002F000012323F0400343F40123CB608B6881F892
:1003000025008B634B68C1E901224B6370474FF0B6
:10031000FF30704738B50D46044608B9012A05D0AC
:1003200029462046BDE8384001F010B9FBF769FACC
:100330002870204638BDFFFFF8B5C36804461E0389
:1003400009D5426B23F400234260826BC360826054
:1003500090F82500F8BD9D0601D500F0A9F846F2F9
:10036000C902E3681A40012A0FD00022626044F2F9
:100370004002134276D023F4A04323F0400343F01D
:100380004003E3604FF0FF30E4E7474A13420CD1EB
:100390004FF4807000F078FA4FF48073E361E36803
:1003A000206143F400632060E3606268E368501CEE
:1003B0000DDA43F48053C2F1FF22E36002F57F02BD
:1003C0002368FE3262605A1C22601878C2E7D906A0
:1003D000676904D5DA033ED5204600F029F9E268C2
:1003E000E56942F48053E360D303266921684CD564
:1003F000E36A99422CBFC6EB0106C6EB0306AD1BB0
:1004000033D1204600F014F9E569E6692169761BCD
:100410000E44E3682A4623F01003E3603146384671
:10042000FFF778FF0028BEBFE36820F0004043F4E8
:100430008043A5EB0005B8BFE3607319E362E3698D
:100440002363E36835BB23F4805343F04003E36048
:10045000C4E9006596E7A169384601F079F80028FB
:10046000BDDAE36843F080038BE7104B1340002BA9
:10047000CBD1A1693846314401F06AF80028E3681D
:10048000F0DB43F40033E360BFE7A369891B194441
:10049000A161BEE7013D721C43F400336560226038
:1004A000E360307856E700BF000F01001000020043
:1004B000C36810B523F02003C3608269836A0446D1
:1004C0009A420ED000F0B4F8E36823F4405323F0CE
:1004D000100343F01003E360A36AA3612369E3629E
:1004E0002360E36823F4804323F04003E36010BDFE
:1004F000CB6870B523F400220C46CA609906054605
:1005000002D52046FFF7D4FFD4E902365A1C10DA90
:10051000B0050ED4C3F1FF2303F57F03FE33A360C0
:10052000236846F490365A1CE66022601D70E8B2DB
:1005300070BD41F28A023240022A07D0002346F001
:100540008006A360E6604FF0FF30F1E74AF2100347
:100550003340B3F5004F0AD10021204600F0A4F942
:10056000E368990602D52046FFF7A2FFE66846F445
:10057000903316F4706FE3600ED1606900F0E3FF12
:1005800000B372051ED504F1240323612360012307
:10059000E36146F49233E36013F4106F2168266937
:1005A00026D0E36A99422CBFC6EB0101C6EB0301DA
:1005B000B9B9731CE3622360E3695A1EA260236326
:1005C0003570B4E74FF4807000F05EF94FF480733B
:1005D000E268E36146F494331A4320612060E260EC
:1005E000DAE72246304600F09DF80028E1D0AAE77D
:1005F0004A1CEDB222600D70E26A216891422CBF64
:10060000C6EB0101C6EB0201E2695B05226303D47C
:100610000A2D01D08A4209DC0023E6622660A3602D
:100620002246304600F07EF800288CD128467FE72D
:1006300038B5044605690168C36AC06820F4002221
:10064000E26000F08202022A02D04FF0FF3038BD93
:1006500010F48030FBD0994238BF19468D4208D142
:100660000020E368E56223F480332560A060E36046
:10067000EDE72246491B284600F054F80028EFD049
:10068000E3E7F8B516460023002204460D4600F0C5
:10069000C9FC20B10023002000213360F8BDC5F360
:1006A0000A5320462946A3F2FE327BB9C5F3130351
:1006B000E70F03F4002547EA4303C3F31303640081
:1006C0000DB9013AF4E7204663F3130140F2FE331B
:1006D000326063F31E51E1E770B500231646002235
:1006E00004460D4600F09EFC10B10020002170BDB4
:1006F00040F2FE73C5F30A5232449A42204629461C
:1007000006DD2222054B1A60054BD3E90001EEE716
:10071000002AEADD62F31E51E9E700BFAC61001078
:10072000B82801002DE9F041D5688046EB020E465D
:100730001446576905D5384600F002FF45F010050C
:10074000A061124B2B408BB1A169384600F000FF2D
:10075000002806DAE3684FF0FF3043F08003E360DF
:1007600011E025F4003525F01005E56032464146DC
:100770003846FBF72AF820F00043F61AA3691E4416
:10078000A6610028E6D1BDE8F08100BF100002009C
:10079000F8B5304F3C68002851D10020F8BD2368DF
:1007A000B3F1805F39D1D4E9013151B10A68B2F1B6
:1007B000805F06D1DA1C4B681A448B686260A360C4
:1007C000F1E7AB4207DB9E4505DB20464FF00053C7
:1007D00040F80C3BE2E7634511D920464FF0005248
:1007E000656040F80C2B00EB8502A2604FF080544E
:1007F0005B1B033B40F82540C2E90131CEE761B9FC
:10080000A0EB830000F0F2F80130C6D04FF00053A7
:1008100004F10C00C4E90035C0E72646A468002CAA
:10082000BDD10C3000F0E2F8431CB6D04FF00053BD
:100830008460C0E9003556B938600C30AEE7C31C9F
:100840009D08002605F10A0C05F1030EE7E7B060EC
:10085000F3E700BFB4610010A8B14FF0805340F837
:100860000C3C50F8042C72B11368B3F1805F0AD1CC
:1008700050F8083C516803330B4440F8083C936837
:1008800040F8043CEDE7704710B5FFF781FF0446E0
:1008900028B917220349FAF798FF00F050FE2046C6
:1008A00010BD00BFC02801002DE9F843C6683D4BCC
:1008B000044633400D4690460BB9022747E0D0F876
:1008C0001490484600F03FFE07460028F5D1B8F1E5
:1008D000010F2CD0B8F1020F2ED0B8F1000FECD1DF
:1008E000002DEADBB00404D52368E26A9A4238BFDF
:1008F000E362A169A9420EDC2368E26A934238BF31
:10090000134622695818801AA84204DB206B01EBB9
:10091000000CAC4536DC0023C4E9013346F0200668
:10092000A56226F4032626F04006E6600FE0204686
:1009300000F03AF80544D3E7484600F001FEB0F174
:10094000000CE26806DA012742F08002E2603846D5
:10095000BDE8F883E36A1846A36919462368834211
:100960002CBFC91809180B4621699206A3EB010395
:1009700003D5A26A9342B8BF13466345ACBFED18D6
:100980006544ADE76D1AB10744BF281AA060F107AE
:1009900044BF9B1AEB1A154448BF6360256026F0DC
:1009A0002006BEE703001000C3689A0705D1212284
:1009B0000D4B4FF0FF301A60704703F020021B030D
:1009C00009D512B1806A01387047036882690069ED
:1009D0001344181AF7E70AB1806A704703688269FE
:1009E00000691344181A7047AC61001070B50B4DC4
:1009F0002B680BB90A4B2B60C41C2E6824F003042F
:100A00003444204600F010F810B92C60304670BD18
:100A10000C22044B4FF0FF361A60F7E7B06100106C
:100A20009C630010AC610010044B23B1984234BFAA
:100A30000020012070471846704700BF986B0010D7
:100A40002DE9F04F81EA0306C1F30A5740F2FF7522
:100A500006F00046002F5AD0AF4258D0C3F30A54D4
:100A6000002C54D0AC4252D04FEA525CC1F3130177
:100A700041F480114CEAC3234FEAC22843F0004CF2
:100A8000A1FB0823A8FB0089924627444A461C463E
:100A900000230025E0FB0C234FF0000B12EB0A00B3
:100AA0008246ECFB014543EB0B01601845F1000168
:100AB000B1F5801F4AEA98021DD2041841EB0105E6
:100AC0002946D30FA7F5806744EA03005200D30FED
:100AD000C41841F10005B2F1004F40F2FD72234607
:100AE00008BF24F00103974208D818462E4306EBAE
:100AF0000751BDE8F08FA7F2FF37E8E7002F03DBCF
:100B000046F0FF4646F4E00600203146F1E7490092
:100B100011F5001F12D25A0012F5001FF4D3094A32
:100B20005B0093420BD811424FF0000008D01342F3
:100B300006D046F0FF4141F4E001DAE7EFD00020B3
:100B40000149D6E70000E0FF0000F87F2DE9F043FF
:100B5000C1F30A5740F2FF7E83EA0104002F58D008
:100B6000774556D0C3F30A56002E52D0764550D062
:100B70009446BA1B460D46EAC12141F000474FEAB0
:100B80005C5141EAC32343F00049C6024FEACC2836
:100B90004F4508BF46452CD202F2FD315FEA5909A4
:100BA0004FEA3808352200234F4508BF46454FEA33
:100BB000430305D3B6EB080667EB090743F00103CF
:100BC000B6197F41212A08BF1D46013AECD14F4595
:100BD00008BF464502D3013308BF013540F2FD701E
:100BE000814204F000420AD802EB01525119184622
:100BF0000DE07F084FEA360602F2FE31CEE700290B
:100C0000A4BF42F0FF4242F4E00200201146BDE8DA
:100C1000F083184A4800904202D85D00954202D9FC
:100C200000201549F3E70B4312EA430301D11249AF
:100C3000DDE704F0004310EA020402D11946204621
:100C4000E5E72A4005D143F0FF4141F4E0011046B9
:100C5000DDE715F5001F05D043F0FF41002041F40A
:100C6000E001D4E710F5001F4FF00000D9D019467D
:100C7000CDE700BF0000E0FF0000F87F944693EA54
:100C80000102F0B405460E4606D503F100452B4699
:100C9000F0BC624600F0CAB88B4203D8844508D342
:100CA0008B4206D102F10042564053402A46654627
:100CB000944640F2FF71370D27F400628A42A7EB99
:100CC000135400F0A680944200F09F80C6F31302F4
:100CD000C3F313031F2C42F4801143F4801352D842
:100CE00023FA04F2891A2CFA04F2C4F12004A34076
:100CF00013439D42A5EB03022CBF0023012315469D
:100D000003B101391CFA04F303D05B42551E02B94A
:100D1000013911F4C01F57D1EA0FDB0F42EA41023B
:100D200043EA450352EA030470D0BC1E510B24D0A1
:100D3000510C01BF190F41EA02121B01043CD10CF6
:100D400001BF990F41EA82029B00023C110D02BFD4
:100D5000D90F41EA420204F1FF344FEAD67108BFCD
:100D60005B00B1EBD42F4FF0000006BF184602EB3A
:100D7000045106F00041F0BC7047190E41EA02220E
:100D80001B02083CD2E7352C1ED8203C23FA04F283
:100D90009542A5EB02002CBF00220122054602B1BC
:100DA0000139C4F1200293402CFA04F45FEA0C628A
:100DB00043EA040306D043F0FF035B42451E18B923
:100DC000013901E0002BF8D1CA0209D4013F7A05AC
:100DD0000FD0EA0F42EA4101DA0F42EA45055B0013
:100DE000002B21F480124FEA075405DB1119284625
:100DF000C1E739051046BEE7013508BF0132B3F13E
:100E0000004F08BF25F00105F0E75CB921462046F8
:100E1000B1E733034FF0000001D00349ABE70CB951
:100E20000149F4E73146E2E70000F87F93EA010F59
:100E3000F0B405460E4605D503F100452B46F0BC3F
:100E4000FFF71CBF8B4288BF1E4640F2FF7488BF6D
:100E50000B464FEA165184BF1546024621F4006046
:100E6000A0425ED0A1EB1354844255D0C6F31307C1
:100E7000C3F313031F2C47F4801743F4801327D8C0
:100E800023FA04F0074422FA04F0C4F12004A3403A
:100E90000343ED1828BF013702FA04F3BA022BD539
:100EA000013508BF01370BB925F00205360D3605AF
:100EB00006EB5706730013F5001F35BF31460020BF
:100EC000FF074B1C34BF47EA55001905F0BC7047BB
:100ED000352CE3D8203C23FA04F02D18C4F120006F
:100EE00003FA00F322FA04F428BF01372343120661
:100EF00018BF43F0FF03D1E7002B01F1FF3207DAFF
:100F0000013508BF0137B3F1004F08BF25F00105D7
:100F100007EB02512846D9E74CB906F000412046BC
:100F2000D4E733034FF0000001D00249CEE7314649
:100F3000F0E700BF0000F87F21F0004230B502F179
:100F4000474505F57005B5F17E6F01F000440FD2FD
:100F500002F14843420FC10042EAC30202EBD173DF
:100F6000B1F1004F08BF23F0010343EA040030BD94
:100F7000002D01DA2046FAE7490011F5001F94BF61
:100F800044F0FF400048F2E70000C07FCB0243EA94
:100F9000505040F21E43A3EB115340F00040FF2B92
:100FA00020FA03F011D913F4E06F01D140427047E9
:100FB00011F0804009D04B0013F5001F04D86FF0EA
:100FC000004000EBD17070470020704720B9034605
:100FD0000246104619467047030C0CBF000401F18D
:100FE0008071030E0CBF000201F50001030F0CBF5E
:100FF000000101F58001830F0CBF800001F5001195
:101000000028ACBF400001F5801101EBE023420550
:10101000DFE700F00041002801F18041B8BF404205
:10102000FFF7D4BF10B54C0054EA000C02D152EACD
:10103000430C09D0994209D1904207D114F5001F01
:101040008CBF0020012010BD0120FCE70020FAE742
:1010500030B5054651EA03000BD4580010F5001FC7
:101060001ED899421AD31BD195422CBF00200120D3
:1010700030BD480010F5001F12D85C0014F5001FA9
:101080000ED8284302D154EA0200F1D0994205D883
:1010900006D1954294BF00200120E9E70120E7E74F
:1010A0000020E5E730B551EA03040BD45C0014F5E9
:1010B000001F1FD899421BD31CD190428CBF002027
:1010C000012030BD4D0015F5001F13D85C0014F54C
:1010D000001F0FD899420BD801D1904208D255EA8F
:1010E000000307D154EA02030CBF01200020E8E707
:1010F0000120E6E70020E4E730B551EA03054FEAB6
:1011000041040AD414F5001F1ED899421AD81BD1E5
:10111000904234BF0020012030BD14F5001F13D8C9
:101120005D0015F5001F0FD899420BD301D19042F5
:1011300008D950EA040307D155EA02030CBF012085
:101140000020E9E70120E7E70020E5E7C0F3C75208
:1011500030B581EA00039AB3FF2A31D0C1F3C754F6
:1011600074B3FF2C2CD022440902040241F0004148
:1011700044F00044A4FB01452946002DA8BF6900A6
:1011800003F0004040EA11234FEA0161B4BF7F3A07
:10119000803AB1F1004F03EBC25304D0FD2A02D8CC
:1011A00003EBD17030BD01330CB923F00103FD2AEC
:1011B00001D81846F6E7002AF4DB40F0FF40F1E7DB
:1011C0004000B0F17F4F06D24A00B2F17F4F03D208
:1011D00003F00040E6E70CD14900B1F17F4F08D899
:1011E00010F07F4F05D011F07F4F02D003F0004088
:1011F000E3E70148D6E700BF0000C07F30B5C0F389
:10120000C75581EA0003CDB3FF2D37D0C1F3C752D4
:10121000A2B3FF2A32D00402090244F0004441F094
:1012200000418C42A5EB020532BF7D357E35640856
:10123000FD2D1CD8090AB4FBF1F201FB1244D80FB2
:10124000240202EBC030B4FBF1F201FB1244240291
:10125000B4FBF1F301FB134402EB002003EB00208D
:1012600000EBC550A1EB440100EBD17030BD002D67
:1012700003F00040FADB40F0FF40F7E74200B2F134
:101280007F4F13D84C00B4F17F4F0FD80843400074
:1012900010F07F4F0AD012F07F4F03F00040E5D0EE
:1012A000B4F17F4FE7D1B2F17F4FDFD10048DDE7E6
:1012B0000000C07F91EA000230B4034604D530BC80
:1012C00001F1004100F066B8814284BF02F10042A2
:1012D00053404FEAD35488BF5140E2B2FF2AA4EBF7
:1012E000D1554DD0954247D009021A0241F0004134
:1012F00042F0004221FA05F0121A13D502F1004221
:101300008032E00500EB1223120608D1C5F120005F
:1013100011FA00F20CBF23F0010303F1FF3318466A
:1013200030BC70475200002A18DADB0D8032DB0532
:1013300003EB2223120604F0FE0401D0002CEED1B0
:10134000C5F1200011FA00F20CBF23F0010303F1F4
:10135000FF33002CE3D103F00043E0E716D0B2FAEC
:1013600082F1A01E401AC00593EA000FF3D402FADE
:1013700001F300EB1323D2E7002D08BF2B46CEE785
:101380005A0201D1002DCAD1014BC8E70023C6E79C
:101390000000C07F91EA000F30B4024604D530BC93
:1013A00001F10041FFF786BF81429CBF0B46014619
:1013B0004FEAD15098BF1A46C3B2FF2B3BD0A0EBE7
:1013C000D2549C4232D012020B0242F0004243F04F
:1013D000004322FA04F55B190AD203F1004380337B
:1013E000C00500EB13211B0618D030BC084670471F
:1013F000013003F58073C50505EB5321DB05C0B251
:1014000001D0FF28F1D1C4F1200412FA04F308BF7F
:1014100021F00101FF2808BF2946E6E7C4F12004B6
:1014200012FA04F3E1D121F00101DEE7002CDCD156
:1014300001F00041D9E74B0218BF0149D5E700BFD1
:101440000000C07F78B1B0FA80F200FA02F3C2F176
:101450001F00803301EBC05000EB23201B0603D19B
:1014600020F0010070470020704700F00041002884
:1014700001F18041B8BF4042FFF7E4BF4FF0804127
:10148000FFF7E0BFC31013F07F610AD0B1F17F6FA7
:101490004FEA407243F0E04308D003F14841104660
:1014A000704703F0004300201946704752EA0332A8
:1014B000014A18BF1346F6E70000F87F40EA01032F
:1014C000DB0703460CD40346043A22BF51F804CB91
:1014D00043F804CBB2F10402F7D2043208BF7047DC
:1014E000013A24BF11F801CB03F801CBF8D87047BB
:1014F0008B18814238BF9842BFF4E0AF8141801819
:10150000013A0B5C00F8013DFAD87047034613F02E
:10151000030F0ED101F0FF0141EA012141EA01412F
:10152000043A24BF43F8041BB2F10402F9D202F1D9
:101530000402013A24BF03F8011BFAE77047FEE7F3
:101540004FF0FF3070474FF0FF3070471046704744
:101550004FF0FF307047FFFF454D414300FFFFFF55
:10156000000000004E657442756653656D00FFFF14
:10157000FFFFFFFFFFFF0000000000000806000162
:101580000800060400010000000000000000000048
:10159000000000000000FFFF4E657445766E740089
:1015A00049502D7461736B00FFFFFFFFFFFFFFFFCA
:1015B000000000000000000049444C4500FFFFFF10
:1015C000546D725100FFFFFF546D7220537663001B
:1015D000741200100030000000C0072000800000DE
:1015E000000000000000000073656C65637400007B
:1015F0000D0A546F6F206D616E7920616374697696
:101600006520636F6E6E656374696F6E732C206303
:101610006C6F73696E67210D0A0A00000D0A52751E
:101620006E6E696E67206C6F77206F6E206D656DD2
:101630006F72792C20636C6F73696E67210D0A439A
:101640006F6E736964657220636C6F73696E672077
:10165000756E7573656420636F6E6E656374696F14
:101660006E732E0D0A0A0000FFFD22FFFA2201010F
:10167000FFF00D0A0A436F6E6E6563746564207433
:101680006F202573200D0A25733E2000626174745B
:101690006572793E2000FFFF25733E2000FFFFFFAB
:1016A000636F6E74726F6C0075617274300000004D
:1016B0007561727433000000626174746572790040
:1016C000636F6D6D00000000736572636F6D6D0078
:1016D000332E312E3400FFFF73657474696E6720FA
:1016E000493243256420746F20706F6C6C696E679B
:1016F000206D6F64650A00FF62617425643A20669C
:1017000065740D0A00FFFFFF7475726E696E6720C5
:101710006F666620737461636B20626563617573C5
:1017200065206F6E20636F756E7420697320256469
:101730000A00FFFF232A242E48494C46450000009A
:1017400020403939414620202E2E2E2020547572FB
:101750006E206F6666207061636B732C2064697302
:1017600061626C6520616C6C207377697463686575
:101770007320200D0A000000204039394143202009
:101780002E2E2E2020456E61626C6520636861728A
:101790006765207377697463680D0A0020403939E2
:1017A000414420202E2E2E2020456E61626C652043
:1017B00064697363686172676520737769746368CD
:1017C000204120286D61696E290D0A0020403939B9
:1017D000424420202E2E2E2020456E61626C652012
:1017E000646973636861726765207377697463689D
:1017F00020422028415558290D0A0000204039393F
:10180000424620202E2E2E202044697361626C6592
:1018100020646973636861726765207377697463B4
:101820006820422028415558290D0A0020403939A6
:10183000434420202E2E2E2020456E61626C6520B0
:10184000646973636861726765207377697463683C
:101850002043202841555832290D0A0020403939AB
:10186000434620202E2E2E202044697361626C6531
:101870002064697363686172676520737769746354
:10188000682043202841555832290D0A00000000E5
:1018900020403F3F504620202E2E2E20205475728F
:1018A0006E206F6666207061636B203F3F2028309A
:1018B000302D3534290D0A0020403F3F504E202066
:1018C0002E2E2E20205475726E206F6E2070616354
:1018D0006B203F3F202830302D3534290D0A000081
:1018E00020403939525120202E2E2E202052657151
:1018F00075657374207374617475730D0A0000004C
:1019000020403F3F435620202E2E2E202047657436
:101910002063656C6C20766F6C74616765732066FC
:101920006F72207061636B203F3F2028332E34415B
:1019300068207061636B73206F6E6C79290D0A00EB
:1019400020403939534820202E2E2E2020507574E7
:10195000207061636B7320696E746F207368757497
:10196000646F776E206D6F6465200D0A00000000C3
:101970002057444F464620202E2E2E2020446973A7
:1019800061626C652063686172676520776174636A
:1019900068646F670D0A00002057444143542020BB
:1019A0002E2E2E2020456E61626C65206368617268
:1019B0006765207761746368646F670D0A000000D3
:1019C00020574452535420202E2E2E20205265732F
:1019D0006574207761746368646F670D0A000000A6
:1019E000426174746572792064617461206E6F74F1
:1019F000207265616479210A000000004039395382
:101A00004800000043616E27742074616B6520629A
:101A10006174746572792073656D6170686F726549
:101A2000210D0A005368757474696E6720706163D4
:101A30006B7320646F776E202E2E2E0020646F6EE5
:101A4000650D0A0057445253540000004368617208
:101A50006765207761746368646F6720726573657A
:101A6000742E0D0A0000000057444F464600000047
:101A7000436861726765207761746368646F67208B
:101A800064697361626C65642E0D0A0057444143BA
:101A90005400000043686172676520776174636871
:101AA000646F67206163746976617465642E0D0AE2
:101AB0000000000040393941430000005365747450
:101AC000696E672062617474657269657320746FF2
:101AD00020636861726765202E2E2E0040393941DF
:101AE0004400000053657474696E67206261747409
:101AF000657269657320746F2064697363686172CD
:101B00006765202E2E2E0000403939424400000027
:101B1000456E61626C696E6720415558202E2E2EED
:101B200000000000403939424600000044697361FA
:101B3000626C696E6720415558202E2E2E000000E1
:101B400040393941460000005475726E696E672055
:101B5000616C6C20626174746572696573206F6674
:101B600066202E2E2E0000004025326450460000D4
:101B7000696E76616C6964207061636B206E756D4F
:101B80006265720D0A0000007475726E696E6720DE
:101B90006F6666207061636B2025640A0000000098
:101BA00040253264504E00007475726E696E672075
:101BB0006F6E207061636B2025640A0040393952D2
:101BC000510000007175657279696E6720626174F9
:101BD0007465727920737461747573202E2E2E20B3
:101BE0000D0A00004E6F2061636365737320746F8C
:101BF00020626174746572792073746174757321E5
:101C00000D0A0000253032643A253034642C25302A
:101C100034642C253035642C253034642C25303345
:101C2000642C253034580D0A00000000456E763AC9
:101C3000253364432C253364432C253364252552F6
:101C4000480D0A004D656173313A253034642C2506
:101C50003034642C253034642C253034642C253009
:101C600034640D0A000000004D656173323A25337B
:101C7000642C2533642C2533642C2533642C2533C4
:101C8000640D0A005061636B747970653A203239D3
:101C90003C253032643E2C33343C253032643E0DDA
:101CA0000A0000004348473A2025642C2000000029
:101CB00044495343483A2025642C20004155583A62
:101CC0002025640D0A000000534D42555365727281
:101CD0003A256C752028256C7520756E7265636FCA
:101CE00076657261626C65290D0A000040253264D8
:101CF000435600007175657279696E672062617480
:101D0000746572792063656C6C20766F6C746167A2
:101D10006573202E2E2E200D0A000000253032641F
:101D20003A253034642C253034642C253034642C2E
:101D3000253034642C253034642C253034642C2533
:101D40003034642C253034640D0A0000535441545F
:101D5000530000006D696E20766F6C746167653AA0
:101D60002020202025362E3266560D0A6D617820FF
:101D7000766F6C746167653A2020202025362E32FC
:101D800066560D0A61766720766F6C746167653AF6
:101D90002020202025362E3266560D0A61766720D7
:101DA00063617061636974793A20202025362E3290
:101DB0006641680D0A746F74616C20637572726598
:101DC0006E743A202025362E3266410D0A746F74E7
:101DD000616C20706F7765723A20202025372E3293
:101DE00066570D0A0A616D6269656E742074656DCF
:101DF000703A20202025362E31662A430D0A687558
:101E00006D69646974793A202020202020202536CD
:101E10002E316625250D0A0068656C7000000000F3
:101E20000D0A2020257320636F6D6D616E64733A17
:101E30000D0A0A0062617564203C76616C75653E2E
:101E400020202020736574206261756420726174A3
:101E50006520746F203C76616C75653E20627073FE
:101E60000D0A00006D6F6465203C76616C75653EFF
:101E700020202020736574206D6F64653A203C77C4
:101E80006F72646C656E3E3C7061726974793E3C41
:101E900073746F70626974733E2028652E672E20FC
:101EA000384E31290D0A0000627265616B202020D6
:101EB000202020202020202073656E64206272651F
:101EC000616B207369676E616C0D0A006361636802
:101ED00065203C76616C75653E202020736574201A
:101EE0006361636865206D6F6465203C76616C7525
:101EF000653E2028303A2074696D65642C20313AA3
:101F0000206E65776C696E65290D0A0073746174C3
:101F100075732020202020202020202073686F77D8
:101F20002055415254206170702073746174757330
:101F30000D0A000073746174757320202020202026
:101F40002020202073686F77206261747465727935
:101F500020617070207374617475730D0A00000045
:101F60006170702020202020202020202020202090
:101F700073686F7720617070730D0A006170702054
:101F80003C76616C75653E20202020206D616E617D
:101F9000676520617070203C76616C75653E0D0A46
:101FA000000000006970203C76616C75653E202061
:101FB000202020207365742049502061646472657C
:101FC000737320287265717569726573204D43556E
:101FD000207265736574290D0A0000006E6D203C47
:101FE00076616C75653E202020202020736574206A
:101FF0004950206E65746D61736B20287265717530
:1020000069726573204D4355207265736574290D9F
:102010000A0000006777203C76616C75653E2020E1
:1020200020202020736574206761746577617920B2
:102030006164647265737320287265717569726575
:1020400073204D4355207265736574290D0A000095
:102050006D6163203C76616C75653E2020202020F8
:10206000736574204D41432061646472657373200D
:10207000287265717569726573204D4355207265CC
:10208000736574290D0A00007374617475732020E0
:10209000202020202020202073686F77206E657418
:1020A000776F726B207374617475730D0A00000092
:1020B000636C69656E74732020202020202020200E
:1020C00073686F7720636F6E6E65637465642063F9
:1020D0006C69656E74730D0A0000000072657365AB
:1020E000742020202020202020202020726573656D
:1020F0007420746865204D43550D0A00766572732F
:10210000696F6E20202020202020202073686F77A8
:102110002076657273696F6E0D0A0000706F7274BD
:10212000203C76616C75653E20202020736574200C
:1021300054435020706F72742028646973636F6E0B
:102140006E6563747320636C69656E7473290D0A20
:1021500000000000657869742020202020202020C5
:10216000202020206C65617665206D656E750D0AF6
:102170000000000061707000417070202874797058
:1021800065290D0A0A00000073657269616C000020
:102190002020257320282573290D0A004170702006
:1021A00027257327206973206E6F74206465666924
:1021B0006E6564210D0A000072657365740000008D
:1021C000726573657474696E67204D4355202E2EB9
:1021D0002E0D0A00636C69656E74730025752E25DB
:1021E000752E25752E25750028796F75290000003C
:1021F000282573290000000020205B25645D202530
:10220000732025730D0A0000706F727400000000C7
:10221000417267756D656E7420726571756972655E
:1022200064210D0A00000000496E76616C6964202B
:10223000706F72742027257327210D0A000000009B
:10224000436F6E74696E75696E67207573696E672A
:10225000206F6C6420706F727420272564270D0A2C
:1022600000000000506F72742027256427206973D6
:1022700020616C72656164792074616B656E2062A7
:10228000792027257327210D0A00000053657474F7
:10229000696E6720706F727420746F2025642C2023
:1022A000636C69656E74732077696C6C206265205D
:1022B000646973636F6E6E65637465642E0D0A00E6
:1022C000697000004E6F7420612076616C69642033
:1022D00049502061646472657373210D0A00000027
:1022E0004E657720495020616464726573732027BE
:1022F0002573272061637469766520616674657251
:10230000207265736574210D0A0000006777000074
:102310004E65772047572049502061646472657389
:1023200073202725732720616374697665206166B1
:10233000746572207265736574210D0A00000000D7
:102340006E6D00004E6F7420612076616C696420B0
:102350006E65746D61736B210D0A00004E65772008
:102360006E65746D61736B2027257327206163741C
:102370006976652061667465722072657365742183
:102380000D0A00006D6163004E6F7420612076615C
:102390006C6964204D4143206164647265737321EC
:1023A0000D0A28666F726D61743A2058583A585871
:1023B0003A58583A58583A58583A5858290D0A0035
:1023C0004E6577204D4143206164647265737320CC
:1023D0006973206163746976652061667465722033
:1023E0007265736574210D0A0000000073746174D6
:1023F00075730000506F72743A2020202020202036
:102400002025640D0A000000495020616464726553
:1024100073733A20202573200000000028257329BB
:102420000D0A00006E65746D61736B3A20202020E8
:102430002025732000000000676174657761793A98
:102440002020202020257320000000004D41432043
:10245000616464726573733A20253032783A2530AE
:1024600032783A253032783A253032783A2530328F
:10247000783A25303278200028253032783A2530D5
:1024800032783A253032783A253032783A2530326F
:10249000783A25303278290D0A000000766572738B
:1024A000696F6E004261744D616E3A2020202020D9
:1024B00025730D0A00000000424F4C4F0000000041
:1024C000426F6F746C6F616465723A2025730D0AF8
:1024D00000000000426F6F746C6F616465723A2097
:1024E0006E2F610D0A000000627265616B000000D2
:1024F00073656E64696E6720627265616B202E2E53
:102500002E0D0A006261756400000000496E76615C
:102510006C6964206261756420726174652027258E
:10252000732721204D6F7374206265206120706FC6
:1025300073697469766520696E74656765722E0DBE
:102540000A0A000053657474696E672062617564DD
:10255000207261746520746F2025642E0D0A0A00B4
:102560006D6F64650000000053657474696E6720C8
:102570006D6F646520746F202563256325632E0DC0
:102580000A0A00006361636865000000496E7661B5
:102590006C6964206361636865206D6F64652027E2
:1025A00025732721204D6F73742062652030206FC2
:1025B0007220312E0D0A0A0053657474696E67200B
:1025C0006361636865206D6F646520746F202563A7
:1025D0002E0D0A0A000000000D0A506F72743A2096
:1025E0002020202020202020202025640D0A00000B
:1025F000554152542073657474696E67733A202094
:10260000256C752025730D0A000000004361636886
:1026100065206D6F64653A202020202074696D6507
:10262000640D0A004361636865206D6F64653A203C
:10263000202020206E65776C696E650D0A00000011
:10264000545820746F74616C2062797465733A20F9
:10265000256C6C750D0A0000525820746F74616C03
:102660002062797465733A20256C6C750D0A000040
:102670005258206C6F73742062797465733A20200D
:10268000256C75200D0A0A000D0A506F72743A20ED
:102690002020202020202020202025640D0A0A0050
:1026A000657869740000000073617920776861744F
:1026B0003F0D0A00496E76616C6964206261756441
:1026C0002072617465210D0A202061636365707456
:1026D00061626C652076616C7565733A20313135C5
:1026E0003230302C2035373630302C2033383430EF
:1026F000302C2031393230302C2031343430302CF1
:1027000020393630302C20343830302C20323430E0
:10271000302C20313230302C203630302C203330E9
:10272000302C203131300D0A00000000496E7661F6
:102730006C6964206D6F64652076616C7565210D30
:102740000A20206578616D706C653A20384E310D35
:102750000A000000496E76616C696420776F7264CC
:10276000206C656E677468210D0A202061636365C3
:10277000707461626C652076616C7565733A2035A2
:102780002C20362C20372C20380D0A00496E76611B
:102790006C696420706172697479210D0A2020616E
:1027A000636365707461626C652076616C756573D6
:1027B0003A206E2C20652C206F0D0A00496E766140
:1027C0006C696420616D6F756E74206F6620737420
:1027D0006F702062697473210D0A616363657074A0
:1027E00061626C652076616C7565733A20312C20CE
:1027F000320D0A00001BB70000800000000A000034
:10280000080A00001009000018090000B0080000C4
:10281000B8090000010900000909000021090000B1
:102820004109000049090000510900007109000038
:10283000790900008109000089090000D909000018
:102840000406080A0E141C24282C3034383C40FF9F
:1028500007131A2B002000307825637025640030A0
:1028600058256350256400307825632E252E2A6C68
:102870006C7870256400305825632E252E2A6C6CE8
:1028800058502564002D00286E756C6C2900305856
:102890000030780030003031323334353637383953
:1028A00041424344454600303132333435363738BF
:1028B0003961626364656600FFFFFFFFFFFFEF7F22
:1028C0002A2A2A205F437379735F616C6C6F6320DF
:1028D0006661696C65640A00000000000000000089
:1028E00000000000000000000000000000000000E8
:1028F00000000000000000000000000000000000D8
:1029000000000000000000000000000000000000C7
:1029100000000000000000000000000000000000B7
:1029200000000000000000000000000000000000A7
:102930000000000000000000000000000000000097
:102940000000000000000000000000000000000087
:102950000000000000000000404040404040404077
:102960004041414141414040404040404040404062
:102970004040404040404040050202020202020244
:102980000202020202020202202020202020202037
:102990002020020202020202029090909090901079
:1029A0001010101010101010101010101010101027
:1029B00010101002020202020288888888888808A3
:1029C0000808080808080808080808080808080887
:1029D0000808080202020240000000000000000097
:1029E00000000000000000000000000000000000E7
:1029F00000000000000000000000000000000000D7
:102A000000000000000000000000000000000000C6
:102A100000000000000000000000000000000000B6
:102A200000000000000000000000000000000000A6
:102A30000000000000000000000000000000000096
:102A40000000000000000000000000000000000086
:082A500000000000000000007E
:102A5800AAAAAAAA00000000000008004500000079
:102A680000000000801100000000000031302E300E
:102A78002E302E31000000000000000031302E30D2
:102A88002E302E3200000000000000003235352EB6
:102A98003235352E3235352E30000000000C6A01F3
:102AA80003100101FFFFFFFF0000001000C00140FC
:102AB8000700000029CD0000000000000000000011
:102AC800000000000000000000C0054013000000E6
:102AD80029CD0000000000000000000000000000F8
:102AE8000000000000000A401A00000029CD000084
:102AF80000000000000000000000000000000000CE
:082B0800000080FF0000807F47
:040000030000214B8D
:00000001FF
